:100000000C946D0A0C948E0A0C948E0A0C94E50FD5
:100010000C941F100C948E0A0C948E0A0C948E0A69
:100020000C948E0A0C948E0A0C948E0A0C948E0AF0
:100030000C948E0A0C948E0A0C948E0A0C943A132B
:100040000C948E0A0C948E0A0C948E0A0C948E0AD0
:100050000C948E0A0C94F6640C948E0A0C948E0AFE
:100060000C948E0A0C9471650C948E0A0C948E0A72
:100070000C948E0A0C948E0A0C948E0A0C948E0AA0
:100080000C94EE780C948E0A0C948E0A0C948E0AC2
:100090000C94A0650C948E0A0C948E0A0C948E0A13
:1000A0000C948E0A0C948E0A0C948E0A0C948E0A70
:1000B0000C948E0A0C948E0A0C948E0A0C948E0A60
:1000C0000C948E0A0C948E0A0C948E0A0C948E0A50
:1000D0000C948E0A0C948E0A0C948E0A0C948E0A40
:1000E0000C948E0A0C942C6C0C94366C0C94226C30
:1000F0000C94E26B0C94626C0C94586C0C944C6CE9
:100100000C94406C0C948E0A0C948E0A0C948E0AFB
:100110000C948E0A0C948E0A0C948E0A0C948E0AFF
:100120000C948E0A0C948E0A0C948E0A0C948E0AEF
:100130000C948E0A1C7F3B7FB47FA680C680E6802D
:10014000EE809B80084AD73B3BCE016E84BCBFFD4E
:10015000C12F3D6C74319ABD56833DDA3D00C77F97
:1001600011BED9E4BB4C3E916BAAAABE0000008030
:100170003F07634236B79BD8A71A39685618AEBAFC
:10018000AB558C1D3CB7CC5763BD6DEDFD753EF690
:10019000177231BF000000803F08000000BE9224AB
:1001A00049123EABAAAA2ABECDCCCC4C3E000000E0
:1001B00080BEABAAAAAA3E00000000BF00000080DB
:1001C0003F0000000000084178D3BB4387D1133DB6
:1001D000190E3CC3BD4282AD2B3E68EC8276BED97F
:1001E0008FE1A93E4C80EFFFBE01C4FF7F3F0000BE
:1001F000000000000C94235B0C94AD720C94EA1088
:100200000C940E680C94A1770C94C9680C94176830
:100210000C9401660C943F6A0C94B6750C943D786E
:100220000C94E5730C94F9150C94EA730C9449370B
:100230000C94730E0C94B47F0C9447730C94EF736E
:100240000C9401890C94E6800C94EB1C0C94C978F6
:100250000C94E0730C94590E0C94F4730C940C4CA5
:100260000C9444670C9406150C949B800C94696B59
:100270000C94C6800C94EC690C945E850C940F4D24
:100280000C941C7F0C94B1820C94D7810C949F6DBC
:100290000C942E870C9499770C946E820C940282A5
:1002A0000C94A6800C94B9720C9427820C947D6CEB
:1002B0000C94FF850C944F670C9484690C947073B4
:1002C0000C9454660C94F7730C94B14C0C943B7FD3
:1002D0000C949E770C94A3730C9458780C948066BD
:1002E0000C94EE800C94C0786E616E00696E6600AE
:1002F00025630025730A005854414C5F5452494D00
:100300003D25640025730A0025730A005465737443
:1003100020362025730A0054657374203520257318
:100320000A005465737420342025730A00546573E1
:100330007420332025730A005465737420322025FD
:10034000730A005465737420312025730A006368B2
:10035000616E3D25640A0074787077723D25640AE9
:10036000003530306B0A003235306B0A00313135E0
:100370006B0A0035366B0A0033386B0A0025730AA6
:1003800000765F6C6F773D252D332E32660A00258F
:10039000730A0073656E743D252D75206475703D7C
:1003A000252D752069676E6F7265643D252D75205A
:1003B00074746C5F7A65726F3D252D750A00253760
:1003C0002E33662025372E33660025352E326620E3
:1003D000004572726F72203020566F6C74004E6F41
:1003E0007420737570706F727465640A0045727260
:1003F0006F72203020566F6C74004572726F7220DD
:100400003020566F6C740062756C6B5F64656C6154
:10041000793D252D750062756C6B3D252D75005657
:10042000616C7565206E6F7420616C6C6F776564AC
:100430000062756C6B3A206D61783D257520737490
:100440006172743D25752C20656E643D25752C20E8
:10045000696E5F7573653D25750A007062323D25D2
:10046000730A007062313D25730A00256C750041E6
:100470006C6C6F77656420737065656420312F3113
:10048000302F3130302F343030206B6269742F734D
:100490000025630074746C3D252D64200074746C19
:1004A0003D252D6420004E65772074746C3D252D0C
:1004B0006420002563004D533536313120503D25F1
:1004C0002D372E326620252D372E32666D0A0042DA
:1004D0004D5030383520256C642050612020252D6A
:1004E000372E32666D00256300545F484541545FE6
:1004F0004944583D252D352E32662000545F444531
:10050000573D252D352E3266200041483D252D359D
:100510002E32662000545F53485432583D252D3505
:100520002E3266200052485F53485432583D252DE4
:10053000352E32662000545F52483D252D342E3131
:1005400066200052483D252D342E3166200025635B
:100550000025630025630025630025630072657034
:100560006F72745F616C6C3D007265706F72743D88
:1005700000256300256300256300256300204F5399
:100580004343414C3D2564200020467573653A2065
:1005900065653D253032782068663D25303278200B
:1005A0006C663D25303278206C623D253032780013
:1005B0004D43553D2530366C780025630074785FD7
:1005C0006C656E3D252D6C752C765F6C6F773D25C7
:1005D0002D6C752C73687432783D252D6C752C62EA
:1005E000756C6B3D252D6C75002563004F4B0A0023
:1005F000256300256300256300256300256300252E
:10060000630025630025630064656275675F616C44
:100610006C3D0064656275673D0064656275673DA9
:100620000025730A00646565700A006E6F6E650AC6
:1006300000707772733D007062323D25730A00705E
:1006400062313D25730A00696E74725F7365635F82
:1006500070313D252D372E33660A00696E74725F46
:1006600070313D252D6C640A00696E74725F73658C
:10067000635F70303D252D372E33660A00696E7436
:10068000725F70303D252D6C640A00765F6D637576
:100690003D252D352E32660A00745F6D63753D254C
:1006A0002D352E32660A00707077723D25730A0070
:1006B00064656275673D0072636D643D25730A0071
:1006C00025730A006175746F0A006C6F675F6D6F48
:1006D00064653D007573625F7077723D25730A0033
:1006E00072656C61793D25730A0074746C3D252D2B
:1006F000640A0052494D455F616464723D252D6472
:100700002E252D640A006E65696768626F725F74DA
:1007100061626C655F73697A653D25640A00765F86
:100720006C6F773D252D332E32660A007478707712
:100730003D25640A006368616E3D25640A006964B2
:100740003D006932635F6275733D006932635F73B8
:10075000706565643D252D6C750A007478743D25BF
:10076000730A0053797374656D2053756D6D6172F2
:10077000790A002530366C780041744D6567613226
:100780003536524652320041744D65676131323818
:10079000524652320041744D6567613634524652BA
:1007A000320041744D656761313238524641310043
:1007B0004D43553D006D61736B3D002C00696E74B7
:1007C000657276616C3D252D750023252D642C0006
:1007D0007062320070623100745F686561745F69D5
:1007E000647800745F64657700616800705F6D73A2
:1007F000353631310072685F736874327800745F27
:100800007368743278007061007000616434006154
:10081000643300616432006164310061330061322D
:1008200000613100765F696E007268006572720067
:10083000757074696D650070315F6C737400703130
:100840005F740070310070305F6C73740070305FE3
:100850007400703000765F6D637500745F6D637552
:100860000074310074006964006536340074787473
:10087000002D002B006175746F006E6F6E65006255
:10088000756C6B00706F7765725F736176655F6C16
:10089000656472790072656C61795F6C656479007A
:1008A000636F6D7061737300616363656C00707278
:1008B000657300705F707772006165730070315FFF
:1008C0006C6564790070305F6C6564720065766594
:1008D0006E74006C6564006F7700706B74007478E0
:1008E0005F6C6564790072785F6C656472006F702C
:1008F0006572006E6F6E65002530327800765F613C
:1009000064343D252D382E3666002000765F616404
:10091000333D252D382E3666002000765F61643227
:100920003D252D382E3666002000765F6164313D0E
:10093000252D382E3666002000765F6C6967687456
:100940003D252D382E3666002000765F61323D252C
:100950002D372E3366002000765F61313D252D371F
:100960002E3366002000765F696E3D252D352E32D0
:100970006600204E657665722D757365642073740C
:1009800061636B203E2025642062797465730A00E0
:10099000757074696D653D252D642D646179732DC5
:1009A000253032643A253032643A253032642D687D
:1009B0006F7572730A0074657374205B6F66667C72
:1009C000317C327C337C347C355D2020202020201B
:1009D00020202D2074657374206D6F6465730A0D7B
:1009E000007478205B706B74207061796C6F616447
:1009F0005D2020202020202020202020202D20735A
:100A0000656E6420726164696F20706B74206B6521
:100A100079626F6172640A0D00776474205B6F6E97
:100A20007C6F66667C746573745D202020202020B6
:100A300020202020202D207761746368646F670A6E
:100A40000D00765F6C6F77205B765F6C6F775D2053
:100A500020202020202020202020202020202D2089
:100A60006C6F77657374207265706F727420766F27
:100A70006C746167650A0D00757067722020202014
:100A80002020202020202020202020202020202066
:100A9000202020202D207265626F6F74207669619E
:100AA00020626F6F746C6F616465720A0D0075610E
:100AB0007274205B33386B7C35366B7C3131356B2F
:100AC0007C3235306B7C3530306B5D202D2073658A
:100AD00074207465726D2F75617274207370656512
:100AE000640A0D00626F6F742020202020202020D7
:100AF00020202020202020202020202020202020F6
:100B00002D207265626F6F740A0D0070777273200A
:100B10005B646565707C6E6F6E655D2020202020B3
:100B2000202020202020202D206D637520736C65EF
:100B30006570206D6F64650A0D00726573742065C1
:100B40006570726F6D202020202020202020202022
:100B50002020202020202D20726573746F72652064
:100B6000656570726F6D0A0D0070707772205B6F33
:100B70006E7C6F66665D20202020202020202020B3
:100B800020202020202D2070726F6772616D6D61B2
:100B9000626C65207077720A0D0070623220205BF3
:100BA0006F6E7C6F66665D20202020202020202034
:100BB0002020202020202D2070726F6772616D6DC3
:100BC00061626C652070696E2062320A0D0070628D
:100BD0003120205B6F6E7C6F66665D2020202020B8
:100BE000202020202020202020202D2062756C6BCA
:100BF000204750494F2070696E0A0D0074787420A8
:100C00005B737472696E675D202020202020202095
:100C100020202020202020202D2053657420726564
:100C2000706F7274207465787420737472696E6763
:100C30000A0D0074787077205B31352D305D2020EF
:100C40002020202020202020202020202020202D97
:100C5000205458205077722E204869676865737455
:100C6000203020283364426D290A0D0074746C20F2
:100C70005B302D31355D20202020202020202020B9
:100C800020202020202020202D2074696D652D74C7
:100C90006F2D6C69766520666F72207061636B657D
:100CA00074730A0D00737320202020202020202040
:100CB0002020202020202020202020202020202034
:100CC000202D2073797374656D2073756D6D61725D
:100CD000790A0D007273202020202020202020205F
:100CE0002020202020202020202020202020202004
:100CF0002D20726164696F2073746174730A0D0032
:100D00007269205B236E5D205B696E745D2020201C
:100D10002020202020202020202020202D2072652F
:100D2000706F727420696E74657276616C0A0D0062
:100D300072636D64205B6F6E7C6F66665D20202041
:100D40002020202020202020202020202D20616C09
:100D50006C6F7720636D642066726F6D206E6574B2
:100D60006F726B0A0D007265205B236E5D205B2B3A
:100D70007C2D5D205B6D61736B7C6175746F2C6D78
:100D800061736B5D202D206D6F7465207265706FCF
:100D90007274207365742F6D6F646966790A0D0033
:100DA0006F7720202020202020202020202020209D
:100DB0002020202020202020202020202D206F6E89
:100DC000652D776972652073656E736F72730A0D96
:100DD000006C6F67205B6175746F7C6F6E7C6F66F3
:100DE000665D20202020202020202020202D206D26
:100DF0006F7465732064617461206F6E2055534277
:100E00000A0D006E65205B666C7573685D2020209E
:100E10002020202020202020202020202020202DC5
:100E2000206E65696768626F72207461626C650A22
:100E30000D006572722020202020202020202020FC
:100E400020202020202020202020202020202D2095
:100E50006572726F722073746174730A0D006D6332
:100E6000752020202020202020202020202020202D
:100E7000202020202020202020202D206D63752080
:100E8000696E666F0A0D00693263205B70726F6273
:100E9000657C737065656420236E5D2020202020B2
:100EA0002020202D206932632070726F62652062DD
:100EB00075737C73657420627573207370656564E7
:100EC0000A0D006964205B72657365745D202020E3
:100ED0002020202020202020202020202020202D05
:100EE0002069642068616E646C696E670A0D006831
:100EF000756D202020202020202020202020202050
:100F000020202020202020202020202D2068756DEA
:100F100069646974792073656E736F720A0D00726B
:100F2000656C6179205B6F6E7C6F66667C73746143
:100F300074735D20202020202020202D2072656CDD
:100F40006179206E6574776F726B207265706F7255
:100F500074730A0D006465205B6D61736B5D202006
:100F60002020202020202020202020202020202081
:100F7000202D2064656275670A0D006368616E202C
:100F80005B31312D32365D20202020202020202092
:100F9000202020202020202D206368616E20313108
:100FA0002D32362028322E3430352D323438302050
:100FB0004D687A290A0D0063616C69205B5B765F7E
:100FC000696E7C61317C61325D20766F6C747C72FD
:100FD000657365747C6E6F6E655D202D2063616C3A
:100FE0006962726174650A0D0062756C6B205B5BEF
:100FF00073686F777C666C7573685D205B7365746E
:101000002074687273682064656C61795D5D20206E
:101010002D2062756C6B696E67207061636B6574FF
:1010200073200A0D006164632020202020202020EE
:1010300020202020202020202020202020202020B0
:10104000202D2073686F7720765F696E2C206131C8
:101050002C20613220766F6C74616765730A0D0015
:10106000752020202020202020202020202020202B
:101070002020202020202020202020202D207570BE
:1010800074696D650A0D0076202020202020202024
:101090002020202020202020202020202020202050
:1010A0002020202D2076657273696F6E0A0D00680E
:1010B0002020202020202020202020202020202030
:1010C00020202020202020202020202D2068656C3A
:1010D000700A0D00256300756E6B6E6F776E20636E
:1010E0006D640A00484D43353838330025730025B8
:1010F0007300202573002025362E3266200025300F
:1011000032780074656D705F65787465726E3D2528
:101110002D362E326600202573002025362E3266AD
:10112000204F6E2D426F617264002530327800745A
:10113000656D705F626F6172643D252D362E32667B
:10114000000A0042756C6B2072656D3A2073746101
:1011500072743D25752C20656E643D25752C2069C3
:101160006E5F7573653D25750A0042756C6B206175
:1011700064643A2073746172743D25752C20656E29
:10118000643D25752C20696E5F7573653D25750A74
:101190000042756C6B207468726573683A207469DC
:1011A0006D65723D25750A00503A20256C6420500B
:1011B000612020252D372E3266206D0A00493243EA
:1011C0003A20004A54414720726573657474210ABD
:1011D000005761746368646F67207265736574217A
:1011E0000A0042726F776E6F757420726573657452
:1011F000210A0045787465726E616C2072657365B2
:1012000074210A00506F7765722D6F6E20726573BE
:101210006574212E0A004F6E6C696E650A00526F6C
:101220007574696E6720456E61626C65640A005270
:10123000504C20456E61626C65640A002573202560
:10124000732C206368616E6E656C202575202C20E0
:10125000636865636B207261746520257520487A28
:1012600020747820706F7765722025750A000A2A2D
:101270002A2A2A2A2A2A426F6F74696E67202573E8
:101280002A2A2A2A2A2A2A0A004A54414720726511
:10129000736574210A005761746368646F67207214
:1012A00065736574210A0042726F776E6F757420E2
:1012B0007265736574210A0045787465726E616C9D
:1012C000207265736574210A00506F7765722D6F07
:1012D0006E2072657365742E0A00726E67206973E2
:1012E000737565732025640A00454550524F4D20A3
:1012F000697320636F72727570742C2072657772D7
:101300006974696E672077697468206465666175C1
:101310006C74732E0A006C6F63616C686F73740079
:1013200041544D45474132353672667232000200F3
:1013300000FFFE000001452025642E256420636C1B
:101340006F636B20256C752063707520256C75208C
:101350006C706D20256C752069727120256C75206C
:10136000676C656420256C7520796C656420256C3C
:101370007520726C656420256C7520747820256C4E
:1013800075206C697374656E20256C752073656EAD
:10139000736F727320256C752073657269616C20A0
:1013A000256C750A0000407A10F35A00A0724E189E
:1013B000090010A5D4E80000E87648170000E40B07
:1013C00054020000CA9A3B000000E1F505000080CD
:1013D000969800000040420F000000A08601000027
:1013E00000102700000000E8030000000064000077
:1013F0000000000A00000000000100000000002CB6
:1014000076D888DC674F0823DFC1DFAE59E1B1B77A
:1014100096E5E3E453C63AE651997696E8E6C28447
:1014200026EB898C9B62ED407C6FFCEFBC9C9F405F
:10143000F2BAA56FA5F490055A2AF75C936B6CF984
:10144000676DC11BFCE0E40D47FEF520E6B500D05A
:10145000ED902E0300943577050080841E0800006F
:10146000204E0A000000C80C333333330F986E123D
:10147000831141EF8D2114893BE65516CFFEE6DB43
:1014800018D1844B381BF77C1D901DA4BBE424208D
:101490003284725E228100C9F124ECA1E53D274E21
:1014A000414E494E495459494E46CDCCCC3D0AD7C0
:1014B000233C17B7D13877CC2B329595E6241FB152
:1014C0004F0A000020410000C84200401C4620BCDA
:1014D000BE4CCA1B0E5AAEC59D7411241FBECFEF61
:1014E000D1E8DEBFCDBF00E00CBF1AE0A0E0B2E063
:1014F000E0E6FCE201E00BBF02C007900D92A634CB
:10150000B107D9F729E3A6E4BAE001C01D92AD3FC7
:10151000B207E1F70E94D0630C942E960C94000061
:101520002F923F924F925F926F927F928F929F92F3
:10153000AF92BF92CF92DF92EF92FF920F931F93E1
:10154000CF93DF93CDB7DEB763970FB6F894DEBFC6
:101550000FBECDBF6C014B012A01FC011782168220
:10156000838181FF43C3AE014F5F5F4F3A01F601B4
:101570009381F40193FD859193FF81914F0188231D
:1015800009F430C3853239F493FD859193FF81913D
:101590004F01853239F4B60190E00E94FA9252016F
:1015A0002501E5CF10E0F12C20E02032A0F48B32B1
:1015B00069F030F4803259F0833269F420612CC034
:1015C0008D3239F0803339F4216026C022602460E6
:1015D00023C0286021C027FD27C030ED380F3A30E6
:1015E00078F426FF06C0FAE01F9F300D1124132F58
:1015F00013C04AE0F49E300D1124F32E20620CC07B
:101600008E3221F426FDEEC2206406C08C3611F421
:10161000206802C0883641F4F40193FD859193FF60
:1016200081914F018111C1CF9BEB980F933018F43A
:101630002061805E06C09BE9980F933008F071C16D
:101640002F7E26FF16E02F73322E853619F4206484
:10165000322E08C0863621F4F22FF0683F2E02C0E9
:101660001111115037FE07C01C3350F4EE24E394DF
:10167000E10E27E00BC0183038F027E017E005C076
:1016800027E04CE3E42E02C0212FE12C520144E07C
:10169000A40EB11CF20160817181828193810E2DB3
:1016A000A3010E9471912C01098100FF02C003FF78
:1016B00007C031FC08C032FE09C030E2232E07C04B
:1016C0002DE2222E04C09BE2292E01C0212C802F66
:1016D0008C7019F0211068C2A8C237FE0FC0E40C4C
:1016E00004FF04C08A81813309F4EA941E1474F55E
:1016F000F8E0FE1578F588E0E82E2CC036FC2AC00C
:10170000812F90E0841595059CF02CEF42162FEF69
:10171000520674F0432D4068342E0AC0E2E0F0E037
:10172000EC0FFD1FE10FF11D8081803319F4115082
:101730001111F4CF37FE0EC0EE24E394E10E812F99
:1017400090E0481659062CF4141904C0EE24E394D2
:1017500001C010E037FE06C01414150434F4C201B1
:10176000019605C085E090E002C081E090E0211084
:101770000196112331F0212F30E02F5F3F4F820F70
:10178000931F2F2D30E08217930714F4F81A01C02D
:10179000F12C832D897049F4FF2039F0B60180E2E5
:1017A00090E00E94FA92FA94F7CF222029F0B60135
:1017B000822D90E00E94FA9233FC09C0FF2039F09C
:1017C000B60180E390E00E94FA92FA94F7CF37FED8
:1017D0005AC0942D852D57FE02C090E080E0292E3E
:1017E000382E20E030E0A2014E1951095D874C8768
:1017F000A201421953095F874E87612F70E0442789
:101800005527461B570B598B488B5FEF251635061E
:1018100049F4B6018EE290E02A8B3B8B0E94FA924B
:101820003B892A89421453046CF04C855D8542152E
:10183000530544F4EE85FF85E20FF31FE60DF71D17
:10184000818101C080E351E0251A31082F5F3F4FAD
:1018500048895989241635064CF0B60190E02A8B48
:101860003B8B0E94FA922A893B89CFCF24143504FE
:1018700039F49A81963318F4953311F404FF81E317
:10188000B60190E04BC08A81813309F00F7EB6012A
:1018900090E00E94FA92111105C034FC18C085E650
:1018A00090E017C0B6018EE290E00E94FA9282E0CA
:1018B000EE24E394E80EF301E80FF11D8081B601F8
:1018C00090E00E94FA9211508E2D91F7E6CF85E4B8
:1018D00090E0B6010E94FA9257FC05C041145104F1
:1018E00039F404FF05C05194419451088DE201C0C0
:1018F0008BE2B60190E00E94FA9280E39AE04916EA
:1019000051042CF08F5F5AE0451A5108F7CFB60109
:1019100090E00E94FA92B601C201C0960E94FA922B
:1019200057C1833631F0833779F0833509F058C0D9
:1019300021C05201E2E0AE0EB11CF2018081898328
:1019400001E010E0230114C05201F2E0AF0EB11C1F
:10195000F2014080518026FF03C0612F70E002C079
:101960006FEF7FEFC2012A8B0E94A6928C012A8919
:101970002F7715C05201F2E0AF0EB11CF20140808A
:10198000518026FF03C0612F70E002C06FEF7FEF30
:10199000C2012A8B0E945B928C012A892068322E18
:1019A00023FD1AC08F2D90E008171907A8F4B6017F
:1019B00080E290E00E94FA92FA94F4CFF20137FCB0
:1019C000859137FE81912F01B60190E00E94FA9235
:1019D000F110FA94015011090115110579F7F8C0B9
:1019E000843611F0893659F5520127FF09C0F4E019
:1019F000AF0EB11CF20160817181828193810AC0B6
:101A0000F2E0AF0EB11CF20160817181072E000C73
:101A1000880B990B2F76322E97FF09C090958095F1
:101A2000709561957F4F8F4F9F4F2068322E2AE02F
:101A300030E0A3010E940B94E82EE6183FC0022F6D
:101A4000853721F40F7E2AE030E01DC0097F8F36F4
:101A500091F018F4883559F0C5C0803719F08837EF
:101A600011F0C0C0006104FF09C0046007C024FF7A
:101A700008C0066006C028E030E005C020E130E084
:101A800002C020E132E0520107FF09C0F4E0AF0ECE
:101A9000B11CF201608171818281938108C0F2E002
:101AA000AF0EB11CF2016081718180E090E0A30172
:101AB0000E940B94E82EE6180F77302E36FE0BC0EE
:101AC000332D3E7FE11650F434FE0AC032FC08C0CC
:101AD000332D3E7E05C00E2D332D03C00E2D01C0CB
:101AE000012F34FF0CC0FE01EE0DF11D808180330B
:101AF00011F4397E08C032FF05C00E5F04C0832F89
:101B0000867809F00F5F33FD13C030FF06C01E2D2D
:101B10000F1518F41F0D101B0F2D0F1568F4B601CB
:101B200080E290E03B8B0E94FA920F5F3B89F5CFF9
:101B30000F1510F4F01A01C0F12C34FF12C0B601D9
:101B400080E390E03B8B0E94FA923B8932FF17C002
:101B500031FD03C088E790E002C088E590E0B6015F
:101B60000CC0832F867859F031FF02C08BE201C090
:101B700080E237FD8DE2B60190E00E94FA92E11614
:101B800038F4B60180E390E00E94FA921150F7CF4A
:101B9000EA94F301EE0DF11D8081B60190E00E9400
:101BA000FA92E110F5CF14C0F4E0FF1558F584E087
:101BB000F81A33FE1EC0211026C003FF2AC008EE0B
:101BC00012E0F32DF0713F2EF8018491811124C0B1
:101BD000FF2009F4E5CCB60180E290E00E94FA9281
:101BE000FA94F6CFF6018681978126C08FEF9FEF9A
:101BF00023C0B60180E290E00E94FA92FA94F110BC
:101C0000F8CFD9CFF12CB601822D90E00E94FA9244
:101C1000D4CF0CEE12E0D5CF31108052B60190E057
:101C20000E94FA920F5F1F4FCFCF23E02F1510F4C1
:101C300083E0BECFF12CC1CF63960FB6F894DEBF20
:101C40000FBECDBFDF91CF911F910F91FF90EF900D
:101C5000DF90CF90BF90AF909F908F907F906F90CC
:101C60005F904F903F902F9008958115910511F04E
:101C70000197F1F7089581E396E09F938F930E9477
:101C800046938091660290916702A0916802B0919C
:101C900069020F900F9093FF03C08BE296E002C0A1
:101CA00085E296E09F938F930E9446930F900F904A
:101CB0000895E091F81CEF73F0E0E75BF24E80834B
:101CC0008091F81C8F5F8093F81C80919935886013
:101CD000809399354CE452E061E1CA010E94E16FC2
:101CE00080E090E00895CF93DF93EC0180919F1303
:101CF0009091A013A091A113B091A21386FF1DC0D3
:101D00008E811F928F938D811F928F938C811F9252
:101D10008F938B811F928F938A811F928F9389EE6D
:101D200092E09F938F930E9432938DB79EB70C964B
:101D30000FB6F8949EBF0FBE8DBFBE0181E99AE039
:101D40000E94DA70BE0188E092E0DF91CF910C949E
:101D5000677152985A981DBAE9E6F0E08081806276
:101D60008083EA9A53985B98EB9A8081806880839D
:101D7000E8E6F0E08081816080830895EEEAFDE18D
:101D80001182128210820895CF92DF92EF92FF9219
:101D90000F931F93CF93DF93EC019B018091AE1DB6
:101DA000843108F0BBC08091B01D64E10E94C187FE
:101DB0009093B01DC090CB30D090CC30E090CD301F
:101DC000F090CE30092F10E08DE8989FD0011124BB
:101DD000A255B24E1396CD92DD92ED92FC921697DB
:101DE0004115510559F0FA018081FD01EA57FF4F75
:101DF0008083FA018181A957BF4F8C932097A9F066
:101E000089819DE8909FF001919FF00D1124E2558A
:101E1000F24EDF01A657BF4F8C93E557FF4F8881E5
:101E20008F70808388818F70808321153105E1F167
:101E3000D90116964C9116975DE8509FC001519FAD
:101E4000900D11248255924EFC01E757FF4F4083BD
:101E500015964C9115973197408334961B964D916A
:101E60005D916D917C911E97452F562F672F772797
:101E7000518340837C01BEE8EB0EF11CF901238500
:101E8000348545855685A4E6B0E00E945C88672FBE
:101E9000782F892F992724E630E040E050E00E9417
:101EA000F587D7016D937C938DE8809FD001819F4A
:101EB000B00D1124AB54B24EFE0132968FE7019063
:101EC0000D928A95E1F78091B01D8F5F8093B01DD0
:101ED0009091AE1D9F5F9093AE1D40919F135091C6
:101EE000A0136091A1137091A21360FF2DC01F92E7
:101EF0009F931F928F938091AF1D1F928F938AE6BD
:101F000091E19F938F930E944693EDB7FEB7389669
:101F10000FB6F894FEBF0FBEEDBF16C08091DB3048
:101F20009091DC30A091DD30B091DE300196A11DA2
:101F3000B11D8093DB309093DC30A093DD30B09303
:101F4000DE3080E090E002C081E090E0DF91CF9150
:101F50001F910F91FF90EF90DF90CF900895209107
:101F6000AE1D222361F18091AF1D8F5F2150209320
:101F7000AE1D64E10E94C1879093AF1D40919F13F5
:101F80005091A0136091A1137091A21360FF1AC029
:101F90001F922F938091B01D1F928F931F929F933A
:101FA00083E491E19F938F930E9446938DB79EB7F0
:101FB00008960FB6F8949EBF0FBE8DBF03C080E099
:101FC00090E0089581E090E008951F920F920FB67F
:101FD0000F9211248F939F93AF93BF9380916800CA
:101FE00080FF24C08091743590917535A09176352D
:101FF000B09177350196A11DB11D809374359093F2
:102000007535A0937635B093773580919F13909175
:10201000A013A091A113B091A21387FF07C07498D9
:1020200082E090E09093920280939102BF91AF91F1
:102030009F918F910F900FBE0F901F9018951F9238
:102040000F920FB60F9211248F939F93AF93BF936C
:102050008091680080FF24C0809178359091793517
:10206000A0917A35B0917B350196A11DB11D809369
:10207000783590937935A0937A35B0937B358091FC
:102080009F139091A013A091A113B091A21390FF60
:1020900007C0739882E090E090939202809391023F
:1020A000BF91AF919F918F910F900FBE0F901F9096
:1020B000189580937C0080917B00877F80937B00C4
:1020C00080917C00806C80937C0085E080937A0016
:1020D00080917A00806880937A0080917B0087FFEE
:1020E000FCCF80917B0085FFFCCF80917A008064DB
:1020F00080937A0080917A0086FDFCCF109279005F
:102100001092780084E090E060E070E020917A0026
:10211000206420937A0020917A0026FDFCCF209144
:10212000780030917900620F731F019779F7109250
:102130007C0080917A008F7780937A0076956795FE
:102140007695679580E090E00E94CA8B089580E0C4
:102150000E9459102091890230918A0240918B028D
:1021600050918C020E94C48D21EE3AE744E95EE36F
:102170000E94358A08950F931F93CF93DF930FE149
:1021800010E0CBE5DEE00093510182E991E00E948E
:10219000350E8091510185FD0DC00031110521F0F2
:1021A0002CF0CB54D10903C0C4ECD9E0E297015024
:1021B0001109E9CFBE0180E090E00E94CA8B20E0C7
:1021C00030E04AE754E40E94188BDF91CF911F91D1
:1021D0000F910895CF93DF93EC0188819981009747
:1021E00099F08A3F914121F01982188283E011C051
:1021F000623171F40E94BB106093C7307093C83095
:102200008093C9309093CA308AEF91E19983888393
:1022100081E0DF91CF91089580917B008860809369
:102220007B0089EC80937C0085E080937A0080912C
:102230007A00806880937A0080917B0087FFFCCFD2
:1022400080917B0085FFFCCF80917A008064809331
:102250007A0080917A0086FDFCCF80917A008064BC
:1022600080937A0080917A0086FDFCCF609178009F
:102270007091790080917A008F7780937A0080E066
:1022800090E00E94CA8B27ED33EA40E95FE30E94A9
:10229000C48D26E636E648E853E40E94348A089561
:1022A000CF92DF92EF92FF921F93CF93DF93CDB740
:1022B000DEB729970FB6F894DEBF0FBECDBF6C0115
:1022C000109299138FEF898781E0E82E8DE1F82E27
:1022D00010E089858823E9F11830D9F1BE016F5FDC
:1022E0007F4FCE0109960E94DF5E99859F3F11F0D6
:1022F0009E3F19F4909399132CC0CE010196C114FE
:10230000D10481F40E94F85E80939635AEE8B5E37F
:10231000FE01319688E08E0F91919D938E13FCCF34
:1023200081E018C00E94F85EF7018087FE013196B7
:1023300020E030E08191D701A20FB31F8C932F5F73
:102340003F4F28303105B1F71F5FF9E0EF0EF11C68
:10235000C0CF812F29960FB6F894DEBF0FBECDBF38
:10236000DF91CF911F91FF90EF90DF90CF90089574
:1023700081E491E19F938F930E9446930F900F9079
:1023800008952F923F924F925F926F927F928F9219
:102390009F92AF92BF92CF92DF92EF92FF920F93F4
:1023A0001F93CF93DF93EC015B01009711F427E0BB
:1023B00003C0019749F426E04AE250E06BE270E086
:1023C00089E290E00E94BF5DCE010E9450119E0103
:1023D00026563C4E6901D9018C93CD2B69F0C1E0A2
:1023E000DDE1E12CF12C86EF282E80E1382E92EFF2
:1023F000892E90E1992E9EC08EE895E30E948B5F16
:10240000BC01990F880B990B0E94CC8B6B017C014E
:10241000AB2869F020E030E048EC52E40E94188BD1
:102420009F938F937F936F938FE291E1A4C0CEE847
:10243000D5E30AE211E189911F928F931F930F93C5
:102440000E9446930F900F900F900F90B5E3C639FE
:10245000DB0789F720E030E048EC52E4C701B60121
:102460000E94188B9F938F937F936F938AE191E1E2
:102470009F938F930E9446930F900F900F900F9011
:102480000F900F9080919635811103C08CE893E0F6
:1024900002C088E193E09F938F9386E191E19F933F
:1024A0008F930E9446930F900F900F900F906DC0E6
:1024B00000E010E0FE01E00FF11F80811F928F937A
:1024C000AEEFB0E1BF93AF930E9446930F5F1F4FF3
:1024D0000F900F900F900F900830110559F720E0E2
:1024E00030E048EC52E4C301B2010E94188B9F9384
:1024F0008F937F936F933F922F920E9446930F90FA
:102500000F900F900F900F900F908885811151C000
:102510008CE893E09F938F939F928F920E944693B3
:102520000E94B811FFEFEF1AFF0A29960F900F9043
:102530000F900F90D6018C9190E0E816F906E4F523
:10254000CE010E948B5FBC01990F880B990B0E94F2
:10255000CC8B2B013C01A114B10409F4A9CF20E0DC
:1025600030E048EC52E40E94188B9F938F937F9346
:102570006F9383E091E19F938F930E9446930F9016
:102580000F900F900F900F900F90DF91CF911F91B0
:102590000F91FF90EF90DF90CF90BF90AF909F9002
:1025A0008F907F906F905F904F903F902F900C9402
:1025B000B81188E193E0AECFDF91CF911F910F91D9
:1025C000FF90EF90DF90CF90BF90AF909F908F9053
:1025D0007F906F905F904F903F902F900895CF9392
:1025E000DF931F921F92CDB7DEB7EEE8F5E381814E
:1025F000898387818A83CE0101960E940B740F9094
:102600000F90DF91CF910895CF93DF93EC0120914C
:102610008E3530918F354091903550919135609144
:102620009235709193358091943590919535AFEFB7
:102630000E94288AE1F427E04AE250E06BE270E071
:1026400089E290E00E94BF5D80E090E00E9450111E
:10265000C656DC4E888349E050E06EE070E08EE8BC
:1026600095E30E941196DF91CF910C94EF12DF91C8
:10267000CF9108951F920F920FB60F9211240BB6AF
:102680000F92FF920F931F932F933F934F935F935C
:102690006F937F938F939F93AF93BF93CF93DF936A
:1026A000EF93FF9380919935826080939935809163
:1026B000660286FD2B9A8091660287FD2B9A809197
:1026C0009102909192021816190614F4749A739A52
:1026D00080919F139091A013A091A113B091A21388
:1026E00085FF02C07498739880910602909107024A
:1026F00001979093070280930602892B09F04CC141
:102700008091540A9091550A01969093550A8093AE
:10271000540A8091CB309091CC30A091CD30B091C3
:10272000CE300196A11DB11D8093CB309093CC305B
:10273000A093CD30B093CE3080E190E0909307022B
:10274000809306028091660280FD02C01D9B05C039
:1027500010929E1310929D1306C081E090E090931A
:102760009E1380939D1380919F139091A013A0912D
:10277000A113B091A21397FF08C080919D1390916F
:102780009E13892B49F0749A739808EA1CE1C0EEF5
:10279000D0E3FF24F39421C0739A7498F6CF80910C
:1027A000540A9091550A01960E94CD87892BE1F039
:1027B000F8016085718561157105A1F5F8016085E5
:1027C00071856115710509F03FC0065F1F4F2596A1
:1027D000F0E3C43FDF0709F44CC0F8016085718560
:1027E0006115710529F3DBCF4281417020E030E0B3
:1027F00050E060E070E080E090E0A0E00E94288A75
:10280000B9F2779880919F139091A013A091A11392
:10281000B091A21392FFCCCF7498109292021092B2
:102820009102C6CF8091540A9091550A01960E9458
:10283000CD87892B19F61C821B82AE0162E184E2EE
:1028400092E00E94E16FBACF8091540A9091550AAC
:102850000E94CD87892B09F0B8CFF8821A830983AB
:102860001C821B82AE0162E182E492E00E94E16F71
:10287000ACCF60916C0270916D0261157105A1F190
:102880008091540A9091550A0E94CD87892B61F559
:102890008091743590917535A0917635B0917735EA
:1028A0004091BD285091BE286091BF287091C028EA
:1028B000841B950BA60BB70B8093D01C9093D11C57
:1028C000A093D21CB093D31C809174359091753530
:1028D000A0917635B09177358093BD289093BE282E
:1028E000A093BF28B093C02860916A0270916B02D8
:1028F00061157105A1F18091540A9091550A0E94C9
:10290000CD87892B61F58091783590917935A091AB
:102910007A35B0917B354091C1285091C2286091A1
:10292000C3287091C428841B950BA60BB70B80930A
:10293000D41C9093D51CA093D61CB093D71C809127
:10294000783590917935A0917A35B0917B35809327
:10295000C1289093C228A093C328B093C428809123
:10296000660286FD2B988091660290916702A09185
:102970006802B091690291FF0FC00E9407698A3115
:1029800019F0C1E0C80F01C0CBE00E9444678C2F52
:102990000E941F690E940E6840E050E060E085EBF5
:1029A00092E00E94E16FFF91EF91DF91CF91BF9193
:1029B000AF919F918F917F916F915F914F913F91D7
:1029C0002F911F910F91FF900F900BBE0F900FBE94
:1029D0000F901F9018958091F81C9091DF30891B03
:1029E00008950E94EB14882371F0E091DF30EF73BB
:1029F000F0E0E75BF24E808190E02091DF302F5FC6
:102A00002093DF3008958FEF9FEF0895CF93DF93EA
:102A1000EC011092850A1092840A888199810097AE
:102A2000C1F0863E934021F01982188283E0BDC038
:102A3000613109F0B9C00E94F11499279093800A7E
:102A400080937F0A8D30910509F444C08F3F910532
:102A500049F40E94EB148111EECF86EE93E0998346
:102A60008883A2C08231910509F45AC08F3791053D
:102A700009F052C080917D0A90917E0A18161906BD
:102A80000CF56091F7397091F83988E090E00E9478
:102A9000FA926091F7397091F83980E290E00E94E3
:102AA000FA926091F7397091F83988E090E00E94CD
:102AB000FA9280917D0A90917E0A019790937E0A06
:102AC00080937D0A80917D0A90917E0A8F379105CF
:102AD00009F0BFCF1092DF301092F81C80917D0A70
:102AE00090917E0AFC01EC50FF4C10829093850A75
:102AF0008093840A10927E0A10927D0A8091973505
:102B000090919835009709F4A4CF40E050E060918F
:102B100097130E94E16F9DCF8830910571F5AACF80
:102B20006091F7397091F8398DE090E00E94FA9247
:102B300010927C0A10927B0A20917B0A30917C0AC9
:102B400080917D0A90917E0A281739070CF0BACF40
:102B5000F901EC50FF4C80816091F7397091F839A0
:102B600090E00E94FA9280917B0A90917C0A0196F3
:102B700090937C0A80937B0ADFCF6091F739709144
:102B8000F8390E94FA9220917D0A30917E0A809154
:102B90007F0AF901EC50FF4C80832F5F3F4F309349
:102BA0007E0A20937D0A8ECF81E0DF91CF91089538
:102BB00080919D1390919E13892BD1F08091660294
:102BC00090916702A0916802B091690293FD10C0D4
:102BD0000E94446783B7817F866083BFF89483B780
:102BE000816083BF7894889583B78E7F83BF789404
:102BF0000895CF93DF93FC012081318121153105A8
:102C000051F02D32324129F0FC011182108283E013
:102C100015C0653891F4EC010E9445660E94D815F4
:102C200040E050E065E88091E1149091E2140E9448
:102C3000E16F8DE292E19983888381E0DF91CF910A
:102C40000895CF93DF931F921F92CDB7DEB7892BE4
:102C500081F05F934F938FEE90E19F938F93698301
:102C60007A830E9446930F900F900F900F907A8175
:102C700069817F936F938CEE90E19F938F930E9475
:102C800046930F900F900F900F900F900F90DF9141
:102C9000CF910895EF92FF920F931F93CF93DF93FD
:102CA0000E94456680EB0E94186081111CC00E9442
:102CB0007C608091C52C9091C62C81609093C62C2D
:102CC0008093C52C81E293E09F938F938CEE90E1EB
:102CD0009F938F930E9446930F900F900F900F90A9
:102CE000C1E0D0E002C0C0E0D0E01EB11470729A22
:102CF0000E9445668EE40E941860811117C00E94F0
:102D00007C608091C52C9091C62C82609093C62CDB
:102D10008093C52C7E018FEFE81AF80A48E259E04B
:102D200069E273E0CE010E942116E701111101C092
:102D300072980E9445668EEE0E941860811116C03E
:102D40000E947C608091C52C9091C62C84609093E9
:102D5000C62C8093C52C8E010F5F1F4F48E259E0AF
:102D600061E373E0CE010E942116E8010E944566EE
:102D700086EA0E941860811116C00E947C608091D2
:102D8000C52C9091C62C88609093C62C8093C52C3E
:102D90008E010F5F1F4F48E259E068E373E0CE01F8
:102DA0000E942116E8010E9445668CE30E9418608B
:102DB00081111EC00E947C608091C52C9091C62C10
:102DC00080619093C62C8093C52C8E010F5F1F4F9E
:102DD00048E259E060E473E0CE010E94211684EEDF
:102DE00090E19F938F930E9446930F900F90E8017C
:102DF0000E94456682ED0E941860811116C00E94F3
:102E00007C608091C52C9091C62C80629093C62CDA
:102E10008093C52C8E010F5F1F4F48E259E068E494
:102E200073E0CE010E942116E8010E94456680E809
:102E30000E941860811116C00E947C608091C52C90
:102E40009091C62C91609093C62C8093C52C8E01D6
:102E50000F5F1F4F48E259E061E573E0CE010E9429
:102E60002116E8010E94456680ED0E9418608111DC
:102E700016C00E947C608091C52C9091C62C806801
:102E80009093C62C8093C52C8E010F5F1F4F48E294
:102E900059E067E573E0CE010E942116E8010E9427
:102EA00045668CEE0E941860811116C00E947C60FD
:102EB0008091C52C9091C62C92609093C62C8093E3
:102EC000C52C8E010F5F1F4F48E259E06FE573E09C
:102ED000CE010E942116E80107E010E00E9445663D
:102EE0008CE70E941860811113C00E947C60809161
:102EF000C52C9091C62C80649093C62C8093C52CD1
:102F000048E259E066E673E0CE010E94211603C054
:102F10000150110919F70E947C60DF91CF911F9138
:102F20000F91FF90EF900C94B811CF93DF931F9205
:102F30001F92CDB7DEB74A8369830E9453606981CF
:102F4000862F0E9484604A81842F0E9484600F90A3
:102F50000F90DF91CF910C947C60AF92BF92CF9293
:102F6000DF92EF92FF920F931F93CF93DF9300D0E6
:102F7000CDB7DEB7182F022F4A835B8369830E9487
:102F800053606981862F0E948460812F81600E9436
:102F90007A604A81A42E5B81B52E10E0E12CF12CE1
:102FA000680181E0C81AD108E016F10689F0EC1436
:102FB000FD0419F40E949F6002C00E949560F50113
:102FC0008083FFEFEF1AFF0A8FEFA81AB80AECCF41
:102FD0000F900F900F90DF91CF911F910F91FF9065
:102FE000EF90DF90CF90BF90AF900C947C60BF9239
:102FF000CF92DF92EF92FF920F931F93CF93DF93C5
:10300000CDB7DEB760970FB6F894DEBF0FBECDBF69
:10301000F82EE42E6623D9F18E010F5F1F4F80E159
:10302000F80111928A95E9F728E0A80168E980EB98
:103030000E94AD17FF2041F08FE693E09F938F939E
:103040000E9432930F900F9026E7C22E23E0D22EDB
:1030500037E0B32EB00EF80181918F011F928F934C
:10306000DF92CF920E9432930F900F900F900F90AB
:10307000B012F1CF88851F928F938BEC93E09F93D2
:103080008F930E9432930F900F900F900F90EE202D
:10309000D9F18E010F5F1F4F80E1F80111928A95DF
:1030A000E9F720E1A80160E880EB0E94AD17FF205E
:1030B00041F08BE793E09F938F930E9432930F90A0
:1030C0000F9086E7E82E83E0F82E9FE0D92ED00EF1
:1030D000F80181918F011F928F93FF92EF920E94CE
:1030E00032930F900F900F900F90D012F1CF8889EC
:1030F0001F928F938BEC93E09F938F930E94329358
:103100000F900F900F900F9060960FB6F894DEBF5F
:103110000FBECDBFDF91CF911F910F91FF90EF9028
:10312000DF90CF90BF9008950F931F93CF93DF93BD
:103130001F921F92CDB7DEB71A82198222E0AE012C
:103140004F5F5F4F6AEA8EEE0E94AD1709E81DE1FE
:10315000898190E0982F88272A81822BF80191831A
:10316000808322E0AE014F5F5F4F6CEA8EEE0E94DB
:10317000AD17898190E0982F88272A81822BF8014A
:103180009383828322E0AE014F5F5F4F6EEA8EEE43
:103190000E94AD17898190E0982F88272A81822B81
:1031A000F8019583848322E0AE014F5F5F4F60EBAF
:1031B0008EEE0E94AD17898190E0982F88272A8192
:1031C000822BF801938B828B22E0AE014F5F5F4F21
:1031D00062EB8EEE0E94AD17898190E0982F8827D0
:1031E0002A81822BF801958B848B22E0AE014F5F00
:1031F0005F4F64EB8EEE0E94AD17898190E0982FAF
:1032000088272A81822BF801978B868B22E0AE01DA
:103210004F5F5F4F66EB8EEE0E94AD17898190E0A5
:10322000982F88272A81822BF8019783868322E0B2
:10323000AE014F5F5F4F68EB8EEE0E94AD17898144
:1032400090E0982F88272A81822BF8019187808728
:1032500022E0AE014F5F5F4F6AEB8EEE0E94AD172A
:10326000898190E0982F88272A81822BF801958701
:10327000848722E0AE014F5F5F4F6CEB8EEE0E94C1
:10328000AD17898190E0982F88272A81822BF80139
:103290009787868722E0AE014F5F5F4F6EEB8EEE21
:1032A0000E94AD17898190E0982F88272A81822B70
:1032B000F801918B808B0F900F90DF91CF911F9130
:1032C0000F9108952F923F924F925F926F927F924B
:1032D0008F929F92AF92BF92CF92DF92EF92FF9226
:1032E0000F931F93CF93DF93CDB7DEB76C970FB6D5
:1032F000F894DEBF0FBECDBF182F042F2D8B19827F
:103300001A821B828091AD1D811107C06C8F0E94B3
:10331000941881E08093AD1D6C8D662309F472C012
:103320004EE264EF8EEE0E94951762E174E380E056
:1033300090E00E94F65F22E0AE014F5F5F4F66EFC4
:103340008EEE0E94AD172981822F90E0A0E0B0E0C0
:103350004427582F692F7A2F8A81482B80919F1DEF
:103360009091A01D9A01AB01281B390B410951090D
:10337000A0919D1DB0919E1D0E945C886B017C01F7
:103380003FE0F594E794D794C7943A95D1F76091CC
:10339000971D7091981DCB01770FAA0BBB0BBC0139
:1033A000CD014BE0660F771F881F991F4A95D1F713
:1033B0002091991D30919A1D4901330FAA08BB082D
:1033C000A7019601280D391D4A1D5B1D0E94178813
:1033D000C20ED31ED092941DC092931D28E0C20E3F
:1033E000D11C54E0D594C7945A95E1F70D2C000CEC
:1033F000EE08FF08C092A11DD092A21DE092A31D6D
:10340000F092A41D812F8295880F880F807C8C5CA0
:103410008887212E312CA3E0B0E0012E02C0AA0F34
:10342000BB1F0A94E2F72AE63AE00E9455889B0106
:10343000AC012E5F3F4F4F4F5F4F29873A874B8735
:103440005C8780E593ECA0E0B0E09C01AD0104C096
:1034500055954795379527951A95D2F7298B3A8B2D
:103460004B8B5C8B10E0412C512C320188E090E0BA
:10347000AC01421953095B8F4A8F101709F43EC102
:10348000488564EF8EEE0E94951769857A858B8555
:103490009C850E94F65F23E0AE014F5F5F4F66EFB1
:1034A0008EEE0E94AD17E091931DF091941DE05AAD
:1034B000FF409F01DF010E943E886C837D838E83E5
:1034C0009F8380918B1D90918C1D9E878D8720916D
:1034D000891D30918A1D388B2F8720918D1D309149
:1034E0008E1D0E943E886B017C01ADE0F594E7944F
:1034F000D794C794AA95D1F7A0918F1DB091901D34
:103500002C813D814E815F818CE0559547953795A3
:1035100027958A95D1F70E946788BB2797FDB095BC
:10352000AB2F8C0D9D1DAE1DBF1D0296A11DB11DA3
:1035300032E0B595A795979587953A95D1F79C0177
:10354000AD0130584F4F5F4FA0919B1DB0919C1D16
:103550000E945C884B015C014FE0B694A79497945D
:1035600087944A95D1F739818A8190E0A0E0B0E054
:10357000BA2FA92F982F8827A32B2B81822B9C0150
:10358000AD010A8C04C055954795379527950A9447
:10359000D2F72E8B3F8B488F598F4F8558896A0100
:1035A000550FEE08FF0862E0CC0CDD1CEE1CFF1C82
:1035B0006A95D1F7A091911DB091921D2C813D810A
:1035C0004E815F810E9467889B01AC0177E1559530
:1035D0004795379527957A95D1F72C833D834E8370
:1035E0005F832D853E85DF010E943E88DC01CB0193
:1035F000EBE0B595A79597958795EA95D1F72C813E
:103600003D814E815F81820F931FA41FB51FC80E9D
:10361000D91EEA1EFB1E022C04C0CC0CDD1CEE1CC5
:10362000FF1C0A94D2F732E0C30ED11CE11CF11C3E
:10363000F2E0F594E794D794C794FA95D1F72E89E0
:103640003F89488D598D2C193D094E095F096989BB
:103650007A898B899C890E94B18797FD0BC0660F80
:10366000771F881F991FA50194010E94F5876901A2
:103670007A010AC0A50194010E94F58769017A01C7
:10368000CC0CDD1CEE1CFF1C9927F7FC9A958F2DA6
:103690007E2D6D2D9B01AC010E94B1879B01AC0179
:1036A000AEEDBBE00E945C884C01BB2497FCB0945B
:1036B000AB2CA3E4B3EEA70196010E946A88BB2756
:1036C00097FDB095AB2F880E991EAA1EBB1E4FEC1E
:1036D000840E4EE0941EA11CB11C44E0B594A79446
:1036E000979487944A95D1F7C80CD91CEA1CFB1C07
:1036F0004C0C5D1C6E1C7F1C1F5FBFCE112381F024
:10370000212F30E040E050E0C301B2010E94F58774
:103710002093A51D3093A61D4093A71D5093A81D6F
:103720005D89552389F16091A51D7091A61D809139
:10373000A71D9091A81D611571058105910521F1C5
:103740000E94CC8B20E836EE45EC57E40E94188BA3
:1037500021E03EED42E45EE30E94318E9B01AC012C
:1037600060E070E080E89FE30E94348A2BE43AE353
:103770004DEB57E30E94188B6093A91D7093AA1D0F
:103780008093AB1D9093AC1D6C960FB6F894DEBF82
:103790000FBECDBFDF91CF911F910F91FF90EF90A2
:1037A000DF90CF90BF90AF909F908F907F906F9061
:1037B0005F904F903F902F9008950F931F93CF935A
:1037C000DF9300D000D0CDB7DEB78E010F5F1F4F63
:1037D00086E0F80111928A95E9F780919F1C81118A
:1037E00013C040E061E386EA0E9495174AE06CE26C
:1037F00086EA0E94951781E080939F1C68EF7CE722
:1038000080E090E00E94F65F48E06DE286EA0E9468
:10381000951768EF7CE780E090E00E94F65F26E075
:10382000A80162E386EA0E94AD1747E06DE286EAEE
:103830000E9495178A8190E0982F88272981822BF2
:1038400090939A1C8093991C2C8130E0322F222770
:103850004B81242B30939C1C20939B1C4E8150E069
:10386000542F44276D81462B50939E1C40939D1CE2
:103870005F934F933F932F939F938F938FE793E0A3
:103880009F938F930E9432930FB6F894DEBF0FBEC2
:10389000CDBF26960FB6F894DEBF0FBECDBFDF9129
:1038A000CF911F910F910895CF92DF92EF92FF92E7
:1038B0000F931F93CF93DF93CDB7DEB72A970FB641
:1038C000F894DEBF0FBECDBF8E010F5F1F4F86E0A5
:1038D000F80111928A95E9F741E062E08CE30E94D9
:1038E000951748E560E08CE30E94951764E278E65E
:1038F00080E090E00E94F65F26E0A80163E08CE3A0
:103900000E94AD1743E062E08CE30E9495170981A5
:1039100010E0102F00278A81082BE9E7FCE11183D2
:103920000083EB80F12CFE2CEE248C81E82AF382BC
:10393000E282CD80D12CDC2CCC248E81C82AD58289
:10394000C482B801012E000C880B990B0E94CC8B0D
:103950009B01AC01B7010F2C000C880B990B2F8336
:10396000388749875A870E94CC8B2F8138854985B3
:103970005A850E94B48A20EE3EE245E652E40E9457
:10398000C48D20E030E044E353E40E94358A9F93E5
:103990008F937F936F93DF92CF92FF92EF921F935B
:1039A0000F938DE893E09F938F930E9432930FB60D
:1039B000F894DEBF0FBECDBF2A960FB6F894DEBFD7
:1039C0000FBECDBFDF91CF911F910F91FF90EF9070
:1039D000DF90CF900895CF93DF93EC018881998198
:1039E000009759F18631924121F01982188283E0C3
:1039F00071C082E69AE00E946F6E892B51F180912E
:103A00009F139091A013A091A113B091A21393FDC5
:103A100022C080919F139091A013A091A113B09107
:103A2000A21394FD49C080919F139091A013A0917F
:103A3000A113B091A21395FD46C040E850E060E0AC
:103A400070E082E69AE00E94516E86E192E19983ED
:103A5000888381E03FC08091C52C82FFDACF21E0CE
:103A600048E061E083E00E9462198091AC1D8F9371
:103A70008091AB1D8F938091AA1D8F938091A91D7A
:103A80008F938091A81D8F938091A71D8F93809114
:103A9000A61D8F938091A51D8F9388EA91E19F9336
:103AA0008F930E9446938DB79EB70A960FB6F894EF
:103AB0009EBF0FBE8DBFADCF8091C52C83FFB3CF0E
:103AC0000E94DD1BB0CF8091C52C84FFB6CF0E9431
:103AD000541CB3CFDF91CF910895CF93C82F8CEEB4
:103AE0000E947A608C2F0E9484606AE67AE080E00F
:103AF00090E00E94F65F8DEE0E947A600E949560D1
:103B0000C82F0E949F602C2F30E0322F2227A9015E
:103B1000482BCA01CF9108950F931F93CF93DF9342
:103B2000C82F8CEE0E947A608C2F0E94846064E221
:103B300078E680E090E00E94F65F8CEE0E947A606A
:103B400080E00E9484606AE67AE080E090E00E9473
:103B5000F65F8DEE0E947A600E949560C82F0E94E9
:103B60009560D82F0E949F604D2F50E060E070E07C
:103B7000762F652F542F44276C2B8A019B01082B2D
:103B8000C901B801DF91CF911F910F9108952F9234
:103B90003F924F925F926F927F928F929F92AF92DD
:103BA000BF92CF92DF92EF92FF920F931F93CF932A
:103BB000DF93CDB7DEB7CB54D1090FB6F894DEBF93
:103BC0000FBECDBF8091040290910502892BD1F1E7
:103BD00010920502109204028CEE0E947A608EE12F
:103BE0000E94846066E37CE980E090E00E94F65FDA
:103BF00082EA0E946D1D9093530A8093520A84EAD0
:103C00000E946D1D9093510A8093500A86EA0E948B
:103C10006D1D90934F0A80934E0A88EA0E946D1D95
:103C200090934D0A80934C0A8AEA0E946D1D9093EE
:103C30004B0A80934A0A8CEA0E946D1D9093490AB0
:103C40008093480A88E40E948C1D6DAB7EAB8FABDD
:103C500098AF88E50E948C1D4B015C0180914A0A57
:103C600090914B0A8C0120E030E040E050E0BA0136
:103C700022968FAF229723961FAF239724962FAFBC
:103C8000249725963FAF259726964FAF26972796E0
:103C90005FAF279728966FAF289729967FAF299710
:103CA0009C0140E050E060E070E080E090E008E0DF
:103CB0000E94CA890E9483893901B42FA52FF62F4B
:103CC000E72F8C019401A50160E070E080E090E0B6
:103CD0005301CB2EDA2EEF2EFE2E0E94018A2CA34A
:103CE0003BA34B83252E362E472E582E792E632D3F
:103CF000742D852D972D315041095F4F6F4F7F4FA8
:103D00008F4F9F4F88248394912C21153F4F4F4F05
:103D10005140610571058105910509F010F4812C70
:103D2000912C9A8289820091480A1091490A58017F
:103D3000C12CD12CE12CF12C00E010E02CA13BA1F6
:103D40004B81522D632D742D852D972D0E946F88E8
:103D5000F22E032F142FB52FF62FE72FD82EE92E92
:103D6000A0E00E94288A84F42150310940485F4F26
:103D70006F4F7F4F8F4F9F4FF22E032F142FB52F72
:103D8000F62FE72FD82EE92E2F2D302F412F5B2F26
:103D90006F2F7E2F8D2D9E2D07E10E94E3892B8FA3
:103DA0003C8F4D8F5E8F6F8F78A389A39AA320538A
:103DB000384F4F4F5F4F6F4F7F4F8F4F9F4F2B8B22
:103DC0003C8B4D8B5E8B6F8B788F898F9A8F2056B3
:103DD000304F4F4F5F4F6F4F7F4F8F4F9F4F243D5F
:103DE000304341055105610571058105910529F0B3
:103DF00020F0F4013196FA83E9838090500A909084
:103E0000510A940140E050E060E070E080E090E012
:103E100000E10E94CA892C833D834E835F83662E16
:103E200078874C0140914C0A50914D0AACA0BBA040
:103E3000CB80D22CE32CF42C052D172D9A0140E0D9
:103E400050E060E070E080E090E00E946F88F22E29
:103E5000032F142FB52FF62FE72FD82EE92EA0E031
:103E60000E94288A5CF4AFE70E940A8AF22E032F90
:103E7000142FB52FF62FE72FD82EE92E2F2D302F08
:103E8000412F5B2F6F2F7E2F8D2D9E2D07E00E94DF
:103E9000E38959016A017B018C012C813D814E81AE
:103EA0005F81662D7885C4010E94018A2C833D8341
:103EB0004E835F8368877E878F87988B2E5F3F4F07
:103EC000434051096E4F7F4F8F4F9F4F2230310536
:103ED000494F5F4F644071058105910539F030F01D
:103EE00009811A810F5F1F4F1A8309836091520A5B
:103EF0007091530A80E090E020E030E840E050E02C
:103F00000E94C88829873A874B875C87662E7D8701
:103F10004C0140914E0A50914F0AACA0BBA0CB80FF
:103F2000D22CE32CF42C052D172D9A0140E050E003
:103F300060E070E080E090E00E946F88F22E032F36
:103F4000142FB52FF62FE72FD82EE92EA0E00E94D0
:103F5000288A84F421503F4F4F4F5F4F6F4F7F4F60
:103F60008F4F9F4FF22E032F142FB52FF62FE72FD1
:103F7000D82EE92E2F2D302F412F5B2F6F2F7E2F24
:103F80008D2D9E2D08E00E94E38959016A017B0175
:103F90008C0129853A854B855C85662D7D85C4011C
:103FA0000E94018A29873A874B875C876D87798BC6
:103FB0008A8B692E2F5F3F4F41405109610971097A
:103FC00081099109213030484C4F5F4761407105AC
:103FD0008105910539F030F029813A812F5F3F4FFB
:103FE0003A8329832B893C894D895E896F89788D35
:103FF000898D9A8D2F3C374041055105610571052A
:104000008105910511F00CF0A4C1ACA0BBA0CB8040
:10401000D22CE32CF42C052D172D95014C2D522D6F
:10402000632D742D852D972D0E946F88A12CB12CA6
:10403000C12CE0E8DE2EE12CF12C00E010E00E9423
:10404000F58829AF3AAF4BAF5CAF6DAF7EAF8FAFA6
:1040500021969FAF2197AB8CBC8CCD8CDE8CEF8CE6
:10406000F8A009A11AA19501A601B701C8010E94F3
:104070006F8859016A017B01E82F192F02E00E9425
:10408000CA890E2F0E94018A7901142F552EF62F0E
:10409000E72F6C01922EAF2CB42E052F462EB72F92
:1040A000782E8D2CA0E00E94288A5CF4A1E00E946A
:1040B0000A8A922EA32EB42E052F462EB72F782EC5
:1040C000892E292D3A2D4B2D502F642D7B2F872D96
:1040D000982D01E00E94E3892AA7732E4A012C96AD
:1040E0006FAF2C972B967FAF2B978BA79CA72B831B
:1040F0003BA34CA39DA26EA37FA388A799A7B52D30
:104100009701412F552D6F2F7E2FC601A0E00E94F1
:10411000288A4CF4A3E00E940A8A7901142FB52F53
:10412000F62FE72F6C019701412F5B2F6F2F7E2F0A
:10413000C60102E00E94E3892DA73EA74FA758AB16
:1041400069AB7AAB8BAB9CAB2901B42FA52F229620
:104150006FAF2297F72F1C012B893C894D895E890F
:104160006F89788D898D9A8D24323A4F4F4F5F4FEA
:104170006F4F7F4F8F4F9F4F0CF08BC02B8D3C8D1F
:104180004D8D5E8D6F8D78A189A19AA12455324FF6
:104190004F4F5F4F6F4F7F4F8F4F9F4F59016A01B6
:1041A0007B018C010E946F8819012A01B62FA72F6D
:1041B000FC0103E00E94CA8951016201EB2EFA2E34
:1041C0008F010E94168A59016A017B018C012AA580
:1041D000372DA4012C966FAD2C972B967FAD2B9786
:1041E0008BA59CA50E94018A2B833BA34CA35DA3B6
:1041F0006EA37FA388A799A79101A2016B2F7A2FA5
:10420000CF0102E00E94CA8951016201EB2EFA2E11
:104210008F010E94168A02E00E94CA890E2F0E9416
:10422000168A122FD32EE42EB52FF62FE72FF82E55
:10423000092FA0E00E94288A5CF4A1E00E940A8A6B
:10424000122FD32EE42EB52FF62FE72FF82E092F9D
:10425000212F3D2D4E2D5B2F6F2F7E2F8F2D902FD9
:1042600001E00E94E38959016A017B018C012DA5BF
:104270003EA54FA558A969A97AA98BA99CA90E9416
:10428000018A2901B42FA52F22966FAF2297F72F0D
:104290001C012C813D814E815F8168857E858F85E3
:1042A0009889AB80BBA0CCA0DDA0EEA0FFA008A5A4
:1042B00019A50E94168A2C833D834E835F836887ED
:1042C0007E878F87988B29853A854B855C856D85A0
:1042D00079898A89962D5201CB2EDA2E2296EFAC5F
:1042E0002297FF2E81010E94168A29873A874B87E1
:1042F0005C876D87798B8A8B692E2B893C894D89E8
:104300005E896F89788D898D9A8DA9ACBAACCBAC5A
:10431000DCACEDACFEAC0FAD21961FAD21970E9439
:10432000168A2056304F4F4F5F4F6F4F7F4F8F4F42
:104330009F4F243D304341055105610571058105BD
:10434000910539F030F009811A810F5F1F4F1A83F0
:1043500009834DA95EA96FA978AD9A01AB0160E010
:1043600070E0CB0122962FAF229723963FAF239781
:1043700024964FAF249725965FAF259726966FAF6B
:10438000269727967FAF279728968FAF289729964D
:104390009FAF2997A984BA84CB84DC84ED84F98803
:1043A0000A89162D60E070E080E090E00E946F883E
:1043B000122FD32EE42EB52FF62FE72FF82E092F2C
:1043C000A0E00E94288A84F421503109404E5F4FBA
:1043D0006F4F7F4F8F4F9F4F122FD32EE42EB52F4D
:1043E000F62FE72FF82E092F212F3D2D4E2D5B2F75
:1043F0006F2F7E2F8F2D902F05E10E94E389AC80D7
:10440000BD80CE80DF80E884FE840F8518890E94FD
:10441000168A122FD32EE42EB52FF62FE72FF82E63
:10442000092FA0E00E94288A84F4215030484F4F81
:104430005F4F6F4F7F4F8F4F9F4F122FD32EE42E22
:10444000B52FF62FE72FF82E092F212F3D2D4E2DBA
:104450005B2F6F2F7E2F8F2D902F0FE00E94E3890F
:1044600039014A015B016C0179018A011B012C01B0
:10447000285E334041095109610971098109910997
:10448000283D304D4140510561057105810591057B
:1044900031F028F0E981FA813196FA83E9830E94AC
:1044A0007C6029813A81232B51F09301A401B5014D
:1044B000C6010E94838979018A011B012C019701A1
:1044C000A801B101C2010E94C48B20E030E048EC99
:1044D00052E40E94188BC55BDF4F0FB6F894DEBF25
:1044E0000FBECDBFDF91CF911F910F91FF90EF9045
:1044F000DF90CF90BF90AF909F908F907F906F9004
:104500005F904F903F902F9008954F925F926F92DF
:104510007F928F929F92AF92BF92CF92DF92EF9253
:10452000FF922B013C0169017A0123EC35EF4CE845
:1045300051E4C701B6010E94C48D4B015C0128EB18
:104540003EE143E753E4C701B6010E94358A9B016F
:10455000AC01C501B4010E94188B0E94928B4B01E3
:104560005C0120E030E048EC52E4C301B2010E945B
:10457000188B21E835E943EC50E40E94C48DA50175
:1045800094010E94C48D4B015C0123E333E948E8A8
:1045900053E4C701B6010E94358A9B01AC01C501F5
:1045A000B4010E94188B23E333EB48E553E40E94E7
:1045B000C48DFF90EF90DF90CF90BF90AF909F9011
:1045C0008F907F906F905F904F9008954F925F9281
:1045D0006F927F928F929F92AF92BF92CF92DF9213
:1045E000EF92FF9269017A010E94388D20E030E05D
:1045F00040E050E40E94348A22E93CE54EED5EE35F
:104600000E94188B4B015C0123EC35EF4CE851E420
:10461000C701B6010E94C48D2B013C0128EB3EE18D
:1046200043E753E4C701B6010E94358A9B01AC0100
:10463000C301B2010E94188B9B01AC01C501B401FA
:104640000E94358A6B017C0128EB3EE143E753E48D
:104650000E94C48D4B015C01A701960163EC75EFCC
:104660008CE891E40E94348A9B01AC01C501B4013D
:104670000E94188BFF90EF90DF90CF90BF90AF908B
:104680009F908F907F906F905F904F9008954F9282
:104690005F926F927F928F929F92AF92BF92CF92D2
:1046A000DF92EF92FF922B013C0169017A0123EC2A
:1046B00035EF4CE851E4C701B6010E94C48D4B01AF
:1046C0005C0128EB3EE143E753E4C701B6010E94D9
:1046D000358A9B01AC01C501B4010E94188B0E9470
:1046E000928B4B015C0120E030E048EC52E4C301C6
:1046F000B2010E94188BA50194010E94C48D20E094
:1047000030E040E251E40E94348A24EE38E34EE087
:104710005FE30E94C48D9B01AC01C701B6010E94FA
:10472000358AFF90EF90DF90CF90BF90AF909F9031
:104730008F907F906F905F904F90089580E80E94D7
:104740007A6081110DC08EEF0E948460811108C0D3
:1047500066E37CE980E090E00E94F65F0C947C6068
:104760000E947C608091D7309091D830A091D93050
:10477000B091DA300196A11DB11D8093D73090938E
:10478000D830A093D930B093DA300895FC01DC0121
:10479000AC014E5F5F4F90E031E38D91982788E048
:1047A000292F220F97FF03C0922F932701C0922F2A
:1047B0008150B1F7A417B50781F721E030E082817D
:1047C000981711F020E030E0C9010895DF92EF92D0
:1047D000FF920F931F93CF93DF930E949E2380E855
:1047E0000E947A6081116DC08AEF0E9484608111FD
:1047F00068C08FE00E948460811163C06AE67AE03D
:1048000080E090E00E94F65F81E80E947A6081116A
:1048100058C00E949560D82F0E9495600E949560B4
:10482000182F0E9495600E949560082F0E94956045
:104830000E949F60F82E80E80E947A60811141C03A
:104840008CEF0E94846081113CC089EC0E948460DE
:10485000811137C06AE67AE080E090E00E94F65F5E
:1048600081E80E947A600E949560E82E0E9495601F
:10487000D82E0E9495600E949560C82F0E949F606C
:104880001F92DF921F92EF921F92FF921F920F933F
:104890001F921F931F92DF931F928F931F92CF93AC
:1048A00082EA93E09F938F930E9432930E947C60F0
:1048B0008DB79EB742960FB6F8949EBF0FBE8DBFC0
:1048C00017C00E947C608091D7309091D830A09121
:1048D000D930B091DA300196A11DB11D8093D73047
:1048E0009093D830A093D930B093DA300E949E23B1
:1048F00020E030E040E050E060E070E080E090E0F8
:10490000DF91CF911F910F91FF90EF90DF9008956D
:10491000EF92FF920F931F93CF93DF9300D0CDB709
:10492000DEB78C0180E80E947A60811154C00115C5
:10493000110551F085EE0E94846081114CC062E047
:104940007EE281E090E009C083EE0E9484608111E4
:1049500042C062E375E783E090E00E94F65F81E881
:104960000E947A60811137C00E949560E82E898389
:104970000E949560F82E8A830E949F608B830E941C
:104980007C60CE0101960E94C623892B21F16F2DF8
:1049900070E07E296C7F80E090E0012B69F00E943E
:1049A000CA8B20E030E04AEF5AE30E94C48D20E039
:1049B00030E040EC50E40CC00E94CA8B22E538EB9A
:1049C0004FE25BE30E94C48D26E636E64BE352E4F9
:1049D0000E94348A1BC00E947C608091D7309091E5
:1049E000D830A091D930B091DA300196A11DB11D17
:1049F0008093D7309093D830A093D930B093DA30E9
:104A00000E949E2360EF7FEF89E794E40F900F9060
:104A10000F90DF91CF911F910F91FF90EF9008952C
:104A20000F931F93CF93DF93729A8091660283FF57
:104A300008C08EE40E941860811165C0C0E5D0E016
:104A400009C0C0E5D0E08FED97E00E94350E2197B8
:104A5000D1F7EFCF8FED97E00E94350E2197D1F778
:104A60008FE40E9418600E949560D82FDF730E9427
:104A70009560082F0E949560C82F0E949F60182F94
:104A80000E947C608091660283FF72986D2F70E0B7
:104A9000762F6627600F711D80E090E00E94CA8B20
:104AA00020E134E048EC5BE30E94C48D6093B928B8
:104AB0007093BA288093BB289093BC286C2F70E029
:104AC000762F6627610F711D7695679576956795A8
:104AD00080E090E00E94CA8B24EA3CEF44E25CE371
:104AE0000E94C48D20E030E040E252E40E94348A0B
:104AF00060939A3570939B3580939C3590939D3548
:104B000080E090E002C081E090E0DF91CF911F91C2
:104B10000F9108957298729A8EE40E94186080EA4C
:104B20000E94846080E00E94846080E00E94846033
:104B30008FE40E9418600E9495608EE40E941860C5
:104B400080E80E94846080E00E94846080E00E948F
:104B500084600E947C6080E090E0089587ED90E1A1
:104B60009F938F930E944693809180020F900F90A5
:104B7000882361F01F928F9384ED90E19F938F9330
:104B80000E9446930F900F900F900F9008958FEA18
:104B900090E19F938F930E94469387E890E19F93C3
:104BA0008F930E94469380E690E19F938F930E949B
:104BB000469385E290E19F938F930E94469389EEFE
:104BC0009FE09F938F930E94469387EB9FE09F9374
:104BD0008F930E9446938BE79FE09F938F930E9451
:104BE000469385E59FE09F938F930E9446938FE1C4
:104BF0009FE09F938F930E9446938091C52C909144
:104C0000C62C827091702DB73EB72E5E3F4F0FB607
:104C1000F8943EBF0FBE2DBF892B41F08FEE9EE072
:104C20009F938F930E9446930F900F9083EC9EE08A
:104C30009F938F930E94469387E89EE09F938F9364
:104C40000E9446938EE59EE09F938F930E94469329
:104C500082E39EE09F938F930E94469383E09EE0C1
:104C60009F938F930E94469381ED9DE09F938F9336
:104C70000E94469380EA9DE09F938F930E94469303
:104C800086E69DE09F938F930E94469380E39DE08C
:104C90009F938F930E94469380E09DE09F938F9314
:104CA0000E94469384ED9CE09F938F930E944693CD
:104CB00085EA9CE09F938F930E9446938CE69CE04C
:104CC0009F938F930E94469383E39CE09F938F93DF
:104CD0000E9446938CEF9BE09F938F930E94469394
:104CE0008EEC9BE09F938F930E9446938DB79EB767
:104CF00080960FB6F8949EBF0FBE8DBF8AE99BE0E9
:104D00009F938F930E94469389E69BE09F938F9396
:104D10000E9446938AE39BE09F938F930E94469361
:104D20008BE09BE09F938F930E94469384EE9AE0E2
:104D30009F938F930E9446938EEA9AE09F938F935E
:104D40000E94469388E79AE09F938F930E94469330
:104D500082E49AE09F938F930E94469389E19AE0C0
:104D60009F938F930E94469381EE99E09F938F9338
:104D70000E94469386EB99E09F938F930E944693FF
:104D80002DB73EB72A5E3F4F0FB6F8943EBF0FBE19
:104D90002DBF089581ED93E00C946E934F925F9236
:104DA0006F927F928F929F92AF92BF92CF92DF923B
:104DB000EF92FF92CF93DF93CDB7DEB728970FB670
:104DC000F894DEBF0FBECDBF8091CB309091CC3038
:104DD000A091CD30B091CE3089839A83AB83BC83D0
:104DE0004090CB305090CC306090CD307090CE3031
:104DF0008091CB309091CC30A091CD30B091CE301D
:104E00008D839E83AF83B8876091CB307091CC3017
:104E10008091CD309091CE302CE3822E912CA12C1C
:104E2000B12CA50194010E94F5877F936F9330E127
:104E3000C32E3EE0D32EE12CF12C6D817E818F813B
:104E40009885A70196010E94F587A50194010E940B
:104E5000F5873F932F9340E8842E41E5942EAA24B2
:104E6000A394B12CC301B201A50194010E94F5875E
:104E7000A70196010E94F5873F932F9369817A815C
:104E80008B819C81A50194010E94F5873F932F930C
:104E900080E999E09F938F930E9446930FB6F89410
:104EA000DEBF0FBECDBF28960FB6F894DEBF0FBE93
:104EB000CDBFDF91CF91FF90EF90DF90CF90BF906B
:104EC000AF909F908F907F906F905F904F900895DC
:104ED000EDEFF9E3808191818234924479F0ED5FC6
:104EE000F943FF93EF9382E799E09F938F930E949A
:104EF00046930F900F900F900F9008953A96E53FCC
:104F000081E8F80738F30895CF93DF93EC018C9A8A
:104F10000E94A7109F938F937F936F9386E699E0EB
:104F20009F938F930E9446930F900F900F900F9036
:104F30000F900F90209719F00E94B81108C084E6D6
:104F400099E09F938F930E9446930F900F9081E07A
:104F50000E9459102091850230918602409187026B
:104F6000509188020E94C48D9F938F937F936F937B
:104F700088E599E09F938F930E9446930F900F903E
:104F80000F900F900F900F90209719F00E94B8117A
:104F900008C086E599E09F938F930E9446930F90F7
:104FA0000F9082E00E94591020918102309182027C
:104FB00040918302509184020E94C48D9F938F93ED
:104FC0007F936F938AE499E09F938F930E94469317
:104FD0000F900F900F900F900F900F90209719F057
:104FE0000E94B81108C088E499E09F938F930E94B3
:104FF00046930F900F9083E00E9459109F938F93D8
:105000007F936F9389E399E09F938F930E944693D8
:105010008C980F900F900F900F900F900F902097FB
:1050200019F00E94B81108C087E399E09F938F930D
:105030000E9446930F900F908091C52C87FF83C0EC
:1050400021E042E161E080ED0E94DC619F938F935B
:105050007F936F938AE299E09F938F930E94469388
:105060000F900F900F900F900F900F90209719F0C6
:105070000E94B81108C088E299E09F938F930E9424
:1050800046930F900F9021E042E162E080ED0E9494
:10509000DC619F938F937F936F938BE199E09F9354
:1050A0008F930E9446930F900F900F900F900F9048
:1050B0000F90209719F00E94B81108C089E199E07B
:1050C0009F938F930E9446930F900F9021E042E1AF
:1050D00063E080ED0E94DC619F938F937F936F93D9
:1050E0008CE099E09F938F930E9446930F900F90CE
:1050F0000F900F900F900F90CD2B19F00E94B811C8
:1051000008C08AE099E09F938F930E9446930F9086
:105110000F9021E042E164E080ED0E94DC619F930A
:105120008F937F936F938DEF98E09F938F930E945F
:1051300046930F900F900F900F900F900F90DF916C
:10514000CF910C94B811CD2BD1F3DF91CF9108956D
:105150000F931F93CF93DF93882389F049E050E0AA
:105160006FEF70E08EE895E30E94809249E050E096
:105170006EE070E08EE895E30E94119613C0CEE8D1
:10518000D5E308EF18E089911F928F931F930F9337
:105190000E9446930F900F900F900F9085E3C639B1
:1051A000D80789F7DF91CF911F910F910C94B81117
:1051B000882311F0299A089529980895882311F0D9
:1051C0002A9A08952A980895CF92DF92EF92FF923B
:1051D000CF93DF936B017C0160FF11C08EE094E000
:1051E0009F938F938CEE90E19F938F930E944693B1
:1051F0000F900F900F900F9081E090E002C080E040
:1052000090E0C1FE09C0EC01219648E259E063E15B
:1052100074E00E942116CE01C2FE09C0EC01219665
:1052200048E259E06BE174E00E942116CE01C3FE12
:1052300009C0EC01219648E259E063E274E00E9463
:105240002116CE01C4FE09C0EC01219648E259E0C6
:1052500063E975E00E942116CE01C5FE09C0EC018C
:10526000219648E259E067E274E00E942116CE01DF
:10527000C6FE09C0EC01219648E259E06BE274E0F9
:105280000E942116CE01C7FE09C0EC01219648E21A
:1052900059E061E374E00E942116CE01D0FE09C0FE
:1052A000EC01219648E259E069E374E00E9421167E
:1052B000CE01D1FE09C0EC01219648E259E061E43B
:1052C00074E00E942116CE01D2FE09C0EC012196A5
:1052D00048E259E065E474E00E942116CE01209175
:1052E000C52C3091C62C24703270232B59F0D3FE7C
:1052F00009C0EC01219648E259E06BE474E00E9499
:105300002116CE012091C52C23FF0BC0D4FE09C06D
:10531000EC01219648E259E060E574E00E94211614
:10532000CE012091C52C24FF0BC0D5FE09C0EC0195
:10533000219648E259E066E574E00E942116CE010C
:10534000D6FE09C0EC01219648E259E06EE574E012
:105350000E942116CE01D7FE09C0EC01219648E239
:1053600059E069E674E00E942116CE01E0FE0CC00F
:1053700048E259E06AE774E0DF91CF91FF90EF9047
:10538000DF90CF900C942116CD28CE28CF2841F461
:1053900083EF98E09F938F930E9446930F900F9016
:1053A000DF91CF91FF90EF90DF90CF900895CF9253
:1053B000DF92EF92FF92CF93DF93EC01C12CD12CBF
:1053C0007601209709F4A3C06EEE78E0CE010E942A
:1053D0005292892B11F46894C0F866EE78E0CE0101
:1053E0000E945292892B11F46894C1F86EED78E016
:1053F000CE010E945292892B11F46894C2F86AED92
:1054000078E0CE010E945292892B11F46894C3F87F
:1054100067ED78E0CE010E945292892B11F46894D6
:10542000C4F863ED78E0CE010E945292892B11F40A
:105430006894C5F86DEC78E0CE010E945292892BF9
:1054400011F46894C6F865EC78E0CE010E9452929F
:10545000892B11F46894C7F86DEB78E0CE010E94B7
:105460005292892B11F46894D0F869EB78E0CE0160
:105470000E945292892B11F46894D1F863EB78E082
:10548000CE010E945292892B11F46894D2F86EEAF0
:1054900078E0CE010E945292892B11F46894D3F8DF
:1054A00068EA78E0CE010E945292892B11F4689448
:1054B000D4F860EA78E0CE010E945292892B11F470
:1054C0006894D5F865E978E0CE010E945292892B64
:1054D00011F46894D6F864E878E0CE010E94529204
:1054E000892B11F46894D7F86FE778E0CE010E9419
:1054F0005292892B11F46894E0F860917E027091C9
:105500007F0280E090E00E946692EC015ACFC701D2
:10551000B601DF91CF91FF90EF90DF90CF9008958B
:10552000AF92BF92CF92DF92EF92FF920F931F93B1
:10553000CF93DF93D22FC32F8A01F62EC72ED82EFA
:10554000E92E217030E040E050E060E070E080E063
:1055500090E0A0E00E94288A89F08FE794E09F9372
:105560008F938CEE90E19F938F930E9446930F90C0
:105570000F900F900F90E1E0F0E002C0E0E0F0E06B
:105580008091C52C80FF19C02D2F247030E040E0A1
:1055900050E060E070E080E090E0A0E00E94288AA7
:1055A00061F05F018FEFA81AB80A48E259E063E89A
:1055B00074E0CF010E942116F5012D2F227030E0FA
:1055C00040E050E060E070E080E090E0A0E00E9409
:1055D000288A61F05F018FEFA81AB80A48E259E003
:1055E00067E874E0CF010E942116F5012D2F287085
:1055F00030E040E050E060E070E080E090E0A0E06B
:105600000E94288A61F05F018FEFA81AB80A48E269
:1056100059E06FE974E0CF010E942116F5012D2FAA
:10562000207130E040E050E060E070E080E090E029
:10563000A0E00E94288A61F05F018FEFA81AB80AE3
:1056400048E259E06AE874E0CF010E942116F501B2
:105650002D2F207230E040E050E060E070E080E00C
:1056600090E0A0E00E94288A61F05F018FEFA81A05
:10567000B80A48E259E06DE874E0CF010E942116B3
:10568000F5012D2F207430E040E050E060E070E044
:1056900080E090E0A0E00E94288A61F05F018FEF37
:1056A000A81AB80A48E259E063E974E0CF010E9401
:1056B0002116F5012D2F207830E040E050E060E029
:1056C00070E080E090E0A0E00E94288A61F05F0135
:1056D0008FEFA81AB80A48E259E069E974E0CF01EF
:1056E0000E942116F50120E03C2F317040E050E08F
:1056F00060E070E080E090E0A0E00E94288A61F025
:105700005F018FEFA81AB80A48E259E06CE974E02B
:10571000CF010E942116F50120E03C2F327040E0BD
:1057200050E060E070E080E090E0A0E00E94288A15
:1057300061F05F018FEFA81AB80A48E259E061EA08
:1057400074E0CF010E942116F50120E03C2F347057
:1057500040E050E060E070E080E090E0A0E00E9477
:10576000288A61F05F018FEFA81AB80A48E259E071
:1057700068EA74E0CF010E942116F50120E03C2F79
:10578000387040E050E060E070E080E090E0A0E041
:105790000E94288A61F05F018FEFA81AB80A48E2D8
:1057A00059E06BEA74E0CF010E942116F50120E078
:1057B0003C2F307140E050E060E070E080E090E02D
:1057C000A0E00E94288A61F05F018FEFA81AB80A52
:1057D00048E259E060EB74E0CF010E942116F50128
:1057E00020E03C2F307240E050E060E070E080E06C
:1057F00090E0A0E00E94288A61F05F018FEFA81A74
:10580000B80A48E259E067EB74E0CF010E94211624
:10581000F50120E030E040E050E06F2D647070E072
:1058200080E090E0A0E00E94288A61F05F018FEFA5
:10583000A81AB80A48E259E06EEB74E0CF010E9462
:105840002116F5018091C52C81FF19C020E03C2F65
:10585000307440E050E060E070E080E090E0A0E074
:105860000E94288A61F05F018FEFA81AB80A48E207
:1058700059E062EC74E0CF010E942116F50180919D
:10588000C52C9091C62C90FF19C020E030E040E07C
:10589000512F507160E070E080E090E0A0E00E9445
:1058A000288A61F05F018FEFA81AB80A48E259E030
:1058B00065EC74E0CF010E942116F5018091C52CA2
:1058C0009091C62C90FF19C020E030E040E0512FAD
:1058D000507260E070E080E090E0A0E00E94288AD2
:1058E00061F05F018FEFA81AB80A48E259E068EC4E
:1058F00074E0CF010E942116F5018091C52C909192
:10590000C62C90FF19C020E030E040E0512F5074C9
:1059100060E070E080E090E0A0E00E94288A61F002
:105920005F018FEFA81AB80A48E259E06EEC74E004
:10593000CF010E942116F50120E03C2F307840E095
:1059400050E060E070E080E090E0A0E00E94288AF3
:1059500061F05F018FEFA81AB80A48E259E069EDDB
:1059600074E0CF010E942116F50120E030E0402FC5
:10597000417050E060E070E080E090E0A0E00E94C4
:10598000288A61F05F018FEFA81AB80A48E259E04F
:105990006EED74E0CF010E942116F50120E030E0A9
:1059A000402F427050E060E070E080E090E0A0E0C6
:1059B0000E94288A61F05F018FEFA81AB80A48E2B6
:1059C00059E061EE74E0CF010E942116F50120E05C
:1059D00030E040E050E06F2D687070E080E090E0D3
:1059E000A0E00E94288A61F05F018FEFA81AB80A30
:1059F00048E259E064EE74E0CF010E942116F501FF
:105A000020E030E040E050E06F2D607170E080E019
:105A100090E0A0E00E94288A61F05F018FEFA81A51
:105A2000B80A48E259E068EE74E0CF010E942116FE
:105A3000F5018091C52C87FF19C020E030E0402F90
:105A4000487050E060E070E080E090E0A0E00E94EC
:105A5000288A61F05F018FEFA81AB80A48E259E07E
:105A60006CEE74E0CF010E942116F5018091C52CE7
:105A700087FF19C020E030E0402F407150E060E027
:105A800070E080E090E0A0E00E94288A61F05F0171
:105A90008FEFA81AB80A48E259E060EF74E0CF012E
:105AA0000E942116F5018091C52C87FF19C020E0C6
:105AB00030E0402F407250E060E070E080E090E025
:105AC000A0E00E94288A61F05F018FEFA81AB80A4F
:105AD00048E259E064EF74E0CF010E942116F5011D
:105AE0008091C52C87FF19C020E030E0402F407422
:105AF00050E060E070E080E090E0A0E00E94288A42
:105B000061F05F018FEFA81AB80A48E259E068EF28
:105B100074E0CF010E942116F5018091C52C82FF0F
:105B200019C020E030E0402F407850E060E070E0A5
:105B300080E090E0A0E00E94288A61F05F018FEF92
:105B4000A81AB80A48E259E066E276E0CF010E945E
:105B50002116F5018091C52C82FF19C020E030E0AC
:105B600040E0512F517060E070E080E090E0A0E0F4
:105B70000E94288A61F05F018FEFA81AB80A48E2F4
:105B800059E06CEF74E0CF010E942116F50180917D
:105B9000C52C9091C62C90FF19C020E030E040E069
:105BA000512F527060E070E080E090E0A0E00E9431
:105BB000288A61F05F018FEFA81AB80A48E259E01D
:105BC0006FEF74E0CF010E942116F5018091C52C82
:105BD0009091C62C90FF19C020E030E040E0512F9A
:105BE000547060E070E080E090E0A0E00E94288ABD
:105BF00061F05F018FEFA81AB80A48E259E067E048
:105C000075E0CF010E942116F5018091C52C90917D
:105C1000C62C91FF1EC020E030E040E0512F5870AC
:105C200060E070E080E090E0A0E00E94288A89F0C7
:105C300048E259E060E175E0CF01DF91CF911F911B
:105C40000F91FF90EF90DF90CF90BF90AF900C94AA
:105C500021162D2F3C2FA8016F2D7C2D8D2D9E2DD3
:105C6000A0E00E94288A41F48AE798E09F938F93EE
:105C70000E9446930F900F90DF91CF911F910F914B
:105C8000FF90EF90DF90CF90BF90AF900895AF92CC
:105C9000BF92DF92EF92FF920F931F93CF93DF9308
:105CA000EC015B01FB01108265E778E00E945292F3
:105CB000892B59F58091C52C3DE4F32E00E882FF35
:105CC00003C024E8E22E02C094E0E92E10E0D12CBB
:105CD00081FD00EC26E04AE250E06BE270E089E2F0
:105CE00090E00E94BF5D81E090E00E945011882307
:105CF00011F08DE5F82E8091C52C9091C62C90FD69
:105D000016E091FF07C0186005C0F12C00E0E12CFF
:105D100010E0D12C63E778E0CE010E945292892BEB
:105D200061F481E0F501808360917E0270917F02D1
:105D300080E090E00E946692EC0161E778E0CE019D
:105D40000E945292892B61F48FEFF501808360915C
:105D50007E0270917F0280E090E00E946692EC01EA
:105D6000209709F438C16DE678E0CE010E94529286
:105D7000892B19F4FF2DF160FF2E69E678E0CE0142
:105D80000E945292892B19F48F2D8460F82E66E6BA
:105D900078E0CE010E945292892B19F4EF2DE26037
:105DA000FE2E64E678E0CE010E945292892B19F40F
:105DB000FF2DF860FF2E61E678E0CE010E9452923E
:105DC000892B19F48F2D8061F82E6BE578E0CE01D8
:105DD0000E945292892B19F4EF2DE062FE2E65E5A8
:105DE00078E0CE010E945292892B19F4FF2DF064C5
:105DF000FF2E62E578E0CE010E945292892B19F4C1
:105E00008F2D8068F82E6DE478E0CE010E945292CA
:105E1000892B09F4016066E478E0CE010E94529279
:105E2000892B09F4026063E478E0CE010E9452926B
:105E3000892B09F404606EE378E0CE010E9452924F
:105E4000892B09F4086067E378E0CE010E94529242
:105E5000892B09F4006160E378E0CE010E94529240
:105E6000892B09F400626CE278E0CE010E94529224
:105E7000892B19F4ED2DE460DE2E69E278E0CE0185
:105E80000E945292892B09F4006464E278E0CE010A
:105E90000E945292892B09F4006861E278E0CE01F9
:105EA0000E945292892B19F4FE2DF160EF2E6EE1C3
:105EB00078E0CE010E945292892B19F48E2D8260D7
:105EC000E82E6BE178E0CE010E945292892B19F402
:105ED000EE2DE460EE2E67E178E0CE010E94529252
:105EE000892B19F4FE2DF860EF2E63E178E0CE01E6
:105EF0000E945292892B19F48E2D8061E82E6FE05A
:105F000078E0CE010E945292892B19F4EE2DE062C6
:105F1000EE2E6BE078E0CE010E945292892B19F4AC
:105F2000FE2DF064EF2E69E078E0CE010E945292DF
:105F3000892B19F48E2D8068E82E66E078E0CE017A
:105F40000E945292892B09F411606EEF77E0CE0126
:105F50000E945292892B09F4126065EF77E0CE011E
:105F60000E945292892B09F414606CEE77E0CE0106
:105F70000E945292892B09F4186069EE77E0CE01F5
:105F80000E945292892B09F4106163EE77E0CE01F2
:105F90000E945292892B09F4106268ED77E0CE01DD
:105FA0000E945292892B09F4106464ED77E0CE01CF
:105FB0000E945292892B19F4ED2DE860DE2E60EDDF
:105FC00077E0CE010E945292892B09F0C0CEFD2DC0
:105FD000F061DF2EBCCE2F2D302F4E2D512F6D2D89
:105FE00070E080E090E0DF91CF911F910F91FF90E2
:105FF000EF90DF90BF90AF9008955F926F927F9285
:106000008F929F92AF92BF92CF92DF92EF92FF92C8
:106010000F931F93CF93DF93782EC8EADCE100E063
:1060200010E08AECE82E87E0F82E872D8170582E3C
:10603000872D8270682E95EBC92E97E0D92E2DEB17
:10604000A22E27E0B22E3BEB832E37E0932E772053
:1060500051F01F930F93FF92EF920E9446930F907F
:106060000F900F900F905520A1F089858F93888510
:106070008F93BF92AF920E9446930F900F900F9014
:106080000F906620C1F09F928F920E9446930F90CE
:106090000F90662081F0DF92CF920E944693288174
:1060A00039814A815B816C817D818E819F810E94D3
:1060B000902A0F900F900E94B8110F5F1F4F2A96E1
:1060C0000430110521F6DF91CF911F910F91FF90C0
:1060D000EF90DF90CF90BF90AF909F908F907F9088
:1060E0006F905F90089580EB97E09F938F930E944D
:1060F00046938091B5289091B628A091B728B09189
:10610000B8280F900F90813027EA92072EE1A2075E
:10611000B10519F482EA97E01DC0823026EA9207A1
:106120002EE1A207B10519F485E997E013C082308A
:1061300027EA92072EE1A207B10519F487E897E054
:1061400009C0823028EA92072EE1A207B10549F47E
:1061500089E797E09F938F930E9446930F900F904B
:106160000895BF93AF939F938F9383E797E09F9397
:106170008F930E9446930F900F900F900F900F9067
:106180000F90089583E697E09F938F930E94469324
:106190000E94CA260E9473300E94B8118FE89CE1C9
:1061A0009F938F938BE597E09F938F930E944693E5
:1061B000609160027091610280916202909163022D
:1061C00028EE33E040E050E00E94F5875F934F9364
:1061D0003F932F938BE497E09F938F930E94469376
:1061E00082E497E09F938F930E9446930E944A1601
:1061F0008091C52C2DB73EB7225F3F4F0FB6F89464
:106200003EBF0FBE2DBF80FF05C041E061E081E0D1
:106210000E94F7178EE397E09F938F930E94469317
:1062200080E00E94A8280E94CE26809165021F92DD
:106230008F9385E397E09F938F930E94469380917D
:106240009C131F928F938CE297E09F938F930E94F1
:106250004693809190028F9380918F028F938091CB
:106260008E028F9380918D028F938EE197E09F93A2
:106270008F930E9446931F9280E48F9386E097E06D
:106280009F938F930E9446938091A4371F928F9380
:106290008091A3371F928F9383EF96E09F938F9304
:1062A0000E944693809164021F928F938AEE96E03B
:1062B0009F938F930E94469380916602909167020C
:1062C000A0916802B09169022DB73EB7225E3F4FA0
:1062D0000FB6F8943EBF0FBE2DBF96FD03C08CE1F4
:1062E00095E002C089E195E09F938F9380EE96E060
:1062F0009F938F930E94469383E00E94FD2F0F90FF
:106300000F900F900F901D9903C08CE195E002C093
:1063100089E195E09F938F9384ED96E09F938F930F
:106320000E9446938AEC96E09F938F930E94469337
:10633000809166020F900F900F900F900F900F902A
:1063400081FF09C084EC96E09F938F930E9446934F
:106350000F900F9013C080FD03C08CE195E002C048
:1063600089E195E09F938F9380EC96E09F938F93C4
:106370000E9446930F900F900F900F9080916602AD
:1063800090916702A0916802B091690297FD03C0E5
:106390008CE195E002C089E195E09F938F9387EBB4
:1063A00096E09F938F930E94469380EB96E09F9395
:1063B0008F930E94469360919F137091A0138091D8
:1063C000A1139091A2130E94E4280E94B8110F908B
:1063D0000F900F900F900F900F90779B03C08CE160
:1063E00095E002C089E195E09F938F9387EA96E05C
:1063F0009F938F930E9446930E943B0E0E940C1124
:106400009F938F937F936F9389E996E09F938F93E8
:106410000E9446930E94BB109F938F937F936F932C
:106420008BE896E09F938F930E94469381E090E0E3
:106430000E9484278091743590917535A0917635AE
:10644000B0917735BF93AF939F938F938DE796E08D
:106450009F938F930E944693809189358F9380916B
:1064600088358F93809187358F93809186358F9370
:1064700089E696E09F938F930E94469380917835AA
:1064800090917935A0917A35B0917B35BF93AF93D8
:106490009F938F938BE596E09F938F930E944693F3
:1064A0008DB79EB782960FB6F8949EBF0FBE8DBF74
:1064B00080918D358F9380918C358F9380918B3522
:1064C0008F9380918A358F9387E496E09F938F9383
:1064D0000E94469361E070E080E090E00E94C1116C
:1064E00061E070E081E090E00E94C1110F900F9098
:1064F0000F900F900F900F90299903C08CE195E0B9
:1065000002C089E195E09F938F938FE396E09F937C
:106510008F930E9446930F900F900F900F902A999F
:1065200003C08CE195E002C089E195E09F938F93D1
:1065300087E396E09F938F930E9446930F900F906E
:106540000F900F900895F89491E2E0E0F0E09093BE
:1065500057008491E2E0F0E0909357002491E4E04A
:10656000F0E090935700E49190E0A0E0B0E0BC012F
:1065700055274427822F90E0A0E0B0E0BA2FA92F42
:10658000982F8827840F951FA61FB71F8E0F911D68
:10659000A11DB11D8093B5289093B628A093B7286C
:1065A000B093B82878940895CF93DF93CDB7DEB732
:1065B00061970FB6F894DEBF0FBECDBF48E250E042
:1065C00062E270E088EA9CE10E94F3952091A81CA9
:1065D0003091A91C4091AA1C5091AB1C6091AC1C3D
:1065E0007091AD1C8091AE1C9091AF1CAFEF0E94DA
:1065F000288A09F05DC08DE48093A81C80E8809310
:10660000A91C84E08093AA1C1092AB1C1092AC1CB5
:106610001092AD1C1092AE1C1092AF1C8CE390E057
:106620009093B11C8093B01C1092B21C1092B31CBA
:106630001092B41C1092B51C1092B61C1092B71C8C
:106640001092B81C1092B91C1092BB1C1092BA1C6C
:106650001092BC1C1092BD1C1092BE1C1092BF1C4C
:106660001092C01C1092C11C1092C21C1092C31C2C
:106670001092C51C1092C41C1092C61C1092C71C0C
:106680001092C81C1092C91C1092CA1C1092CB1CEC
:106690001092CC1C1092CD1C1092CF1C1092CE1CCC
:1066A00048E250E062E270E088EA9CE10E941196C4
:1066B00044E050E06EE170E0CE010B960E94F3954D
:1066C0008B859C85AD85BE858F3F2FEF9207A207F6
:1066D000B207A9F48AE090E4A0E0B0E080936602FB
:1066E00090936702A0936802B093690244E050E07F
:1066F0006EE170E086E692E00E94119608C08093F9
:10670000660290936702A0936802B0936902809139
:10671000660290916702A0916802B0916902A2FF9F
:1067200002C02A9A03C080E00E94DE2844E050E0C4
:106730006AE570E0CE010B960E94F3958B859C85EF
:10674000AD85BE858F3F2FEF9207A207B20789F470
:1067500010929F131092A0131092A1131092A213E3
:1067600044E050E06AE570E08FE993E10E94119601
:1067700008C080939F139093A013A093A113B0938C
:10678000A21349E050E06EE070E08EE895E30E94CD
:10679000F3950E94EF1244E050E06EE470E0CE0109
:1067A0000B960E94F3958B859C85AD85BE8544E054
:1067B00050E06EE470E08F3F9F4FAF4FBF4F29F422
:1067C00085E892E00E94119604C085E892E00E945C
:1067D000F39544E050E06AE470E0CE010B960E942D
:1067E000F3958B859C85AD85BE8544E050E06AE4D9
:1067F00070E08F3F9F4FAF4FBF4F29F481E892E089
:106800000E94119604C081E892E00E94F39544E052
:1068100050E062E570E0CE010B960E94F3958B8507
:106820009C85AD85BE8544E050E062E570E08F3F19
:106830009F4FAF4FBF4F29F489E892E00E94119615
:1068400004C089E892E00E94F39541E050E06DE1D8
:1068500070E0CE0141960E94F395898941E050E0B5
:106860006DE170E08F3F29F48CE993E10E9411966D
:1068700004C08CE993E10E94F39541E050E06CE1A3
:1068800070E0CE0141960E94F395898941E050E085
:106890006CE170E08F3F29F485E692E00E9411964A
:1068A00004C085E692E00E94F39541E050E06BE180
:1068B00070E0CE0141960E94F395898941E050E055
:1068C0006BE170E08F3F29F484E692E00E9411961C
:1068D00004C084E692E00E94F3954AE050E064E050
:1068E00070E0CE0101960E94F39589814AE050E064
:1068F00064E070E08F3F29F48FE89CE10E941196DC
:1069000004C08FE89CE10E94F39544E050E066E506
:1069100070E0CE010B960E94F3958B859C85AD852A
:10692000BE8544E050E066E570E08F3F9F4FAF4F7B
:10693000BF4F29F48DE892E00E94119604C08DE8C3
:1069400092E00E94F39544E050E067E170E0CE01F0
:106950000B960E94F3958B859C85AD85BE8544E0A2
:1069600050E067E170E08F3F9F4FAF4FBF4F29F47A
:1069700080E692E00E94119604C080E692E00E94B8
:10698000F39542E050E062E070E0CE010F960E9485
:10699000F3958F85988942E050E062E070E08F3F88
:1069A000910529F485E993E10E94119604C085E9D7
:1069B00093E10E94F39542E050E060E070E0CE0188
:1069C0000F960E94F3958F85988942E050E060E031
:1069D00070E08F3F910529F483E993E10E941196BD
:1069E00004C083E993E10E94F39561960FB6F89491
:1069F000DEBF0FBECDBFDF91CF910895CF92DF9262
:106A0000EF92FF9260917E0270917F0280E090E0B1
:106A10000E94669260E275E00E948792892B09F0DD
:106A20003BC18DE48093A81C80E88093A91C84E07E
:106A30008093AA1C1092AB1C1092AC1C1092AD1C3F
:106A40001092AE1C1092AF1C8CE390E09093B11C9E
:106A50008093B01C1092B21C1092B31C1092B41C04
:106A60001092B51C1092B61C1092B71C1092B81C54
:106A70001092B91C1092BB1C1092BA1C1092BC1C34
:106A80001092BD1C1092BE1C1092BF1C1092C01C14
:106A90001092C11C1092C21C1092C31C1092C51CF3
:106AA0001092C41C1092C61C1092C71C1092C81CD5
:106AB0001092C91C1092CA1C1092CB1C1092CC1CB4
:106AC0001092CD1C1092CF1C1092CE1C48E250E0C8
:106AD00062E270E088EA9CE10E9411968AE090E40C
:106AE000A0E0B0E08093660290936702A0936802F2
:106AF000B093690244E050E06EE170E086E692E017
:106B00000E94119610929F131092A0131092A1133D
:106B10001092A21344E050E06AE570E08FE993E13F
:106B20000E94119682E2C82EDD24DA948CECE82EC5
:106B30008BE3F82EC0928502D0928602E092870203
:106B4000F092880244E050E06EE470E085E892E064
:106B50000E941196C0928102D0928202E09283023A
:106B6000F092840244E050E06AE470E081E892E050
:106B70000E94119687ED94E3AFEEBCE38093890207
:106B800090938A02A0938B02B0938C0244E050E071
:106B900062E570E089E892E00E9411968AE999E93D
:106BA000A9E1B0E480938D0290938E02A0938F02AE
:106BB000B093900244E050E066E570E08DE892E02A
:106BC0000E94119610929C1380E00E94316A41E06D
:106BD00050E06DE170E08CE993E10E9411968AE14A
:106BE000809365020E940A6941E050E06CE170E028
:106BF00085E692E00E9411968FE08093640241E066
:106C000050E06BE170E084E692E00E9411968AE029
:106C1000EFE8FCE1DF011D928A95E9F74AE050E0D8
:106C200064E070E0CF010E94119680EA96E8A1E04E
:106C3000B0E08093600290936102A0936202B093EF
:106C4000630244E050E067E170E080E692E00E9479
:106C50001196109296131092951342E050E062E064
:106C600070E085E993E10E941196109294131092BE
:106C7000931342E050E060E070E083E993E10E940A
:106C8000119681E00E94A82880E090E0FF90EF90AC
:106C9000DF90CF900C940413FF90EF90DF90CF9093
:106CA00008950E942D666C9A6B9A6A9A6F9A729AEE
:106CB000749A739A779A809880B3897F80BB8398FF
:106CC000849887E080937E00549A0E94A3320E94A9
:106CD000D4320E94A90E80E090E00E9404136091DB
:106CE00060027091610280916202909163020E9441
:106CF00003600E94BB106093C7307093C8308093CC
:106D0000C9309093CA308091660286FD239A219AF9
:106D1000229A239A0E94BE0E1D9B05C010929E13BC
:106D200010929D13089581E090E090939E138093BC
:106D30009D130895CF93DF9390E040919F1350915E
:106D4000A0136091A1137091A21341FD08C020917E
:106D5000660220FD04C021FF8CC01D9B8AC02DE867
:106D6000289FE001299FD00D1124CE018B54924E13
:106D70009F938F9387E295E09F938F930E94329326
:106D8000FE01E255F24EDF01AA57BF4F2C910F9042
:106D90000F900F900F90438154816581768180918F
:106DA000CB309091CC30A091CD30B091CE30841BBF
:106DB000950BA60BB70B2223D1F1BF93AF939F93F3
:106DC0008F93DF01A257BF4F11968C9111978F932C
:106DD0008C918F93129711968C9111978F938C9120
:106DE0008F9313978C911F928F9311978C911F9271
:106DF0008F9313968C911F928F9311978C911F9262
:106E00008F93E957FF4F80811F928F931F922F938B
:106E10008DE295E09F938F930E9432938DB79EB73A
:106E200046960FB6F8949EBF0FBE8DBF10C0BF939D
:106E3000AF939F938F9384E795E09F938F930E94E6
:106E400032930F900F900F900F900F900F900E9421
:106E5000B81180918002882361F01F928F9380EF98
:106E600092E09F938F930E9446930F900F900F9004
:106E70000F90DF91CF9108958091AE1D882341F04E
:106E80008091AF1D90E00E949A360E94AF0FF4CF20
:106E90000895CF93DF93EC0188819981833E2EE0A2
:106EA0009207F1F018F4892BC1F04BC08B3E2EE015
:106EB000920709F44CC08F3E9E4009F042C086E51F
:106EC0009AE00E946F6E892B09F43FC086E59AE034
:106ED0000E945B6E80E00E94D82883EE9EE02EC068
:106EE000623199F5299A40919313509194135695D4
:106EF000542F44275795479560E070E086E59AE067
:106F00000E94516E80919F139091A013A091A113A4
:106F1000B091A213A0FF10C0809194138F93809121
:106F200093138F9381E991E19F938F930E944693EE
:106F30000F900F900F900F908BEE9EE099838883B7
:106F400004C01982188283E019C081E017C086E569
:106F50009AE00E946F6E892BC1F386E59AE00E9449
:106F60005B6E0E943C3740E250E060E070E086E5F6
:106F70009AE00E94516E8FEE9EE0E0CFDF91CF91BC
:106F800008952F923F924F925F926F927F928F92CD
:106F90009F92AF92BF92CF92DF92EF92FF920F93A8
:106FA0001F93CF93DF93CDB7DEB72B970FB6F8942F
:106FB000DEBF0FBECDBF9B878A873A01FC0180816F
:106FC0009181892B11F00C94EE4B60917E027091AF
:106FD0007F02CA010E94669260E870E0C3010E94CD
:106FE000A692009759F46091F7397091F8398AE0C8
:106FF00090E00E94FA9281E00C94F34B813091056D
:1070000061F4F3011081912E990C9908892C092DB6
:10701000292C392C492C592CB9C082309105B9F44E
:10702000F3018081082E000C990B982F882721816D
:10703000820F911D27FD9A95182F992E892E880C65
:107040008808082D282C382C482C582C9FC08330B9
:107050009105B1F5F3012081922F990F990B392FEA
:10706000492F592F692F792F892F00E10E94CA8952
:1070700019012A014B01B82FA92F2181922F990FB5
:10708000990B392F492F592F692F792F892F08E014
:107090000E94CA8959016A017B018C019101A201F8
:1070A000B4018B2F9A2F0E94018AA2801A2D110FF2
:1070B000110BB12EC12ED12EE12EF12E012F55C074
:1070C00004970CF45BC0F3012081922F990F990B68
:1070D000392F492F592F692F792F892F08E10E94C5
:1070E000CA8919012A014B01B82FA92F2181922F9A
:1070F000990F990B392F492F592F692F792F892FE4
:1071000000E10E94CA8959016A017B018C01910149
:10711000A201B4018B2F9A2F0E94018AA3801A2DFD
:10712000110F110BB12EC12ED12EE12EF12E012FF8
:107130000E94018A19012A014B01B82FA92F22812F
:10714000922F990F990B392F492F592F692F792F8A
:10715000892F08E00E94CA8959016A017B018C01CC
:107160009101A201B4018B2F9A2F0E94018A122F44
:10717000932E842E052F1B012C0108C01AE0912CA0
:10718000812C00E0212C312C412C512C0E94B81173
:10719000212F392D482D502FB101C2012537F3E69B
:1071A0003F07FDE64F075105610571058105910512
:1071B00011F40C94D6462537E3E63E07EDE64E077C
:1071C0005105610571058105910511F008F0B2C105
:1071D0002337F2E73F074105510561057105810538
:1071E000910511F40C946F492337E2E73E074105FE
:1071F0005105610571058105910511F008F0B9C0CF
:107200002536F4E63F074105510561057105810505
:10721000910509F4D1C72536E4E63E07410551053D
:10722000610571058105910511F008F041C0A6E7DF
:107230000E94288A11F40C945E430E94288A09F067
:1072400070F4A8E60E94288A11F40C942D41A5E759
:107250000E94288A11F40C9448430C94EC4B212F83
:10726000392D482D502FB101C2012436F1E63F07D8
:1072700041055105610571058105910511F40C94D5
:1072800097492537E2E63E0741055105610571053D
:107290008105910509F431C52A333642410551056E
:1072A000610571058105910509F430C30C94EC4B1F
:1072B000212F392D482D502FB101C2012737EFE67C
:1072C0003E0741055105610571058105910511F4E0
:1072D0000C943C472737FFE63F0741055105610500
:1072E00071058105910509F0C8F42436E9E63E07E9
:1072F00041055105610571058105910511F40C9455
:10730000214325363E46410551056105710581053C
:10731000910511F40C9470470C94EC4B212F392DEE
:10732000482D502FB101C2012536E2E73E07410545
:107330005105610571058105910511F40C943C48D6
:107340002936F2E73F0741055105610571058105C1
:10735000910511F40C941E49233331474105510521
:10736000610571058105910511F00C94EC4B0C94AD
:107370009749212F392D482D502FB101C2012236B6
:10738000F5E63F07F4E64F075105610571058105F4
:10739000910509F411C72236E5E63E07E4E64E07FB
:1073A0005105610571058105910511F008F05BC07B
:1073B0002133F4E63F07F1E64F07510561057105FA
:1073C0008105910509F4B6C22133E4E63E07E1E602
:1073D0004E075105610571058105910509F0C0F45D
:1073E0002337F3E73F074105510561057105810525
:1073F000910511F40C948349283734474105510510
:10740000610571058105910509F480C20C94EC4B6E
:10741000212F392D482D502FB101C2012837F4E614
:107420003F07F1E64F07510561057105810591059B
:1074300009F47CC22C36E5E73E07E2E64E0751052B
:10744000610571058105910509F457C42336344659
:1074500041465105610571058105910511F00C94B6
:10746000EC4B0C949749212F392D482D502FB10109
:10747000C2012D36E5E73E07E8E64E0751056105F6
:1074800071058105910511F40C94AD492D36F5E790
:107490003F07F8E64F075105610571058105910524
:1074A00009F0E0F42237E2E73E07E5E64E07510532
:1074B000610571058105910511F40C948746233609
:1074C0003D4648465105610571058105910511F05C
:1074D0000C94EC4B0E94541C0C94EE4B212F392D34
:1074E000482D502FB101C2012436E3E63E07ECE6F9
:1074F0004E075105610571058105910511F40C9444
:10750000EA452736FFE63F07FCE64F0751056105D0
:1075100071058105910511F40C94ED452336324334
:1075200049465105610571058105910511F00C94DD
:10753000EC4B20C2212F392D482D502FB101C20113
:107540002037FCE63F07F5E64F07F8E65F076105E1
:1075500071058105910509F480C62037ECE63E07E8
:10756000E5E64E07E8E65E076105710581059105D0
:1075700011F008F0E0C02437F8E73F07F4E74F07C1
:107580005105610571058105910511F40C94CA43FB
:107590002437E8E73E07E4E74E075105610571052A
:1075A0008105910511F008F05DC02033F1E33F073C
:1075B000F1E74F075105610571058105910511F44A
:1075C0000C9487462033E1E33E07E1E74E0751057F
:1075D000610571058105910509F0C0F42133F2E6DA
:1075E0003F07F0E74F0751056105710581059105DA
:1075F00009F498C2223332464047510561057105AE
:107600008105910509F4E3C20C94EC4B212F392D2F
:10761000482D502FB101C2012037F5E63F07F2E7B0
:107620004F075105610571058105910511F40C9411
:107630003C482C36E4E73E074E07510561057105CD
:107640008105910511F40C94124B213331434147CC
:107650005105610571058105910511F00C94EC4B04
:107660000C94D646212F392D482D502FB101C2013F
:107670002B36ECE63E07E5E74E07E2E65E076105DE
:1076800071058105910509F438C32B36FCE63F07E7
:10769000F5E74F07F2E65F07610571058105910582
:1076A00009F0E0F42437E4E63E07E7E74E0751052A
:1076B000610571058105910511F40C94604B243727
:1076C0003F464F465246610571058105910511F00F
:1076D0000C94EC4B0C9400000C94EE4B212F392DA4
:1076E000482D502FB101C2012E36E1E63E07E8E6F3
:1076F0004E07E3E65E07610571058105910511F40A
:107700000C949E432633F9E63F07F5E74F07F5E66D
:107710005F07610571058105910509F4A2C5293648
:107720003C4641465346610571058105910511F0BE
:107730000C94EC4B7FC3212F392D482D502FB101D4
:10774000C2012437F3E73F07F5E64F07F2E75F078B
:10775000610571058105910511F40C94EC472437FE
:10776000E3E73E07E5E64E07E2E75E0761057105E0
:107770008105910511F008F062C02337F5E63F0757
:10778000F2E74F07F0E75F07610571058105910595
:1077900011F40C945D4A2337E5E63E07E2E74E0715
:1077A000E0E75E07610571058105910509F0D0F4F8
:1077B0002136FDE63F07F5E74F07F8E65F0761056D
:1077C00071058105910511F40C945A47223737470A
:1077D00040475047610571058105910509F45CC278
:1077E0000C94EC4B212F392D482D502FB101C201A3
:1077F0002436FDE63F07F3E64F07F2E75F07610532
:1078000071058105910509F437C62136ECE63E077E
:10781000E5E64E07E2E75E07610571058105910522
:1078200009F43CC523373247474750476105710586
:107830008105910511F00C94EC4B0C94EF47212F2E
:10784000392D482D502FB101C2012437E2E73E0700
:10785000E1E64E07E5E75E076105710581059105E3
:1078600009F465C62437F2E73F07F1E64F07F5E76D
:107870005F07610571058105910509F0C8F424379A
:10788000E3E73E07E5E64E07E4E75E0761057105BD
:107890008105910509F4A9C7273730474847544760
:1078A000610571058105910509F41EC70C94EC4B27
:1078B000212F392D482D502FB101C2012F36ECE672
:1078C0003E07EFE54E07E6E75E07610571058105B6
:1078D000910509F47CC52C36F1E63F07F4E74F0724
:1078E000F8E75F07610571058105910511F40C94B6
:1078F000DF4A223737464047554761057105810504
:10790000910511F00C94EC4B0C94C64583E08093E8
:107910007C3510927E3510927D354CE755E362E15F
:1079200082E492E00E94E16F0C94EE4B0E94DD1B1A
:107930000C94EE4B21E042E161E080ED0E94DC61BD
:1079400021E042E161E080ED0E94DC6121E042E162
:1079500061E080ED0E94DC6121E042E161E080EDC8
:107960000E94DC6121E042E161E080ED0E94DC6187
:107970000C94EE4B60917E0270917F0280E090E06B
:107980000E94669260E875E00E948792892B09F058
:10799000C5C060917E0270917F0280E090E00E94FD
:1079A00066928C01009709F497C064E673E00E9428
:1079B0008792892BE1F488EE93E0A0E0B0E0809319
:1079C000600290936102A0936202B093630268EE3A
:1079D00073E080E090E00E94036044E050E067E1E3
:1079E00070E080E692E00E9411960C94EE4B66E8FF
:1079F00075E0C8010E948792892BE1F480E197E24B
:107A0000A0E0B0E08093600290936102A0936202D4
:107A1000B093630260E177E280E090E00E9403604F
:107A200044E050E067E170E080E692E00E94119649
:107A30000C94EE4B69E875E0C8010E948792892B8F
:107A4000E1F480EA96E8A1E0B0E0809360029093D0
:107A50006102A0936202B093630260EA76E881E07B
:107A600090E00E94036044E050E067E170E080E64F
:107A700092E00E9411960C94EE4B6DE875E0C801FF
:107A80000E948792892BE1F480E89AE1A6E0B0E0B9
:107A90008093600290936102A0936202B0936302AC
:107AA00060E87AE186E090E00E94036044E050E004
:107AB00067E170E080E692E00E9411960C94EE4B34
:107AC0008FE694E09F938F930E9446930E94B81193
:107AD0000F900F900C94EE4B6091600270916102D8
:107AE000809162029091630228EE33E040E050E022
:107AF0000E94F5875F934F933F932F938BE694E01B
:107B00009F938F930E9446930E94B8110F900F90FD
:107B10000F900F900F900F900C94EE4B0E944A160E
:107B20000C94EE4B60917E0270917F0280E090E0B9
:107B30000E9466928C0169E175E00E948792892B10
:107B4000A1F48091660290916702A0916802B091C1
:107B50006902A2608093660290936702A093680214
:107B6000B0936902299A0C94EE4B6CE175E0C80160
:107B70000E948792892BB1F48091660290916702EE
:107B8000A0916802B0916902AD7F809366029093E4
:107B90006702A0936802B093690280E00E94D8282F
:107BA0000C94EE4B299903C08CE195E002C089E169
:107BB00095E09F938F9383E694E09F938F930E9429
:107BC00046930F900F900F900F900C94EE4B609196
:107BD0007E0270917F0280E090E00E9466928C01AC
:107BE00069E175E00E948792892BE1F48091660239
:107BF00090916702A0916802B0916902A46080939D
:107C0000660290936702A0936802B09369022A9A71
:107C100044E050E06EE170E086E692E00E9411964A
:107C20000C94EE4B6CE175E0C8010E948792892BA1
:107C3000F1F48091660290916702A0916802B09180
:107C40006902AB7F8093660290936702A0936802FB
:107C5000B093690280E00E94DE2844E050E06EE1CB
:107C600070E086E692E00E9411960C94EE4B2A9901
:107C700003C08CE195E002C089E195E09F938F936A
:107C80008BE594E09F938F930E9446930F900F9003
:107C90000F900F900C94EE4B60917E0270917F02DA
:107CA00080E090E00E9466928C0169E175E00E949C
:107CB0008792892B19F477980C94EE4B6CE175E060
:107CC000C8010E948792892B19F4779A0C94EE4B85
:107CD000779B03C08CE195E002C089E195E09F931A
:107CE0008F9381E296E09F938F930E9446930F902B
:107CF0000F900F900F900C94EE4B60917E0270915C
:107D00007F0280E090E00E9466928C0161E975E05C
:107D10000E948792892BD1F48091AE1D1F928F9380
:107D20008091B01D1F928F938091AF1D1F928F93F2
:107D30001F9284E18F9381E394E09F938F930E943D
:107D400046930FB6F894DEBF0FBECDBF66E975E06F
:107D5000C8010E948792892B19F40E943C3766C0A3
:107D60006EE975E0C8010E948792892BF1F5609158
:107D70007E0270917F0280E090E00E946692009700
:107D800009F454C00E9453918531910528F59093D0
:107D900096138093951342E050E062E070E085E92D
:107DA00093E10E94119660917E0270917F0280E0C3
:107DB00090E00E9466920097C9F10E9453919093BF
:107DC00094138093931342E050E060E070E083E905
:107DD00093E10E9411962AC08FE194E09F938F93C4
:107DE0000E9446930F900F9021C0809196138F931D
:107DF000809195138F9386E194E09F938F930E94D7
:107E000046930E94B811809194138F93809193139D
:107E10008F9387E094E09F938F930E9446930E94F4
:107E2000B8110FB6F894DEBF0FBECDBF0E94B811D7
:107E30000C94EE4B60917E0270917F0280E090E0A6
:107E40000E9466928C016EED74E00E948792892BED
:107E500009F077C060917E0270917F0280E090E02F
:107E60000E9466928C01009711F40C94EE4B6CE921
:107E700075E00E948792892BB1F482E29FEFACEC0F
:107E8000BBE38093850290938602A0938702B09310
:107E9000880244E050E06EE470E085E892E00E94E1
:107EA00011960C94EE4B62EA75E0C8010E9487922D
:107EB000892BB1F482E29FEFACECBAE380938502A8
:107EC00090938602A0938702B093880244E050E02A
:107ED0006EE470E085E892E00E9411960C94EE4BFF
:107EE000C8010E944F912B013C0120E030E0A90124
:107EF0000E94138B8823D9F081E00E9459109B01C6
:107F0000AC01C301B2010E94188B6093850270938B
:107F10008602809387029093880244E050E06EE4EA
:107F200070E085E892E00E9411960C94EE4B8AEF87
:107F300093E09F938F930E9446930F900F900C9421
:107F4000EE4B61EE74E0C8010E948792892B09F024
:107F500077C060917E0270917F0280E090E00E9485
:107F600066928C01009711F40C94EE4B6CE975E06D
:107F70000E948792892BB1F482E29FEFACECBBE3C5
:107F80008093810290938202A0938302B093840233
:107F900044E050E06AE470E081E892E00E941196CB
:107FA0000C94EE4B62EA75E0C8010E948792892B1F
:107FB000B1F482E29FEFACECBAE38093810290933C
:107FC0008202A0938302B093840244E050E06AE40A
:107FD00070E081E892E00E9411960C94EE4BC8018B
:107FE0000E944F912B013C0120E030E0A9010E944A
:107FF000138B8823D9F082E00E9459109B01AC01B9
:10800000C301B2010E94188B6093810270938202B7
:10801000809383029093840244E050E06AE470E02D
:1080200081E892E00E9411960C94EE4B8DEE93E065
:108030009F938F930E9446930F900F900C94EE4B5A
:1080400069ED74E0C8010E948792892B09F073C022
:1080500060917E0270917F0280E090E00E946692C3
:108060008C01009711F40C94EE4B6CE975E00E94C2
:108070008792892BB1F487ED94E3AFEEBCE3809354
:10808000890290938A02A0938B02B0938C0244E001
:1080900050E062E570E089E892E00E9411960C944D
:1080A000EE4B62EA75E0C8010E948792892B51F479
:1080B0008EED93E09F938F930E9446930F900F90C5
:1080C0000C94EE4BC8010E944F912B013C0120E023
:1080D00030E0A9010E94138B882319F180E00E94EF
:1080E00059104B015C0121EE3AE744E95EE3C3011C
:1080F000B2010E94348AA50194010E94188B6093FA
:10810000890270938A0280938B0290938C0244E0E0
:1081100050E062E570E089E892E00E9411960C94CC
:10812000EE4B81ED93E09F938F930E9446930F90C7
:108130000F900C94EE4B0E94A7109F938F937F9308
:108140006F938AEC93E09F938F930E94469382E013
:108150000E94591020918102309182024091830245
:10816000509184020E94C48D162F072FF82EE92EFD
:1081700081E00E945910EF92FF920F931F9320917C
:1081800085023091860240918702509188020E94B8
:10819000C48D9F938F937F936F938EEB93E09F9308
:1081A0008F930E9446930E94B8110FB6F894DEBFD9
:1081B0000FBECDBF0C94EE4B60917E0270917F029A
:1081C00080E090E00E946692009711F10E94D7290A
:1081D00000919F131091A0132091A1133091A2132D
:1081E000601771078207930739F160939F137093AB
:1081F000A0138093A1139093A21344E050E06AE58A
:1082000070E08FE993E10E9411968AE196E002C046
:1082100083E196E09F938F930E94469360919F1312
:108220007091A0138091A1139091A2130E94E42851
:108230000E94B8110F900F9088E096E09F938F9363
:108240000E9446936FEF7FEFCB010E94E4280E94CB
:10825000B8110F900F900C94EE4B0E94C7250C9410
:10826000EE4BF3018481843329F440E061E080E047
:108270000E94F71780918002882311F40C94EE4B32
:108280001F928F9385E096E09F938F930E94469371
:108290000F900F900F900F900C94EE4BF301848190
:1082A000893709F080C060917E0270917F0280E082
:1082B00090E00E9466928C0169E175E00E948792CD
:1082C000892B51F48091660290916702A091680217
:1082D000B0916902906410C06CE175E0C8010E9421
:1082E0008792892BD1F48091660290916702A091C8
:1082F0006802B09169029F7B809366029093670247
:10830000A0936802B093690244E050E06EE170E02F
:1083100086E692E00E94119646C067EA75E0C801C1
:108320000E948792892B21F58091A71C8F938091C1
:10833000A61C8F938091A51C8F938091A41C8F9372
:108340008091A31C8F938091A21C8F938091A11C7C
:108350008F938091A01C8F9383E993E09F938F93D9
:108360000E9446930FB6F894DEBF0FBECDBF1BC070
:108370008091660290916702A0916802B0916902B3
:1083800096FD03C08CE195E002C089E195E09F93E2
:108390008F938FE893E09F938F930E9446930F9063
:1083A0000F900F900F9080918002882311F40C940D
:1083B000EE4B1F928F9382E096E09F938F930E94E3
:1083C00046930F900F900F900F900C94EE4BF3018B
:1083D00084818737E9F560917E0270917F0280E0A9
:1083E00090E00E9466920097D9F00E944F912B0175
:1083F0003C0120E030E0A9010E94138B882381F02A
:1084000040928D0250928E0260928F027092900282
:1084100044E050E066E570E08DE892E00E9411963D
:10842000809190028F9380918F028F9380918E0222
:108430008F9380918D028F9381E893E09F938F9328
:108440000E9446930F900F900F900F900F900F90F7
:1084500080918002882311F40C94EE4B1F928F932D
:108460008FEF95E09F938F930E9446930F900F900C
:108470000F900F900C94EE4B60917E0270917F02F2
:1084800080E090E00E9466928C0169E175E00E94B4
:1084900087924090660250906702609068027090E8
:1084A0006902892B19F4689457F809C06CE175E0EA
:1084B000C8010E948792892B99F4E89457F840925A
:1084C000660250926702609268027092690244E00C
:1084D00050E06EE170E086E692E00E94119613C0D3
:1084E00057FC03C08CE195E002C089E195E09F93C1
:1084F0008F938DE793E09F938F930E9446930F9005
:108500000F900F900F9080918002882311F40C94AB
:10851000EE4B1F928F938CEF95E09F938F930E9469
:1085200046930F900F900F900F900C94EE4B60912C
:108530007E0270917F0280E090E00E9466928C0142
:108540006DEA75E00E948792892B11F489E108C0D9
:1085500061EB75E0C8010E948792892B49F480E1A4
:108560008093C4001092C50082E08093C00055C083
:1085700065EB75E0C8010E948792892B11F488E0B1
:10858000EFCF6AEB75E0C8010E948792892B39F022
:108590006FEB75E0C8010E948792892B11F483E08C
:1085A000DFCF8091C400893141F488E793E09F9345
:1085B0008F930E9446930F900F908091C40080315A
:1085C00041F483E793E09F938F930E9446930F902B
:1085D0000F908091C400883041F48DE693E09F9322
:1085E0008F930E9446930F900F908091C400833028
:1085F00041F487E693E09F938F930E9446930F90F8
:108600000F908091C400883041F481E693E09F93FD
:108610008F930E9446930F900F9080918002882341
:1086200011F40C94EE4B1F928F9389EF95E09F937A
:108630008F930E9446930F900F900F900F900C9481
:10864000EE4B60917E0270917F0280E090E00E948C
:1086500066926CE975E00E948792892B11F481E0A3
:1086600001C080E00E94A82880918002882311F434
:108670000C94EE4B1F928F9386EF95E09F938F9310
:108680000E9446930F900F900F900F900C94EE4B1A
:108690000E94CE2680918002882311F40C94EE4B28
:1086A0001F928F9383EF95E09F938F930E94469341
:1086B0000F900F900F900F900C94EE4B0E94CA26D3
:1086C00080918002882311F40C94EE4B1F928F93BB
:1086D00080EF95E09F938F930E9446930F900F90A9
:1086E0000F900F900C94EE4B60917E0270917F0280
:1086F00080E090E00E9466920E945391803170F475
:1087000080939C130E94316A41E050E06DE170E07B
:108710008CE993E10E9411960C94EE4B80919C138E
:108720001F928F9387E593E09F938F930E944693C8
:108730000F900F900F900F900C94EE4B60917E0273
:1087400070917F0280E090E00E9466920E945391B7
:1087500095EF980F903170F4809365020E940A693A
:1087600041E050E06CE170E085E692E00E941196F5
:108770000C94EE4B809165021F928F938EE493E0F0
:108780009F938F930E9446930F900F900F900F909E
:108790000C94EE4B60917E0270917F0280E090E03D
:1087A0000E946692009789F04AE050E0BC018FE891
:1087B0009CE10E9497924AE050E064E070E08FE80C
:1087C0009CE10E9411960C94EE4B8FE89CE19F93E4
:1087D0008F9384EC95E09F938F930E9432930F9038
:1087E0000F900F900F900C94EE4B60917E02709161
:1087F0007F0280E090E00E9466928C0164E673E064
:108800000E948792892BD9F4219A809166029091D7
:108810006702A0916802B09169028061809366024C
:1088200090936702A0936802B093690244E050E01D
:108830006EE170E086E692E00E941196CFC762EE8C
:1088400074E0C8010E948792892BD9F4229A809102
:10885000660290916702A0916802B09169028062FD
:108860008093660290936702A0936802B0936902B6
:1088700044E050E06EE170E086E692E00E941196DE
:10888000ADC766E473E0C8010E948792892BD9F4D2
:10889000239A8091660290916702A0916802B0913C
:1088A000690280648093660290936702A0936802D5
:1088B000B093690244E050E06EE170E086E692E039
:1088C0000E9411968BC765E874E0C8010E948792E8
:1088D000892BD9F4239A8091660290916702A09126
:1088E0006802B09169028068809366029093670283
:1088F000A0936802B093690244E050E06EE170E03A
:1089000086E692E00E94119669C76EE373E0C801A3
:108910000E948792892B71F581E08093E03088EA8C
:108920009CE19093E2308093E1301092E430109219
:10893000E3308091660290916702A0916802B09145
:10894000690291608093660290936702A093680227
:10895000B093690244E050E06EE170E086E692E098
:108960000E94119640EE50E362E182E492E00E94A0
:10897000E16F34C76DE673E0C8010E948792892BCE
:1089800011F5E8EDFCE1119211922CE1E83FF207BC
:10899000D1F78091660290916702A0916802B09130
:1089A000690292608093660290936702A0936802C6
:1089B000B093690244E050E06EE170E086E692E038
:1089C0000E9411960BC76CE175E0C8010E94879266
:1089D000409166025091670260916802709169024D
:1089E000892BC1F44F705C7F4093660250936702FD
:1089F00060936802709369022B9A44E050E06EE144
:108A000070E086E692E00E941196809185350E9482
:108A10001F69E4C644FD03C08CE195E002C089E112
:108A200095E09F938F9383E493E09F938F930E94AD
:108A30004693809166020F900F900F900F9085FDE6
:108A400003C08CE195E002C089E195E09F938F938C
:108A500088E393E09F938F930E94469380916602F0
:108A60000F900F900F900F9086FD03C08CE195E062
:108A700002C089E195E09F938F938DE293E09F93ED
:108A80008F930E944693809166020F900F900F90F3
:108A90000F9087FD03C08CE195E002C089E195E06D
:108AA0009F938F9382E293E09F938F930E944693CC
:108AB0008091660290916702A0916802B09169026C
:108AC0000F900F900F900F9090FD03C08CE195E0F8
:108AD00002C089E195E09F938F9387E193E09F9394
:108AE0008F930E9446938091660290916702A091B5
:108AF0006802B09169020F900F900F900F9091FD56
:108B000003C08CE195E002C089E195E09F938F93CB
:108B10008CE093E09F938F930E944693809166022E
:108B200090916702A0916802B09169020F900F9036
:108B30000F900F9091FF52C68CEC95E00E946E93BF
:108B400098EDE92E9CE1F92E00E010E024ED822E54
:108B500025E0922EF70180819181F2E0EF0EF11C69
:108B60009F938F93C8010B969F938F939F928F92A1
:108B70000E9432930F5F1F4F0F900F900F900F9036
:108B80000F900F900031110529F728C68CEE95E063
:108B90009F938F930E944693809180020F900F9035
:108BA000882361F01F928F9389EE95E09F938F93B6
:108BB0000E9446930F900F900F900F90F89498E0BA
:108BC00088E10FB6F894A895809360000FBE90934B
:108BD0006000FFCF0E948D6101C660917E0270919E
:108BE0007F0280E090E00E9466928C0169E175E06E
:108BF0000E948792892BE9F40E940E688091660298
:108C000090916702A0916802B09169028D7F8160A6
:108C10008093660290936702A0936802B093690202
:108C200044E050E06EE170E086E692E00E9411962A
:108C3000D5C56CE175E0C8010E948792892BE1F4EB
:108C40000E9444678091660290916702A091680239
:108C5000B09169028C7F8093660290936702A09323
:108C60006802B093690244E050E06EE170E086E68D
:108C700092E00E941196B2C56FED75E0C8010E94A6
:108C80008792892BE9F40E94446780916602909153
:108C90006702A0916802B09169028E7F8260809322
:108CA000660290936702A0936802B093690244E061
:108CB00050E06EE170E086E692E00E9411968EC56B
:108CC0008091660281FF0FC08FED95E09F938F9397
:108CD00088E093E09F938F930E9446930F900F90AC
:108CE0000F900F907BC580FD03C08CE195E002C022
:108CF00089E195E09F938F9384E093E09F938F9316
:108D00000E9446930F900F900F900F9067C580912F
:108D1000DE308F938091DD308F938091DC308F93A4
:108D20008091DB308F938091DA308F938091D930AE
:108D30008F938091D8308F938091D7308F9380918B
:108D4000D6308F938091D5308F938091D4308F938C
:108D50008091D3308F938091D2308F938091D13096
:108D60008F938091D0308F938091CF308F938DEB04
:108D700095E09F938F930E9446930E94B811809133
:108D800080020FB6F894DEBF0FBECDBF882309F472
:108D900025C51F928F938AEB95E09F938F930E9436
:108DA00046930F900F900F900F9018C5F89489E09C
:108DB00021E030E0F90180935700C895E02C20E0D5
:108DC00030E0F90180935700C895F02C7894F8941E
:108DD00023E030E0F90180935700C895002D22E090
:108DE00030E0F90180935700C895102D7894809158
:108DF000B8288F938091B7288F938091B6288F934E
:108E00008091B5288F9380EB95E09F938F930E947C
:108E100046931F92EF921F92FF921F920F931F9201
:108E20001F9389E895E09F938F930E9446930E9439
:108E30006827809166001F928F938DE795E09F933E
:108E40008F930E9446930E94B811809180020FB6C2
:108E5000F894DEBF0FBECDBF882309F4BFC41F92B4
:108E60008F938AE795E09F938F930E9446930F908C
:108E70000F900F900F90B2C460E070E080E090E03F
:108E80000E94C11160E070E081E090E00E94C11199
:108E900080918002882309F4A1C41F928F9387E7F1
:108EA00095E09F938F930E9446930F900F900F90A1
:108EB0000F9094C40E948A250E94B811809180026C
:108EC000882309F48BC41F928F9384E795E09F93C6
:108ED0008F930E9446930F900F900F900F907EC437
:108EE00060917E0270917F0280E090E00E94669225
:108EF00066E975E00E948792892B31F5F89481E943
:108F00009AE00E94BA708C01892B69F0C8010F9613
:108F10000E94276DB80188E092E00E946771C80145
:108F20000E941B71F0CF81E99AE00E940E71892B9B
:108F300029F081E99AE00E94CE70F5CF81E99AE0AC
:108F40000E94B670789436C081E99AE00E94BA70A7
:108F50008C0184EEE82E85E0F82E0115110551F103
:108F6000F80186811F928F9380851F928F93858150
:108F70001F928F9381851F928F9387811F928F936A
:108F800084811F928F9383811F928F9382811F927E
:108F90008F9382851F928F93FF92EF920E9432935C
:108FA000C8010E941B718C010FB6F894DEBF0FBE82
:108FB000CDBFD3CF80918002882309F40FC41F92C4
:108FC0008F9381E795E09F938F930E9446930F9034
:108FD0000F900F900F9002C40E94FE34FFC3609167
:108FE0007E0270917F0280E090E00E9466928C0188
:108FF00063E276E00E948792892BD1F48091660229
:1090000090916702A0916802B0916902977F809366
:10901000660290936702A0936802B093690244E0ED
:1090200050E06EE170E086E692E00E941196D6C3B1
:1090300062EA75E0C8010E948792892BD1F4809181
:10904000660290916702A0916802B09169029860EF
:109050008093660290936702A0936802B0936902BE
:1090600044E050E06EE170E086E692E00E941196E6
:10907000B5C30E943B0EB2C360917E0270917F0225
:1090800080E090E00E946692FC0120812332C1F4CE
:109090004AE050E060E070E001960E94ED8E7B8334
:1090A0006A8360917E0270917F0280E090E00E946E
:1090B00066922A813B81243031050CF096C002C0B3
:1090C0001B821A82009709F490C01982BE016F5F5B
:1090D0007F4F0E94472E19013A014B01B82FA92F4B
:1090E0008AE02A813B81829FF001839FF00D112449
:1090F000E855F34E4080518032813C8383818D83DB
:1091000094819E8325812F83368138878781898743
:109110009101A301B4018B2F9A2F5201CC80DD80E5
:10912000EE80FF80088519850E941F8A09F460C0BF
:109130008981811103C0208231822AC0181684F4EB
:10914000422853289C81692A2D81722A3E81832AD4
:109150008F81982A9885B92B2985A22B408217C028
:10916000209430946094709480949094B095A095DD
:10917000242053203C8163228D8178229E81892284
:109180002F8192223885B3238985A823208251829A
:109190006282738284829582B683A78348E250E01C
:1091A00062E270E088EA9CE10E94119689E695E00F
:1091B0009F938F930E9446938AE02A813B81829FEE
:1091C000F001839FF00D1124E855F34E2081318189
:1091D0004281538164817581868197810E94902AA2
:1091E0000E94B8110F900F9003C082E00E94FD2FE3
:1091F0008DE595E09F938F930E9446932FEF3FEF6D
:109200004FEF5FEF6FEF7FEF8FEF9FEF0E94902A9E
:109210000E94B811809180020F900F90882309F46A
:10922000DDC21F928F938AE595E09F938F930E94F2
:1092300046930F900F900F900F90D0C260917E02D6
:1092400070917F0280E090E00E946692FC01208194
:109250002332A1F44AE050E060E070E001960E9401
:10926000ED8E8B0160917E0270917F0280E090E034
:109270000E94669204301105ECF402C000E010E098
:109280000097C1F04AE050E060E070E00E94189062
:109290002AE0209FF001219FF00D1124E855F34EA4
:1092A0007187608748E250E062E270E088EA9CE102
:1092B0000E94119681E00E94FD2F809180028823F8
:1092C00009F48CC21F928F9387E595E09F938F934B
:1092D0000E9446930F900F900F900F907FC20E94B4
:1092E000AA7180918002882309F478C21F928F931B
:1092F00084E595E09F938F930E9446930F900F9083
:109300000F900F906BC20E94C23080918002882320
:1093100009F464C21F928F9381E595E09F938F9328
:109320000E9446930F900F900F900F9057C280E0CD
:1093300090E00E94842780918002882309F44EC225
:109340001F928F938EE495E09F938F930E94469394
:109350000F900F900F900F9041C28091C52C81FF0C
:109360002DC00E941025892B49F58091BC288F9330
:109370008091BB288F938091BA288F938091B928D0
:109380008F9383E495E09F938F930E9446938091FF
:109390009D358F9380919C358F9380919B358F93D2
:1093A00080919A358F9386E395E09F938F930E94E7
:1093B00046930FB6F894DEBF0FBECDBF0E94B81122
:1093C0008091C52C9091C62C90FF63C081E090E005
:1093D0000E9488247B011C0180E090E00E94882488
:1093E0004B018C010E94E6233F922F92FF92EF9255
:1093F00085E295E09F938F930E9446931F930F936E
:109400009F928F9285E195E09F938F930E94469360
:10941000240138019401A80147018101B701C1016C
:109420000E9485229F938F937F936F938AE095E0AC
:109430009F938F930E944693242D352D462D572DB3
:109440006E2D792D822D912F0E94E6229F938F936E
:109450007F936F938CEF94E09F938F930E9446933A
:10946000242D352D462D572D6E2D792D822D912FA2
:109470000E9447239F938F937F936F9389EE94E08D
:109480009F938F930E9446930FB6F894DEBF0FBE52
:10949000CDBF0E94B81180918002882309F49EC13B
:1094A0001F928F9386EE94E09F938F930E94469332
:1094B0000F900F900F900F9091C18091C52C82FF5B
:1094C0002BC021E048E061E083E00E9462198091B6
:1094D000AC1D8F938091AB1D8F938091AA1D8F93AC
:1094E0008091A91D8F938091A81D8F938091A71DB6
:1094F0008F938091A61D8F938091A51D8F938FECE4
:1095000094E09F938F930E9446930E94B8110FB6E8
:10951000F894DEBF0FBECDBF8091C52C9091C62CB4
:1095200091FF3BC00E94C71D20E030E048EC52E4B0
:10953000162F072FF82EE92E0E94C48D20E836EE54
:1095400045EC57E40E94188B21E03EED42E45EE3D7
:109550000E94318E9B01AC0160E070E080E89FE3E7
:109560000E94348A2BE43AE34DEB57E30E94188BB8
:109570009F938F937F936F93EF92FF920F931F931D
:1095800086EB94E09F938F930E9446930E94B811BC
:109590000FB6F894DEBF0FBECDBF80918002882346
:1095A00009F41CC11F928F9383EB94E09F938F93D8
:1095B0000E9446930F900F900F900F900FC16091F3
:1095C0007E0270917F0280E090E00E94669268E2E5
:1095D00076E00E948792892B99F460917E027091C7
:1095E0007F0280E090E00E946692009709F4F6C046
:1095F0000E94539190915201892B80935201EEC0A9
:10960000809152018F701F928F9387EF92E09F930A
:109610008F930E9446930E94B8110F900F900F9065
:109620000F90DCC060917E0270917F0280E090E03C
:109630000E946692009711F14AE050E060E070E00D
:109640000E94ED8E603198F4609364021F926F93D4
:1096500086EA94E09F938F930E94469341E050E006
:109660006BE170E084E692E00E94119611C0809157
:1096700064021F928F938DE994E006C0809164028A
:109680001F928F9384E994E09F938F930E94469357
:109690000F900F900F900F900E94B8118091800250
:1096A000882309F49BC01F928F9381E994E09F93D4
:1096B0008F930E9446930F900F900F900F908EC043
:1096C00060917E0270917F0280E090E00E9466923D
:1096D0008C0169E175E00E948792892BE1F40E9478
:1096E00039668091660290916702A0916802B091FC
:1096F000690290618093660290936702A09368026A
:10970000B093690244E050E06EE170E086E692E0DA
:109710000E94119663C06CE175E0C8010E948792B7
:10972000892B99F5F8940E9447660FB6F894A8958E
:1097300080916000886180936000109260000FBE8D
:1097400084B7877F84BF80916000886180936000C8
:109750001092600078948091660290916702A091C7
:109760006802B09169029F7E8093660290936702BF
:10977000A0936802B093690244E050E06EE170E0AB
:1097800086E692E00E94119629C06DE276E0C8015B
:109790000E94879240916602509167026091680230
:1097A00070916902892B21F454FF18C0F894FFCFFF
:1097B00054FD03C08CE195E002C089E195E09F93E0
:1097C0008F9383EF92E09F938F930E9446930F9025
:1097D0000F900F900F9002C00E94AE25EA85FB8586
:1097E0001182108283E02B960FB6F894DEBF0FBE75
:1097F000CDBFDF91CF911F910F91FF90EF90DF9040
:10980000CF90BF90AF909F908F907F906F905F9020
:109810004F903F902F900895CF93DF93EC01888174
:109820009981009741F08F3E914109F48CC01982D3
:10983000188283E093C00E9451368091660280FDB9
:1098400005C081FF01C01D9B0E944467809170008C
:109850008C7F809370008091B60080628093B60008
:109860001092B20082E08093B1008091B6008770C0
:10987000E1F78091700081608093700069E57EE07F
:1098800080E090E00E9416660E94CA2680E00E9456
:10989000A8288DEB91E19F938F930E9446930E949D
:1098A0004A168091C52C0F900F9086FD0E94396159
:1098B0008091C52C9091C62C90FD0E949E23809192
:1098C000C52C87FF06C021E04CE061E080ED0E94DE
:1098D000DC6180919C130E94316A809165020E9434
:1098E0000A690E9407698093810A809165020E943B
:1098F0000A6980919C131F928F938091810A1F9215
:109900008F9382E396E09F938F930E9432931092FD
:10991000830A1092820A0F900F900F900F900F9071
:109920000F9086E592E0909398358093973583E287
:1099300090E090939813809397138FEE91E1998321
:10994000888381E00BC06332E1F744EF50E360E0CD
:1099500070E082E89AE00E94C137E3CFDF91CF91B7
:1099600008950F931F93CF93DF93EC018A018881B1
:109970009981009711F18430924121F01982188267
:1099800083E020C06231E9F4A80162E170E082E87E
:109990009AE00E94C13784E080937C3510927E3536
:1099A00010927D351093803500937F354CE755E359
:1099B00062E182E492E00E94E16F84E092E19983A7
:1099C000888381E0DF91CF911F910F9108958436B4
:1099D000910514F19F938F9388E896E09F938F935E
:1099E0000E9432938091CF309091D030A091D130AD
:1099F000B091D2300196A11DB11D8093CF309093CC
:109A0000D030A093D130B093D2300F900F900F9000
:109A10000F9081E090E0089580E090E008952F920B
:109A20003F924F925F926F927F928F929F92AF92EE
:109A3000BF92CF92DF92EF92FF920F931F93CF933B
:109A4000DF93CDB7DEB7CC59D1090FB6F894DEBF9E
:109A50000FBECDBFCB56DF4F99838883C559D04009
:109A60008A01633871F486E89AE0C456DF4F688350
:109A7000CC59D0400E94FB72C456DF4F6881CC594C
:109A8000D040CB56DF4FA881B981C559D0402D9128
:109A90003C912C39B1E13B0711F40C94DC5A40F4B1
:109AA0002115310581F0223C3F4009F43BC42FC40D
:109AB0002E3A41E1340709F409C4253B314111F440
:109AC0000C94E45A24C44AE259E061E870E086E864
:109AD0009AE00E94E07282EC9FE0EFC35A01E3E05B
:109AE000F0E0EC0FFD1FE40FF51F1082CA010E9489
:109AF000E74C892B81F720E030E040E050E0CC5685
:109B0000DF4F6881C459D040627070E080E090E01F
:109B1000A0E00E94288A09F0A0C6212F287030E01A
:109B200040E050E060E070E080E090E0A0E00E9463
:109B3000288A99F127E04AE250E06BE270E089E27E
:109B400090E00E94BF5D8EE895E30E948B5FBC01B0
:109B5000990F880B990B0E94CC8B20E030E048ECE9
:109B600052E40E94188B9F938F937F936F938CEB9B
:109B700096E09F938F931F9287E78F93CE018A0D74
:109B80009B1D03969F938F930E949E93A80EB91ED0
:109B90000FB6F894DEBF0FBECDBF212F207130E08D
:109BA00040E050E060E070E080E090E0A0E00E94E3
:109BB000288AE9F126E04AE250E06BE270E089E2AF
:109BC00090E00E94BF5D81E090E00E945011809380
:109BD0009B1381E09DE10E948B5FBC01990F880B74
:109BE000990B0E94CC8B20E030E048EC52E40E94BC
:109BF000188B9F938F937F936F9386EC96E09F9340
:109C00008F931F9287E78F93C501029621E030E082
:109C10002C0F3D1F820F931F9F938F930E949E9343
:109C2000A80EB91E0FB6F894DEBF0FBECDBFC25747
:109C3000DF4F2881CE58D04030E040E050E060E077
:109C400070E080E090E0A0E00E94288A01F10E948C
:109C50000C119F938F937F936F9381ED96E09F9369
:109C60008F931F9287E78F93C5010296A1E0B0E022
:109C7000AC0FBD1F8A0F9B1F9F938F930E949E93D3
:109C8000A80EB91E0FB6F894DEBF0FBECDBF212FB0
:109C9000207430E040E050E060E070E080E090E070
:109CA000A0E00E94288A31F18091CA308F93809180
:109CB000C9308F938091C8308F938091C7308F9334
:109CC0008FED96E09F938F931F9287E78F93C50147
:109CD000029621E030E02C0F3D1F820F931F9F93CF
:109CE0008F930E949E93A80EB91E0FB6F894DEBF04
:109CF0000FBECDBF212F207830E040E050E060E083
:109D000070E080E090E0A0E00E94288A41F1F894A1
:109D10008091743590917535A0917635B0917735F5
:109D20007894BF93AF939F938F938DEE96E09F931C
:109D30008F931F9287E78F93C5010296A1E0B0E051
:109D4000AC0FBD1F8A0F9B1F9F938F930E949E9302
:109D5000A80EB91E0FB6F894DEBF0FBECDBF20E02F
:109D6000302F317040E050E060E070E080E090E043
:109D7000A0E00E94288A09F082C520E0302F3270CE
:109D800040E050E060E070E080E090E0A0E00E9401
:109D9000288A09F0F2C520E0302F347040E050E00E
:109DA00060E070E080E090E0A0E00E94288A09F086
:109DB00015C620E0302F387040E050E060E070E0E1
:109DC00080E090E0A0E00E94288A09F036C620E0FA
:109DD000302F307140E050E060E070E080E090E0D3
:109DE000A0E00E94288A09F0A6C620E0302F307239
:109DF00040E050E060E070E080E090E0A0E00E9491
:109E0000288A09F0C8C620E030E040E050E0CC5697
:109E1000DF4F6881C459D040647070E080E090E00A
:109E2000A0E00E94288A09F0E4C620E0C856DF4F6F
:109E30003881C859D04040E050E060E070E080E0F8
:109E400090E0A0E00E94288A09F040C720E0C756B1
:109E5000DF4F3881C959D04040E050E060E070E009
:109E600080E090E0A0E00E94288A09F05DC7CE560D
:109E7000DF4F5881C259D0405170952E20E030E01C
:109E8000452F50E060E070E080E090E0A0E00E94AC
:109E9000288A09F077C720E030E0CE56DF4F4881AE
:109EA000C259D040427050E060E070E080E090E045
:109EB000A0E00E94288A09F098C720E030E0C65749
:109EC000DF4F4881CA58D04050E060E070E080E049
:109ED00090E0A0E00E94288A09F0BAC720E030E0B4
:109EE00040E050E0CC56DF4F6881C459D0406870E4
:109EF00070E080E090E0A0E00E94288A09F0D2C7DC
:109F000020E030E040E050E0CC56DF4F6881C4599B
:109F1000D040607170E080E090E0A0E00E94288A6C
:109F200009F0ECC720E030E0CE56DF4F4881C2593F
:109F3000D040487050E060E070E080E090E0A0E049
:109F40000E94288A11F00C94AA5720E030E0CE56E7
:109F5000DF4F4881C259D040407150E060E070E06E
:109F600080E090E0A0E00E94288A11F00C94DD5778
:109F700020E030E0CE56DF4F4881C259D0404072D9
:109F800050E060E070E080E090E0A0E00E94288A6D
:109F900011F00C94105820E030E0CE56DF4F48818D
:109FA000C259D040407450E060E070E080E090E042
:109FB000A0E00E94288A11F00C944358CE56DF4F3F
:109FC000F881C259D040F0787F2E20E030E04F2F4A
:109FD00050E060E070E080E090E0A0E00E94288A1D
:109FE00011F00C947658CD56DF4F2881C359D040DC
:109FF0002170622E20E030E040E0562D60E070E0FD
:10A0000080E090E0A0E00E94288A11F40C94F75AB6
:10A010008091C52C82FD02C00C94BE5821E046E020
:10A0200061E083E00E94621920E030E0472D50E0BB
:10A0300060E070E080E090E0A0E00E94288A11F4E7
:10A040000C94BE588091C52C82FF02C00C9483589A
:10A0500020E030E040E0CD56DF4F5881C359D0407A
:10A06000527060E070E080E090E0A0E00E94288AFA
:10A0700011F00C94F35820E030E040E0CD56DF4F73
:10A080005881C359D040547060E070E080E090E0A7
:10A09000A0E00E94288A11F00C94265920E030E0BC
:10A0A00040E0CD56DF4F5881C359D040507160E039
:10A0B00070E080E090E0A0E00E94288A11F00C940B
:10A0C000595920E030E040E0CD56DF4F5881C35968
:10A0D000D040507260E070E080E090E0A0E00E942C
:10A0E000288A11F00C94985920E030E040E0CD56D9
:10A0F000DF4F5881C359D040507460E070E080E079
:10A1000090E0A0E00E94288A11F00C94D75920E03A
:10A1100030E040E0CD56DF4F5881C359D0405870F1
:10A1200060E070E080E090E0A0E00E94288A11F0FA
:10A130000C94165A20E030E040E0C656DF4F5881BC
:10A14000CA59D04060E070E080E090E0A0E00E945A
:10A15000288A11F00C94475A20E030E0492D50E055
:10A1600060E070E080E090E0A0E00E94288A11F0BA
:10A170000C947E5A212F302FCE56DF4F4881C25982
:10A18000D040CD56DF4F5881C359D040CC56DF4F19
:10A190006881C459D0407D2DC956DF4F8881C75989
:10A1A000D0409C2DA0E00E94288A11F00C94895A7E
:10A1B000809164028061898380917A0A8A83FE019A
:10A1C000EA0DFB1D138280919F139091A013A09123
:10A1D000A113B091A21385010D5F1F4F80FF0CC02A
:10A1E0001F930F938DE898E09F938F930E94329373
:10A1F0000F900F900F900F90B801CE0101960E9422
:10A20000EA748091660282FF0AC024E731E3A80164
:10A21000BE016F5F7F4F8EE692E00E94A960809141
:10A220009F139091A013A091A113B091A21382FD4E
:10A2300073980E940E6886E89AE00E94FD728091F1
:10A24000660290916702A0916802B091690290FD48
:10A2500002C00C94C05A3FEFA31AB30A0E940769C8
:10A26000F82E89E10E941F69809166029091670231
:10A27000A0916802B091690290FD02C00C94BC5A92
:10A28000739880917A0A8F5F80937A0A8A83B501E6
:10A290006F5F7F4FCE0101960E94EA7486E89AE0D4
:10A2A0000E94FD7240E050E065E88091E1149091D9
:10A2B000E2140E94E16F8CE991E1CB56DF4FA88157
:10A2C000B981C559D0408D939C931EC08EE69AE00B
:10A2D0000E946F6E892BC1F00E940E688091660209
:10A2E00087FD2B9840E450E060E070E08EE69AE055
:10A2F0000E94516E85EB91E1CB56DF4FE881F981E9
:10A30000C559D0409183808381E00C94075BCB5684
:10A31000DF4FA881B981C559D0401D921C9283E0BE
:10A320000C94075B623181F780906602909067021F
:10A33000A0906802B090690291FCCDCBF8018081B9
:10A34000813021F50180F281E02D1081018122818F
:10A35000CE56DF4F2883C259D0403381CD56DF4FD0
:10A360003883C359D0404481CC56DF4F4883C45909
:10A37000D040D5805681C956DF4F5883C759D04049
:10A38000C780E084F184212C312C52C08230B9F492
:10A3900023803480E12CF12C11E000E0CE56DF4F19
:10A3A0001882C259D040B0E8CD56DF4FB883C359A8
:10A3B000D040CC56DF4F1882C459D04032C08330D1
:10A3C000D1F0843009F087CBE12CF12C212C312CF9
:10A3D00015E000E0CE56DF4F1882C259D040CD566E
:10A3E000DF4F1882C359D040E2E0CC56DF4FE883FC
:10A3F000C459D04016C0E12CF12C212C312C15E091
:10A4000000E0CE56DF4F1882C259D040CD56DF4F04
:10A410001882C359D040F1E0CC56DF4FF883C459BD
:10A42000D040D12CC956DF4F1882C759D040C12C1B
:10A430004090C7305090C8306090C9307090CA309A
:10A4400020918D0230918E0240918F0250919002A6
:10A45000C657DF4F288339834A835B83CA58D0406D
:10A460002DEC3CEC4CE45EE3C657DF4F688179810C
:10A470008A819B81CA58D0400E94358A9B01AC01D9
:10A48000C301B2010E94F18C87FD0BC0E894A0F8D3
:10A490008092660290926702A0926802B09269026E
:10A4A00046C0C657DF4F288139814A815B81CA582F
:10A4B000D040C301B2010E94138B87FF38C0809146
:10A4C000D3309091D430A091D530B091D630019650
:10A4D000A11DB11D8093D3309093D430A093D5307B
:10A4E000B093D630A0FCF7CA6894A0F880926602B8
:10A4F00090926702A0926802B092690215E400E2AD
:10A50000CE56DF4F1882C259D040CD56DF4F188249
:10A51000C359D04034E0CC56DF4F3883C459D040C3
:10A52000D12CC956DF4F1882C759D040C12CCE5606
:10A53000DF4F4881C259D0404470C657DF4F48832F
:10A54000CA58D04020E030E050E060E070E080E0A9
:10A5500090E0A0E00E94288A09F08C9A512F507256
:10A56000C257DF4F5883CE58D040252F30E040E00F
:10A5700050E060E070E080E090E0A0E00E94288A77
:10A5800011F00E940C11802F8074C856DF4F888311
:10A59000C859D04020E0382F40E050E060E070E043
:10A5A00080E090E0A0E00E94288A11F00E9410252F
:10A5B000902F9078C756DF4F9883C959D04020E03C
:10A5C000392F40E050E060E070E080E090E0A0E0F3
:10A5D0000E94288A51F00E94A710609381357093E1
:10A5E00082358093833590938435212F217030E01C
:10A5F00040E050E060E070E080E090E0A0E00E9489
:10A60000288AF1F08FE89CE19F938F938CE996E084
:10A610009F938F931F9287E78F93CE0103969F930B
:10A620008F930E949E934C010E94E74C0FB6F894C2
:10A63000DEBF0FBECDBF892B09F04DCA540102C049
:10A64000A12CB12C212F227030E040E050E060E0DE
:10A6500070E080E090E0A0E00E94288AD1F1C5017E
:10A66000029664EA76E0E1E0F0E0EC0FFD1F8E0F69
:10A670009F1F0E949092F3E0AF0EB11C2EE8622E55
:10A6800025E3722E36E7832E33E0932E47E7542ED0
:10A69000D3018D913D011F928F939F928F921F92B4
:10A6A0005F92C5010296E1E0F0E0EC0FFD1F8E0F16
:10A6B0009F1F9F938F930E949E93A80EB91E0FB663
:10A6C000F894DEBF0FBECDBF36E9631635E37306DF
:10A6D000F9F6212F247030E040E050E060E070E0B7
:10A6E00080E090E0A0E00E94288A09F450C0C501F3
:10A6F000029668EA76E041E050E04C0F5D1F840F5F
:10A70000951F0E94909254E0A50EB11C2E018AE77D
:10A71000480E511C80E1D2011D928A95E9F728E08C
:10A72000A20168E980EB0E94AD173201B8E06B0E20
:10A73000711C96E7892E93E0992E27E7F20181910B
:10A740002F011F928F939F928F921F922F93C5017B
:10A75000029641E050E04C0F5D1F840F951F9F93C0
:10A760008F93C556DF4F2883CB59D0400E949E93CC
:10A77000A80EB91E0FB6F894DEBF0FBECDBFC556EA
:10A78000DF4F2881CB59D04046145704B9F6CD5637
:10A79000DF4F9881C359D0409078C656DF4F9883D9
:10A7A000CA59D04020E030E040E0592F60E070E02E
:10A7B00080E090E0A0E00E94288AE1F480919D135F
:10A7C00090919E139F938F938DEA96E09F938F9322
:10A7D0001F9287E78F93CE018A0D9B1D03969F934F
:10A7E0008F930E949E93A80EB91E0FB6F894DEBFF9
:10A7F0000FBECDBF20E030E040E050E0CC56DF4F50
:10A800006881C459D040617070E080E090E0A0E0C1
:10A810000E94288A09F46FC9E3E0F0E0EC0FFD1F05
:10A82000EA0DFB1D80E28083A50183E090E08A1998
:10A830009B09FC01E40FF51FEC50FF4C20814F5F9A
:10A840005F4F222309F44AC92081E1E0F0E0EC0FD8
:10A85000FD1FE40FF51F2283ECCFCE018A0D9B1D57
:10A8600064EB76E003960E949092B7E0AB0EB11CC9
:10A87000C5010E94E74C892B09F02DC94EC9E1148E
:10A88000F10409F47ACAF894409074355090753503
:10A89000609076357090773578948091F91C90911E
:10A8A000FA1CA091FB1CB091FC1CA3019201281B77
:10A8B000390B4A0B5B0BCA01B9010E94CA8BC25704
:10A8C000DF4F688379838A839B83CE58D040B7015A
:10A8D00080E090E00E94CA8B9B01AC01C257DF4F21
:10A8E000688179818A819B81CE58D0400E94188BE3
:10A8F0004C019F928F937F936F9388EF96E09F9385
:10A900008F931F9287E78F939E012A0D3B1D2D5F2A
:10A910003F4F3F932F93C456DF4F6883CC59D040AD
:10A92000C556DF4F7883CB59D0400E949E93A80E26
:10A93000B91EC456DF4F6881CC59D040C556DF4F91
:10A940007881CB59D040862F972FA82DB92D809391
:10A95000863590938735A0938835B093893540929A
:10A96000F91C5092FA1C6092FB1C7092FC1C0FB6F2
:10A97000F894DEBF0FBECDBF00CAE114F10409F4A4
:10A980000ACAF8948091D01C9091D11CA091D21C3D
:10A99000B091D31C78949F938F9380916D028F9385
:10A9A00080916C028F9385E097E09F938F931F9225
:10A9B00087E78F93C5010296A1E0B0E0AC0FBD1F01
:10A9C0008A0F9B1F9F938F930E949E93A80EB91E80
:10A9D0000FB6F894DEBF0FBECDBFDDC9F8948091ED
:10A9E000783590917935A0917A35B0917B3578940E
:10A9F000BF93AF939F938F9385E197E09F938F933E
:10AA00001F9287E78F93C501029621E030E02C0F5B
:10AA10003D1F820F931F9F938F930E949E93A80EBA
:10AA2000B91EC5010E94E74C0FB6F894DEBF0FBEF9
:10AA3000CDBF892B09F04FC8BCC9E114F10409F45A
:10AA4000C6C9F894409078355090793560907A3541
:10AA500070907B3578948091FD1C9091FE1CA091A4
:10AA6000FF1CB091001DA3019201281B390B4A0B5A
:10AA70005B0BCA01B9010E94CA8BC257DF4F6883C2
:10AA800079838A839B83CE58D040B70180E090E0E1
:10AA90000E94CA8B9B01AC01C257DF4F688179814C
:10AAA0008A819B81CE58D0400E94188B4C019F9286
:10AAB0008F937F936F9380E297E09F938F931F9282
:10AAC00087E78F939E012A0D3B1D2D5F3F4F3F93DC
:10AAD0002F93C456DF4F6883CC59D040C556DF4F03
:10AAE0007883CB59D0400E949E93A80EB91EC456BD
:10AAF000DF4F6881CC59D040C556DF4F7881CB59A4
:10AB0000D040862F972FA82DB92D80938A3590930A
:10AB10008B35A0938C35B0938D354092FD1C5092AF
:10AB2000FE1C6092FF1C7092001D0FB6F894DEBFF1
:10AB30000FBECDBF4CC9EF2809F457C9F8948091D6
:10AB4000D41C9091D51CA091D61CB091D71C7894A0
:10AB50009F938F9380916B028F9380916A028F9362
:10AB60008DE297E09F938F931F9287E78F93C501A4
:10AB70000296A1E0B0E0AC0FBD1F8A0F9B1F9F9310
:10AB80008F930E949E93A80EB91E0FB6F894DEBF55
:10AB90000FBECDBF2AC98091CB309091CC30A0910F
:10ABA000CD30B091CE30BF93AF939F938F938DE311
:10ABB00097E09F938F931F9287E78F93C50102962B
:10ABC00021E030E02C0F3D1F820F931F9F938F9346
:10ABD0000E949E93A80EB91EC5010E94E74C0FB6B5
:10ABE000F894DEBF0FBECDBF892B11F00C946B4DD6
:10ABF0000AC98091D6308F938091D5308F93809100
:10AC0000D4308F938091D3308F938091D2308F93B3
:10AC10008091D1308F938091D0308F938091CF30BD
:10AC20008F9388E497E09F938F931F9287E7982EE6
:10AC30009F92C5010296A1E0B0E0AC0FBD1F8A0F44
:10AC40009B1F9F938F930E949E93A80EB91EC501D0
:10AC50000E94E74C0FB6F894DEBF0FBECDBF892B24
:10AC600011F00C946B4D8091C52C9091C62C90FFE7
:10AC7000DCC88091DA308F938091D9308F938091A6
:10AC8000D8308F938091D7308F938CE697E09F9345
:10AC90008F931F929F92C501029621E030E02C0F06
:10ACA0003D1F820F931F9F938F930E949E93A80E28
:10ACB000B91EC5010E94E74C0FB6F894DEBF0FBE67
:10ACC000CDBF892B11F00C946B4DAFC88091BC287F
:10ACD0008F938091BB288F938091BA288F93809116
:10ACE000B9288F938EE797E09F938F931F9287E702
:10ACF0008F93C5010296A1E0B0E0AC0FBD1F8A0F93
:10AD00009B1F9F938F930E949E93A80EB91EC5010F
:10AD10000E94E74C0FB6F894DEBF0FBECDBF892B63
:10AD200011F00C946B4D92C8809184358F93809173
:10AD300083358F93809182358F93809181358F9366
:10AD400089E897E09F938F931F9287E78F93C501C0
:10AD5000029621E030E02C0F3D1F820F931F9F933E
:10AD60008F930E949E93A80EB91EC5010E94E74CC6
:10AD70000FB6F894DEBF0FBECDBF892B11F00C9437
:10AD80006B4D75C881E00E94591020918502309169
:10AD9000860240918702509188020E94C48D9F9341
:10ADA0008F937F936F9386E997E09F938F931F9282
:10ADB00087E78F93C5010296A1E0B0E0AC0FBD1FFD
:10ADC0008A0F9B1F9F938F930E949E93A80EB91E7C
:10ADD000C5010E94E74C0FB6F894DEBF0FBECDBF91
:10ADE000892B11F00C946B4D56C882E00E945910CB
:10ADF000209181023091820240918302509184021D
:10AE00000E94C48D9F938F937F936F9383EA97E003
:10AE10009F938F931F9287E78F93C501029621E03E
:10AE200030E02C0F3D1F820F931F9F938F930E9442
:10AE30009E93A80EB91EC5010E94E74C0FB6F89468
:10AE4000DEBF0FBECDBF892B11F00C946B4D35C802
:10AE500083E00E9459109F938F937F936F9380EBB1
:10AE600097E09F938F931F9287E78F93C501029678
:10AE7000A1E0B0E0AC0FBD1F8A0F9B1F9F938F9383
:10AE80000E949E93A80EB91E8C98C5010E94E74CA3
:10AE90000FB6F894DEBF0FBECDBF892B11F00C9416
:10AEA0006B4D1CC8299903C08CE195E002C089E173
:10AEB00095E09F938F938DEB97E09F938F931F92D5
:10AEC00087E78F93C501029621E030E02C0F3D1FEC
:10AED000820F931F9F938F930E949E93A80EB91E7B
:10AEE000C5010E94E74C0FB6F894DEBF0FBECDBF80
:10AEF000892B11F00C946B4D0C94804F2A9903C050
:10AF00008CE195E002C089E195E09F938F9385ECF9
:10AF100097E09F938F931F9287E78F93C5010296C7
:10AF2000A1E0B0E0AC0FBD1F8A0F9B1F9F938F93D2
:10AF30000E949E93A80EB91EC5010E94E74C0FB651
:10AF4000F894DEBF0FBECDBF892B11F00C946B4D72
:10AF50000C94924F8091C52C87FD02C00C94A54F94
:10AF600021E042E161E080ED0E94DC619F938F93DC
:10AF70007F936F938DEC97E09F938F931F9287E75A
:10AF80008F93C501029621E030E02C0F3D1F820F08
:10AF9000931F9F938F930E949E93A80EB91EC50185
:10AFA0000E94E74C0FB6F894DEBF0FBECDBF892BD1
:10AFB00011F00C946B4D0C94A54F8091C52C87FD1E
:10AFC00002C00C94B84F21E042E162E080ED0E94A3
:10AFD000DC619F938F937F936F938BED97E09F93AB
:10AFE0008F931F9287E78F93C5010296A1E0B0E08F
:10AFF000AC0FBD1F8A0F9B1F9F938F930E949E9340
:10B00000A80EB91EC5010E94E74C0FB6F894DEBF2A
:10B010000FBECDBF892B11F00C946B4D0C94B84F23
:10B020008091C52C87FD02C00C94CB4F21E042E1FA
:10B0300063E080ED0E94DC619F938F937F936F9319
:10B0400089EE97E09F938F931F9287E78F93C501B7
:10B05000029621E030E02C0F3D1F820F931F9F933B
:10B060008F930E949E93A80EB91EC5010E94E74CC3
:10B070000FB6F894DEBF0FBECDBF892B11F00C9434
:10B080006B4D0C94CB4F8091C52C87FD02C00C9466
:10B09000DE4F21E042E164E080ED0E94DC619F939D
:10B0A0008F937F936F9387EF97E09F938F931F9278
:10B0B00087E78F93C5010296A1E0B0E0AC0FBD1FFA
:10B0C0008A0F9B1F9F938F930E949E93A80EB91E79
:10B0D000C5010E94E74C0FB6F894DEBF0FBECDBF8E
:10B0E000892B11F00C946B4D0C94DE4F8091C52C84
:10B0F00082FD02C00C94F34F46E061E083E00E94C1
:10B1000062190C94F34F8091A81D8F938091A71D15
:10B110008F938091A61D8F938091A51D8F9385E0BD
:10B1200098E09F938F931F9287E78F93C5010296B4
:10B1300041E050E04C0F5D1F840F951F9F938F934C
:10B140000E949E93A80EB91EC5010E94E74C0FB63F
:10B15000F894DEBF0FBECDBF892B11F00C946B4D60
:10B1600020E030E040E0562D60E070E080E090E0CC
:10B17000A0E00E94288A11F40C9428508091C52CDC
:10B1800082FD02C00C9428508091AC1D8F93809159
:10B19000AB1D8F938091AA1D8F938091A91D8F93D2
:10B1A0008DE098E09F938F931F9287E78F93C5015F
:10B1B0000296E1E0F0E0EC0FFD1F8E0F9F1F9F93C2
:10B1C0008F930E949E93A80EB91EC5010E94E74C62
:10B1D0000FB6F894DEBF0FBECDBF892B11F00C94D3
:10B1E0006B4D0C9428508091C52C9091C62C90FDED
:10B1F00002C00C943B5080E090E00E9488249F9312
:10B200008F937F936F9388E198E09F938F931F9222
:10B2100087E78F93C501029641E050E04C0F5D1F18
:10B22000840F951F9F938F930E949E93A80EB91E23
:10B23000C5010E94E74C0FB6F894DEBF0FBECDBF2C
:10B24000892B11F00C946B4D0C943B508091C52CC4
:10B250009091C62C90FD02C00C944E5081E090E07D
:10B260000E9488249F938F937F936F9388E298E046
:10B270009F938F931F9287E78F93C5010296E1E01A
:10B28000F0E0EC0FFD1F8E0F9F1F9F938F930E9486
:10B290009E93A80EB91EC5010E94E74C0FB6F89404
:10B2A000DEBF0FBECDBF892B11F00C946B4D0C94FB
:10B2B0004E508091C52C9091C62C90FD02C00C94EC
:10B2C000615081E090E00E9488242B013C0180E0E5
:10B2D00090E00E9488249B01AC01C301B2010E944E
:10B2E00085229F938F937F936F9389E398E09F9339
:10B2F0008F931F9287E78F93C501029641E050E03C
:10B300004C0F5D1F840F951F9F938F930E949E93F8
:10B31000A80EB91EC5010E94E74C0FB6F894DEBF17
:10B320000FBECDBF892B11F00C946B4D0C94615066
:10B330008091C52C9091C62C90FD02C00C94745045
:10B3400081E090E00E9488242B013C0180E090E0A5
:10B350000E9488249B01AC01C301B2010E94E62235
:10B360009F938F937F936F9384E498E09F938F9341
:10B370001F9287E78F93C5010296E1E0F0E0EC0FA2
:10B38000FD1F8E0F9F1F9F938F930E949E93A80E69
:10B39000B91EC5010E94E74C0FB6F894DEBF0FBE80
:10B3A000CDBF892B11F00C946B4D0C94745080918F
:10B3B000C52C9091C62C90FD02C00C94875081E062
:10B3C00090E00E9488242B013C0180E090E00E94E4
:10B3D00088249B01AC01C301B2010E9447239F93C3
:10B3E0008F937F936F9382E598E09F938F931F9243
:10B3F00087E78F93C501029641E050E04C0F5D1F37
:10B40000840F951F9F938F930E949E93A80EB91E41
:10B41000C5010E94E74C0FB6F894DEBF0FBECDBF4A
:10B42000892B11F00C946B4D0C9487508091C52C96
:10B430009091C62C91FD02C00C949A500E94C71D99
:10B440009F938F937F936F9385E698E09F938F935D
:10B450001F9287E78F93C5010296E1E0F0E0EC0FC1
:10B46000FD1F8E0F9F1F9F938F930E949E93A80E88
:10B47000B91EC5010E94E74C0FB6F894DEBF0FBE9F
:10B48000CDBF892B11F00C946B4D0C949A50D101C7
:10B4900016968C9116971F928F9315968C911597EF
:10B4A0001F928F9313968C9113971F928F931296DE
:10B4B0008C911F928F9386E798E09F938F931F92B2
:10B4C00087E78F93C5010296E1E0F0E0EC0FFD1FE6
:10B4D0008E0F9F1F9F938F930E949E93A80EB91E5D
:10B4E000C5010E94E74C0FB6F894DEBF0FBECDBF7A
:10B4F000892B11F00C946B4D0C94AC50779A809181
:10B500009F139091A013A091A113B091A21392FD4B
:10B51000749A80919F139091A013A091A113B09160
:10B52000A21382FD0CC08091660280FD08C081FDDF
:10B5300002C00C94D8501D9902C00C94D85040E021
:10B5400050E060E070E0CE0101960E94C40E809150
:10B55000AE1D90E0209195133091961382179307BA
:10B5600010F40C94D85040E050E062E180E192E0A9
:10B570000E94E16F0C94D8508F2D0E941F69739A1E
:10B5800080919D1390919E13892B11F00E94446726
:10B5900080917A0A8F5F80937A0A80919F139091AD
:10B5A000A013A091A113B091A21382FD02C00C942C
:10B5B0006B4D739A0C946B4D653811F00C9484515B
:10B5C000A12CB12C0C9434518EE69AE00E946F6E3F
:10B5D000892B11F40C9484510E9444678091660277
:10B5E00087FD02C00C946B4D2B9A0C946B4D20E0A0
:10B5F00030E0472D50E060E070E080E090E0A0E0B7
:10B600000E94288A11F00C9422500C942850C456A1
:10B61000DF4F0FB6F894DEBF0FBECDBFDF91CF91E5
:10B620001F910F91FF90EF90DF90CF90BF90AF9060
:10B630009F908F907F906F905F904F903F902F9052
:10B6400008950C9493724F925F926F927F929F92A3
:10B65000AF92BF92CF92DF92EF92FF920F931F9320
:10B66000CF93DF93CDB7DEB760970FB6F894DEBF08
:10B670000FBECDBF5B010E940769E82FF0E0EE0F1F
:10B68000FF1FEE53F34E8081918101969183808359
:10B6900080919F139091A013A091A113B091A21338
:10B6A00081FD749840906602509067026090680235
:10B6B000709069020E9446746C01FC018081982F91
:10B6C00092959F70913099F48F7051F48091A61CDF
:10B6D0009091A71C01969093A71C8093A61C3CC137
:10B6E000B50183EA97E30E94FF73892B51F08091A3
:10B6F000A41C9091A51C01969093A51C8093A41C5A
:10B700002BC1D301C2013EE0B695A79597958795C9
:10B710003A95D1F7F82FF1709F2E81E99AE00E94B7
:10B72000BA707C01892B09F44BC0B501C7010296A0
:10B730000E94FF73892B09F43FC0870123E73EE095
:10B7400040E054E660E070E0C7010F960E94EF6CA5
:10B75000F6019181F7018481981321C082858F5F62
:10B7600082878091A21C9091A31C01969093A31CA8
:10B770008093A21C84E00E943675F701208530E09A
:10B780002817390708F078C184E00E943675F70160
:10B790008087F60180818F70F7018187DDC0F70116
:10B7A000128684E00E943675F7018087F601808159
:10B7B0008F70F701818761C1C7010E941B71B1CFF2
:10B7C00088E092E00E9442717C01892B09F4C4C098
:10B7D000B501C70102960E94F873F601818181507C
:10B7E000F701848380E091E0A0E0B0E08387948754
:10B7F000A587B687128684E00E943675F701808798
:10B80000F60180818F70F7018187B70181E99AE0A5
:10B810000E94F570870123E73EE040E054E660E0D7
:10B8200070E0C7010F960E94EF6C11E0F601818174
:10B83000F7018483F60180818F70F701878384E0AC
:10B840000E943675F701858383E00E943675F70103
:10B85000868387818F3009F010E0F6014180F7017F
:10B860008481481A512C612C712C86E0440C551CA3
:10B87000661C771C8A95D1F72385348545855685C6
:10B88000A0ECB0E00E945C88BB27A92F982F872FDF
:10B89000480E591E6A1E7B1E438654866586768630
:10B8A000A501B701C6010E94C40E8091AE1D90E0B3
:10B8B00020919513309196138217930738F040E04A
:10B8C00050E062E180E192E00E94E16F8091951387
:10B8D00090919613029708F44BC08091C52C86FF77
:10B8E0002AC00E942B61C60105960E94F760F601EE
:10B8F00081811F928F93F70186811F928F9385819B
:10B900001F928F938EE998E09F938F931F9280E10F
:10B910008F93CE0101965C019F938F930E949E931B
:10B9200082E00E941161C5010E94F7600FB6F89491
:10B93000DEBF0FBECDBF8091660290916702A091DD
:10B940006802B091690297FD4DC080919513909166
:10B950009613029708F47AC080919F139091A013D8
:10B96000A091A113B091A21381FF89C0749A87C0DE
:10B970008091660290916702A0916802B09169027D
:10B9800096FFABCF992009F4A8CFF6018081982FBC
:10B990009F709230E8F09150807F892B808386E8F9
:10B9A0009AE00E94215B8091A01C9091A11C0196BD
:10B9B0009093A11C8093A01C80919F139091A01341
:10B9C000A091A113B091A21396FF87CF739885CF52
:10B9D0008091A61C9091A71C01969093A71C809320
:10B9E000A61C7BCF8FE89CE120918F1C222309F4B9
:10B9F000ACCF9F938F9381EB98E09F938F93CE0171
:10BA000001963C019F938F930E94DB935C01B301ED
:10BA1000C60102960E94B1920F900F900F900F9066
:10BA20000F900F90009709F490CFEFEFAE1ABE0A77
:10BA30008A0D9B1DAC010196FA0120812032D1F3C1
:10BA400062E18AE192E00E94E16F7FCF112309F465
:10BA500083CF82E08093E0301092E2301092E130A8
:10BA6000F092E430E092E33040EE50E362E182E4B1
:10BA700092E00E94E16F70CF912C10E0D7CE6096DB
:10BA80000FB6F894DEBF0FBECDBFDF91CF911F91EF
:10BA90000F91FF90EF90DF90CF90BF90AF909F906D
:10BAA0007F906F905F904F9008958115910511F0F0
:10BAB0000197F1F70895E091A135F091A2359081B9
:10BAC0008091A03589230895E0919E35F0919F35AE
:10BAD00080819091A035892B8083E091A335F091EE
:10BAE000A43580819091A035892B808308951F9380
:10BAF000CF93DF93E0919E35F0919F3590818091B7
:10BB0000A035809589238083E091A335F091A435F9
:10BB100080819091A035892B80838FE897E00E94E7
:10BB2000555D1FB7F894E091A335F091A43590814D
:10BB30008091A03580958923808389E091E00E94DF
:10BB4000555DE091A135F091A235D081C091A0352D
:10BB50001FBF789485E896E00E94555DE091A1357D
:10BB6000F091A23590818091A035982319F08D2F06
:10BB70008C2301C081E0DF91CF911F9108955093F4
:10BB8000A4354093A33570939F3560939E35909371
:10BB9000A2358093A13581E001C0880F2A95EAF78C
:10BBA0008093A0350C94775DCF93DF93C82FDFB7D8
:10BBB000F894E091A335F091A43580819091A0355F
:10BBC000892B808387E090E00E94555DCC2351F063
:10BBD000E091A335F091A43580819091A0359095A6
:10BBE0009823908384E390E00E94555DE091A13515
:10BBF000F091A23580819091A035892309F4C0E0AD
:10BC000085EB90E00E94555DE091A335F091A4355D
:10BC100080819091A035909598239083DFBF88E72D
:10BC200090E00E94555D8C2FDF91CF910895CF93C6
:10BC3000DF93C82FD8E08C2F81700E94D45DC69509
:10BC40008111C068D150B9F78C2FDF91CF91089541
:10BC50008FEF0C94175EDF92EF92FF920F931F937A
:10BC6000CF93DF93E82EEB010E94775D81112FC007
:10BC700080EF0E94175EF12C10E488EFD82ED10ED1
:10BC800081E00E94D45D082F81E00E94D45D88236A
:10BC900019F0002361F01DC0011109C01E1528F024
:10BCA000888180FF04C0E11611F0F12E01E0802FA1
:10BCB0000E94D45D988196950111906898831150E7
:10BCC0001D11DECF21961111D8CF8F2D03C08FEF1C
:10BCD00001C08EEFDF91CF911F910F91FF90EF90F8
:10BCE000DF900895FF920F931F93CF93DF93F82E69
:10BCF000EB010E94775D209769F085E50E94175E51
:10BD00008E01085F1F4F89910E94175EC017D107EF
:10BD1000D1F703C08CEC0E94175E8F2DDF91CF917D
:10BD20001F910F91FF900C94175E0F931F93CF9369
:10BD3000DF93DB01EC9111969C911197F0E0F92BC8
:10BD4000803181F4BF016E7FE3E0660F771FEA95D3
:10BD5000E1F716969C911697ECE0F0E0E91BF109EB
:10BD6000E60FF71FF7FF07C091E0EA019883F1950E
:10BD7000E195F10902C0EA011882883279F414963B
:10BD80008C91982F9076903649F086FF02C0EE7F16
:10BD900005C085FF02C0EC7F01C0E87FCF0144E011
:10BDA000969587954A95E1F7D9018C93EF70E80154
:10BDB000E88380E0DF91CF911F910F9108950F9359
:10BDC0001F93CF93DF93EC018B01B80188810E9410
:10BDD0002B5E888381508D3F30F4F801808188325A
:10BDE00011F0803191F7DF91CF911F910F9108955C
:10BDF000CF93DF93EC010E94775DBE0184EB0E943C
:10BE0000725E81E00E94D45DC82F0E94775D81E060
:10BE1000C11101C080E0DF91CF9108951F93CF93AE
:10BE2000DF931F921F92CDB7DEB7182F69837A83F5
:10BE30000E94775D0E945B5D69817A81882341F071
:10BE400084E40E94725E113029F00E94645D02C099
:10BE500082E001C080E00F900F90DF91CF911F91A1
:10BE600008954F925F926F927F928F929F92AF92BE
:10BE7000BF92CF92DF92EF92FF920F931F93CF93D7
:10BE8000DF93CDB7DEB729970FB6F894DEBF0FBEAC
:10BE9000CDBF6C015B014A0189010E94775DB6014B
:10BEA0008EEB0E94725ECE0101967C013E019AE00B
:10BEB000690E711C27010E94285EF70181937F01A2
:10BEC000E615F705C1F769E070E0C2010E94D57878
:10BED000811109C09401A501B201F60180810E947F
:10BEE000955E80E001C083E029960FB6F894DEBF2E
:10BEF0000FBECDBFDF91CF911F910F91FF90EF90BB
:10BF0000DF90CF90BF90AF909F908F907F906F9079
:10BF10005F904F900895EF92FF920F931F93CF93EE
:10BF2000DF93CDB7DEB72B970FB6F894DEBF0FBE09
:10BF3000CDBFF82EE92E682F792F88E08F0D0E9453
:10BF40000E5F882319F084E391E243C06CE872E845
:10BF50008EE190E00E94F65F8E01075F1F4F98010F
:10BF6000AE01465F5F4FBE01655F7F4F8F2D9E2DF7
:10BF70000E94315F8111E7CF88E0E1EEF2E0DE015F
:10BF8000119601900D928A95E1F7498521E732E0FB
:10BF9000429FC001439F900D112464E670E00E940F
:10BFA000E1878A8594E6899F600D711D1124FE0149
:10BFB00031968191481303C06F5F7F4F03C0E01734
:10BFC000F107B9F78B85882319F07195619571098F
:10BFD000CB012B960FB6F894DEBF0FBECDBFDF911D
:10BFE000CF911F910F91FF90EF900895DC01CB014D
:10BFF00081159105A105B10529F081509040A0401F
:10C00000B040D9F708959B01AC011092B90060E0EF
:10C0100074E284EF90E00E94F587205131094109D4
:10C02000510956954795379527952093B80008955F
:10C0300094EA9093BC0040EA56E861E070E0909189
:10C04000BC0097FD0BC041505109610971094115B0
:10C0500051056105710599F781E008959091B90046
:10C06000987F983011F09031B9F78093BB0084E845
:10C070008093BC0080EA96E8A1E0B0E02091BC008B
:10C0800027FD08C00197A109B1090097A105B105D5
:10C09000A9F7E2CF8091B900887F883111F0803410
:10C0A000D9F680E0089524EA34E844E92093BC00FE
:10C0B0009091BC0097FFFCCF9091B900987F983089
:10C0C00011F0903199F78093BB003093BC009091B0
:10C0D000BC0097FFFCCF9091B900987F903211F08F
:10C0E000983539F44093BC009091BC0094FDFCCF8E
:10C0F000DDCF08950C94186084E98093BC00809192
:10C10000BC0084FDFCCF08958093BB0084E880933D
:10C11000BC008091BC0087FFFCCF9091B900987F54
:10C1200081E0983209F480E0089584EC8093BC00AB
:10C130008091BC0087FFFCCF8091BB00089584E80C
:10C140008093BC008091BC0087FFFCCF8091BB0036
:10C150000895E0E1DC01FD91CD01F0933F01E15054
:10C16000C9F780913C018F7D80933C0180913C0117
:10C17000877F80933C01FB0180E1919190933E0188
:10C180008150D9F780913C01806880933C01809177
:10C190003D0180FFFCCF4051510980913C018062FC
:10C1A00080933C0180913C01877F80933C01141671
:10C1B00015069CF4FB0180E1919190933E01815022
:10C1C000D9F780913C01806880933C0180913D01CA
:10C1D00080FFFCCF40515109EACFF90180E19091F5
:10C1E0003E0191938150D9F781E090E008950F933B
:10C1F0001F93CF93DF93EC018CE70E9453608CE791
:10C200000E9484608E01005F1F4F89910E948460AC
:10C21000C017D107D1F7DF91CF911F910F910C94E7
:10C220007C60813019F440E050E002C040EC50E006
:10C2300060E070E08CE790E00C949517813019F481
:10C240004EE050E002C048E050E060E070E08CE773
:10C2500090E00C94951741E050E060E070E08CE7CE
:10C2600090E00E94951764ED74E180E090E00C94FA
:10C27000F65F48E350E060E070E08CE790E00E94F9
:10C28000951749E350E060E070E08CE790E00E9491
:10C29000951744E150E060E070E08CE790E00E9488
:10C2A000951748E750E060E070E08CE790E00E946E
:10C2B00095174EE550E060E070E08CE790E00E945A
:10C2C00095174DE650E060E070E08CE790E00E944A
:10C2D000951768E374E38CE090E00E94F65F4CE011
:10C2E00050E060E070E08CE790E00E94951741E03C
:10C2F00050E060E070E08CE790E00E94951746E027
:10C3000050E060E070E08CE790E00E94951764EDEB
:10C3100074E180E090E00C94F65FCF93DF93CDB7AB
:10C32000DEB7A2970FB6F894DEBF0FBECDBF81E196
:10C33000E0E4F9E0DE01529601900D928A95E1F772
:10C3400081E1E1E5F9E0DE01119601900D928A9517
:10C35000E1F70E943961CE0142960E94F76082E0C7
:10C360000E94116164ED74E180E090E00E94F65F4C
:10C37000CE0101960E94F76060E27CE581E590E0E5
:10C380000E94F65F80E00E941E6160E27CE581E52C
:10C3900090E00E94F65F4EE050E060E070E08CE7D5
:10C3A00090E00E949517A2960FB6F894DEBF0FBEDC
:10C3B000CDBFDF91CF910895CF92DF92EF92FF92A0
:10C3C0000F931F93CF93DF9300D0CDB7DEB7F82E36
:10C3D000042F122F213031F0223031F0243031F08F
:10C3E000283031F090E005C091E003C092E001C038
:10C3F00093E00C3059F00E3011F4946007C0003116
:10C4000011F4986003C0023109F49C60613059F066
:10C41000623011F4906207C0633011F4906403C07D
:10C42000643009F490669068692F70E023E030E092
:10C43000AE014F5F5F4F8F2D90E00E94AD1762E11C
:10C4400074E380E090E00E94F65F8F2D8160F82E0B
:10C450000E9418600E94956089830E9495608A837B
:10C46000023119F40E9495608B830E94956087FDCC
:10C47000F1CF0E949F600E947C6062E174E380E0E3
:10C4800090E00E94F65F8F2D0E9418600E949560D8
:10C4900089830E9495608A83023119F40E949F600B
:10C4A0008B830E949F600E947C6039812A810231C7
:10C4B00049F5832F90E0A0E0B0E04B817727662715
:10C4C00031FF0EC030E0322F2227620F731F811D13
:10C4D000911D640F711D811D911D8C6F9F6F0BC08D
:10C4E00030E0322F2227620F731F811D911D640FD0
:10C4F000711D811D911D0E94CC8B20E83FEF4FEFF5
:10C5000057E420C0632F70E0762F6627620F711DFD
:10C51000882777FD8095982F0E94CC8B0C3029F4CA
:10C5200020E030EE4FEF54E40DC00E3029F420E04F
:10C5300038EF4FEF55E406C0003131F420E03EEF14
:10C540004FEF56E40E94188B2FE632E143E050E4AF
:10C550000E94C48D6B017C01612F70E080E090E04F
:10C560000E94CC8B9B01AC01C701B6010E94188BC5
:10C570000F900F900F90DF91CF911F910F91FF902F
:10C58000EF90DF90CF900895CF93E6E4F1E0208123
:10C5900090818081C081C295C695C695C370207C6C
:10C5A000C20F969596959073C90F82958C70C80F9F
:10C5B0001F92CF938AED92E19F938F930E944693AF
:10C5C0000F900F900F900F908C2FCF9108951F9385
:10C5D000CF93DF9346E069E180E00E94CF6580E081
:10C5E0000E9424660E94B26404B600FE08C089EC72
:10C5F00092E19F938F930E9446930F900F9004B601
:10C6000001FE08C088EB92E19F938F930E944693AE
:10C610000F900F9004B602FE08C087EA92E19F9344
:10C620008F930E9446930F900F9004B603FE08C0AC
:10C6300086E992E19F938F930E9446930F900F900B
:10C6400004B604FE08C089E892E19F938F930E948C
:10C6500046930F900F9082E699E09F938F938EE61A
:10C6600092E19F938F930E9446930E943C700E9498
:10C670006D6F60E070E085EB92E00E940F700E94A9
:10C68000E36CE091A609F091A70919950E94C46294
:10C6900090E00E9450660E94107482E08093A3375D
:10C6A0008093A4370E94AA6443EA57E3BC018DEC4F
:10C6B0009BEA0E9424690E941A640E940A690E94EF
:10C6C000AE640E94316A0E944F75E0911C0AF0919D
:10C6D0001D0A1995E091F409F091F5091995E09179
:10C6E000E609F091E70919950E94336A182FC09165
:10C6F000280AD091290AFE0119950F900F900F90EA
:10C700000F90892B49F0FE011995BC0180E890E05B
:10C710000E94CD87EB0102C0C0E8D0E00E9407690B
:10C720001F921F93DF93CF931F928F9380911B0AC9
:10C730008F9380911A0A8F938091F3098F93809140
:10C74000F2098F938CE392E19F938F930E9446931B
:10C750008FE292E19F938F930E9446938EE192E144
:10C760009F938F930E94469360E070E087ED92E084
:10C770000E940F708EE299E00E946E6C86E192E159
:10C780009F938F930E9446938DB79EB742960FB6A4
:10C79000F8949EBF0FBE8DBFDF91CF911F9108957A
:10C7A00080E880936100109261000E94E762C4E01B
:10C7B000D2E103EF11E182EEE82E81E1F82E91ED56
:10C7C000C92E91E1D92E23ECA22E21E1B22E04B67E
:10C7D00000FE06C0DF93CF930E9446930F900F9008
:10C7E00004B601FE06C01F930F930E9446930F905C
:10C7F0000F9004B602FE06C0FF92EF920E9446938D
:10C800000F900F9004B603FE06C0DF92CF920E94F5
:10C8100046930F900F9004B604FE06C0BF92AF92ED
:10C820000E9446930F900F9014BE0E947D6F0E944D
:10C830004566CDCFDF92EF92FF920F931F93CF9378
:10C84000DF93CDB7DEB7A0970FB6F894DEBF0FBE6B
:10C85000CDBF83E690E00E940B96182F282F35EF6E
:10C86000380F303108F0982F9095291709F463C0DC
:10C8700089EE92E19F938F930E944693EEE2F3E15B
:10C880008E010F5F1F4F0F900F90D801D02EE12E19
:10C89000F02E88E0800F94919D9331968A13FBCF00
:10C8A000F89448E050E06FE770E0C8010E941196EC
:10C8B000E0E2F3E1D8018EE08F0D94919D933196E3
:10C8C0008A13FBCF4EE050E061E770E0C8010E94A0
:10C8D0001196E6E1F3E12AE02F0D8491D8018D93C2
:10C8E0008D0131962A13F9CF4AE050E067E670E0F7
:10C8F0008D2D9E2D0E9411966DEC7BEA81E690E0D5
:10C900000E94299660E070E08FE590E00E942996F1
:10C9100060E08EE590E00E941B9660E070E085E6A6
:10C9200090E00E9429961AE16AE175EE83E690E0B4
:10C930000E9429967894812FA0960FB6F894DEBFB6
:10C940000FBECDBFDF91CF911F910F91FF90EF9060
:10C95000DF9008958FE590E00C940B968EE590E0C3
:10C960000C940396F8941092B60016BC89E787BD24
:10C9700082E084BD95E095BD95B395BB80936E0034
:10C98000789408950F931F936091A5137091A61347
:10C990008091A7139091A8130091A5131091A6134D
:10C9A0002091A7133091A81360177107820793078E
:10C9B00059F71F910F9108950F931F936091AD3513
:10C9C0007091AE358091AF359091B0350091AD3515
:10C9D0001091AE352091AF353091B03560177107A9
:10C9E0008207930759F71F910F9108951F920F9295
:10C9F0000FB60F9211240BB60F922F933F934F93C4
:10CA00005F936F937F938F939F93AF93BF93EF93B6
:10CA1000FF938091A5139091A613A091A713B091B5
:10CA2000A8130196A11DB11D8093A5139093A61381
:10CA3000A093A713B093A8138091A4138F5F809342
:10CA4000A41387FF15C01092A4138091AD35909167
:10CA5000AE35A091AF35B091B0350196A11DB11D95
:10CA60008093AD359093AE35A093AF35B093B0358C
:10CA700080914C378823E1F08091A3138F5F8093DE
:10CA8000A31387FF15C01092A3138091A535909131
:10CA9000A635A091A735B091A8350196A11DB11D6D
:10CAA0008093A5359093A635A093A735B093A8356C
:10CAB0000E947A6E892B11F00E949B6DFF91EF917D
:10CAC000BF91AF919F918F917F916F915F914F91A6
:10CAD0003F912F910F900BBE0F900FBE0F901F90A4
:10CAE00018951F920F920FB60F9211240BB60F924A
:10CAF0002F933F934F935F936F937F938F939F9366
:10CB0000AF93BF93EF93FF938091C600E091B3354D
:10CB1000F091B435309709F01995FF91EF91BF91DD
:10CB2000AF919F918F917F916F915F914F913F91C5
:10CB30002F910F900BBE0F900FBE0F901F90189566
:10CB40001F920F920FB60F9211240BB60F922F93D4
:10CB50003F934F935F936F937F938F939F93AF9385
:10CB6000BF93EF93FF938091CE00E091B135F091A8
:10CB7000B235309709F01995FF91EF91BF91AF91C0
:10CB80009F918F917F916F915F914F913F912F91E5
:10CB90000F900BBE0F900FBE0F901F901895811134
:10CBA0000EC01092C5006093C40088E98093C10054
:10CBB0004093C2001092B4351092B335089581307D
:10CBC00069F41092CD006093CC0088E98093C9008D
:10CBD0004093CA001092B2351092B1350895811178
:10CBE00007C08091C00085FFFCCF6093C600089508
:10CBF000813031F48091C80085FFFCCF6093CE0076
:10CC00000895CF93C82F8A3031F46DE08091A91335
:10CC10000E94EF6502C08D3029F06C2F8091A9131E
:10CC20000E94EF6580E090E0CF910895811105C0EA
:10CC30007093B4356093B3350895813021F47093C7
:10CC4000B2356093B13508958093A91383E992E0DA
:10CC50009093F8398093F739089584B7877F84BF1C
:10CC600088E10FB6F89480936000109260000FBEC8
:10CC700008952FE088E190E00FB6F894A89580938E
:10CC800060000FBE209360000895A895089588E184
:10CC90000FB6F89480936000109260000FBE089564
:10CCA0000C94E28E0C94DE8E8091BA3590E008955B
:10CCB0008091390181FF09C0809139018D7F809376
:10CCC000390189E190E00197F1F723E040E06FE15D
:10CCD00082E491E00E948E6B85E090E00197F1F78D
:10CCE00008959091390191FD0AC0282F803108F0F4
:10CCF0002FE040E06FE085E491E00C948E6B0895A6
:10CD00008091390181FD0EC040E06FE181E491E046
:10CD10000E94836B282F2F7E81E090E0213021F04C
:10CD200080E0089580E090E008958091390181FFCE
:10CD300002C081E0089540E06FE181E491E00E944B
:10CD4000836B8F3121F08F7E8150823090F780E0AD
:10CD500008958091390181FD04C00E949566882361
:10CD6000C1F3089510924C378091390181FD8BC039
:10CD70000E94A9668091390181FD85C00E94586694
:10CD800080913901826080933901809184378823B2
:10CD9000D9F18091940090919500409195375091F0
:10CDA000963784179507A0F4809161379091623788
:10CDB000A0916337B0916437875F924CAF4FBF4FFC
:10CDC0008093613790936237A0936337B093643751
:10CDD0002091940030919500241B350B8091613790
:10CDE00090916237A0916337B0916437820F931F9F
:10CDF000A11DB11D8093613790936237A093633773
:10CE0000B093643710928437809186378823D9F1A4
:10CE100080919400909195004091993750919A3764
:10CE200084179507A0F48091693790916A37A09193
:10CE30006B37B0916C37875F924CAF4FBF4F809389
:10CE4000693790936A37A0936B37B0936C37209112
:10CE5000940030919500241B350B80916937909197
:10CE60006A37A0916B37B0916C37820F931FA11D69
:10CE7000B11D8093693790936A37A0936B37B09355
:10CE80006C3710928637089580914C37882321F0B3
:10CE90000E9495660E94B26680E090E0089522E0CC
:10CEA000260F27FF0CC080914A3790914B3701968F
:10CEB00090934B3780934A378FEF9FEF0895AB01E4
:10CEC000BC018AEA93E10E94779280E090E00895A5
:10CED00040E06FE181E491E00C94836B282F40E007
:10CEE0006FEF86E591E00E948E6B0895CF93DF93FC
:10CEF00098EF980F923038F0982F9F7E963019F067
:10CF0000893109F049C09091390191FD48C0C82F7D
:10CF10000E94A9660E946867D82FC81709F442C00A
:10CF2000C83029F4809139010E94586627C0C93160
:10CF300019F4863181F404C0C63169F4893159F499
:10CF400029E040E06FE182E491E00E948E6B85E091
:10CF500090E00197F1F72C2F40E06FE182E491E03F
:10CF60000E948E6BD83031F48FEF0E946E6781ED96
:10CF700092E002C085E090E00197F1F70E946867B7
:10CF80008C1781F0C63019F4813079F40BC0C631AA
:10CF900061F4813151F406C082E490E008C084E479
:10CFA00090E005C080E490E002C083E490E0DF916F
:10CFB000CF910895809194009091950090939A3725
:10CFC0008093993781E08093863780934C37909196
:10CFD000390191FF1EC0209194003091950030934B
:10CFE00096372093953780938437809347372FB7B0
:10CFF000789480913901809139018D7F8093390136
:10D0000080E197E230914737332311F00197D1F750
:10D010002FBF86E10E9476670C94A96680914C37F9
:10D02000811102C00E94DA6781E090E008950F93B9
:10D030001F93CF93DF931F92CDB7DEB780914C370C
:10D04000882361F08091390181FF02C080E07BC0BC
:10D050000E9495668823D1F300E003C00E940E6809
:10D0600001E0809194009091950090939437809383
:10D07000933711E01093833780E88093550186E061
:10D080000E9476671093BB358FB78983789410928E
:10D0900047018091BB358111FCCF89818FBF809181
:10D0A000470111E08E3008F010E0119586E10E94F2
:10D0B000766710925501809183378823D9F180914A
:10D0C0009400909195004091933750919437841734
:10D0D0009507A0F480915D3790915E37A0915F37FE
:10D0E000B0916037875F924CAF4FBF4F80935D37F1
:10D0F00090935E37A0935F37B09360372091940090
:10D1000030919500241B350B80915D3790915E37EF
:10D11000A0915F37B0916037820F931FA11DB11DA1
:10D1200080935D3790935E37A0935F37B0936037FD
:10D130001092833701110E944467812F8295869552
:10D1400086958370817090E00F90DF91CF911F9151
:10D150000F9108958FEF80934E0121E044E060EF3E
:10D160008CE691E00E948E6B25E041E06EE08CE65B
:10D1700091E00E948E6B80E880936F018091460160
:10D1800080936D0121E045E060E284E491E00C943D
:10D190008E6BCF93DF93C9EFD7E0CE010197F1F704
:10D1A0000E94826B1092C135109243361092C536A0
:10D1B0001092C0351092BF35E9E3F1E080818E7F97
:10D1C000808380818D7F808381EC93E00197F1F7EC
:10D1D00080818160808323E040E06FE182E491E020
:10D1E0000E948E6B2197F1F780915D0180915E0125
:10D1F0000E94AA6860E070E081EA92E00E940F70ED
:10D200000E94DA6781E090E0DF91CF9108958091EC
:10D210002B140895CF93DF931F92CDB7DEB7898388
:10D220000E94A966898180932B14282F40E06FE12A
:10D2300088E491E00F90DF91CF910C948E6B0E9467
:10D240000A6986E00C947667EF92FF920F931F9322
:10D25000CF93DF931F921F92CDB7DEB78C017A0177
:10D260007F936F931F938F938CE799E09F938F9396
:10D2700069837A830E943293009362011093630161
:10D280006981609360017A81709361010F900F90C2
:10D290000F900F900F900F90E114F104C9F0F70177
:10D2A000808180936B01818180936A018281809368
:10D2B00069018381809368018481809367018581FE
:10D2C00080936601868180936501878180936401E4
:10D2D0000F900F90DF91CF911F910F91FF90EF90E2
:10D2E000089581EA92E00E94307081E08093BA351F
:10D2F0008091BC359091BD3501969093BD3580935A
:10D30000BC3581E090E008950F931F93CF93209157
:10D31000C035C2E8C29F90011124F901EF53FA4CC5
:10D320004081442309F451C047FD09C0433038F01F
:10D3300050E08A01025011096017710710F4108241
:10D3400044C0B9016E537A4C0E9477928091C035E7
:10D35000C89FF0011124EF53FA4CDF01A058BF4FD2
:10D360009C919093B53510828F5F833018F4809331
:10D37000C03502C01092C035E091C03582E8E89F08
:10D38000F0011124EF53FA4C8081882319F00E9498
:10D39000716902C01092BA35809147018093B63509
:10D3A0009091B935992311F0891710F48093B9350C
:10D3B0006091B63570E084E00E942B756091B535C0
:10D3C00070E083E00E942B7502C000E010E0C8010D
:10D3D000CF911F910F9108950F931F93CF93DF93D8
:10D3E0001F92CDB7DEB78C01FC018081918100973F
:10D3F00009F18334954029F0F8011182108283E00D
:10D400002AC06238E1F40E94D7748FB78983F894F8
:10D410000E94467460E870E00E94846929812FBFF1
:10D420001816190674F40E944174E091220AF091D2
:10D43000230A199583E495E0F8019183808381E0C4
:10D440000AC08091B7359091B83501969093B83560
:10D450008093B735EFCF0F90DF91CF911F910F9150
:10D4600008950C9471668091390181FD06C040E0F9
:10D470006FE085E491E00C94836B80E10895EF9276
:10D48000FF921F93CF93DF931F92CDB7DEB7182F74
:10D490008091390181FD07C00E94A96680914C37B7
:10D4A00081111CC05AC08091940090919500909376
:10D4B00096378093953781E0809384378093473700
:10D4C000809139018D7F8093390180E197E220912D
:10D4D0004737222309F30197D1F7DECF80918637B2
:10D4E0008823D9F1809194009091950040919937CB
:10D4F00050919A3784179507A0F4809169379091DD
:10D500006A37A0916B37B0916C37875F924CAF4F01
:10D51000BF4F8093693790936A37A0936B37B0936E
:10D520006C372091940030919500241B350B80912D
:10D53000693790916A37A0916B37B0916C37820F41
:10D54000931FA11DB11D8093693790936A37A093F3
:10D550006B37B0936C371092863789E10E947667FB
:10D5600086E00E943675892B51F00E94336AE82EBE
:10D5700086E00E94367581500E94716602C0E12CDF
:10D58000F12C80919400909195009093983780931E
:10D59000973781E0809385378FB78983F89480919E
:10D5A0003901826080933901809139018D7F8093A8
:10D5B000390162E0610F8AEA93E10E94D56B8981AB
:10D5C0008FBF8091483790914937019690934937A2
:10D5D000809348370E94A96645E060EE82E491E0BE
:10D5E0000E94836B182F86E00E943675892B19F0F4
:10D5F0008E2D0E947166809185378823D9F18091A4
:10D6000094009091950040919737509198378417E6
:10D610009507A0F48091653790916637A0916737A0
:10D62000B0916837875F924CAF4FBF4F809365379B
:10D6300090936637A0936737B09368372091940032
:10D6400030919500241B350B80916537909166379A
:10D65000A0916737B0916837820F931FA11DB11D4C
:10D660008093653790936637A0936737B093683798
:10D670001092853780914C37882371F08091940007
:10D680009091950090939A378093993781E0809399
:10D6900086370E94DA6702C00E94B266123028F410
:10D6A0008CE00E94367510E00BC0133031F015305D
:10D6B00031F0173029F411E003C012E001C013E08B
:10D6C000812F90E00F90DF91CF911F91FF90EF900D
:10D6D0000895CF93DF93EB010E944F67009729F4E1
:10D6E000CE010E943F6A009751F020914A37309155
:10D6F0004B372F5F3F4F30934B3720934A37DF91A3
:10D70000CF9108950895FC0180816823862F90E0D1
:10D7100002C0959587954A95E2F70895CF93DF93D8
:10D720001F92CDB7DEB7FC01922F8FB78983F89493
:10D730002081362F3095522F5323292F01C0220FDD
:10D740004A95EAF72623252B208389818FBF0F90E6
:10D75000DF91CF910895CF93DF93E0917B012DEF7F
:10D760002E0F2D3740F0FC011082E058FF4F108241
:10D770003196108217C0EC01E993A0E8B1E020E8EF
:10D780002E0F3C91399311962A13FBCFE150F0E014
:10D79000E058FE4F2181FC01E058FF4F2083319675
:10D7A00081E08083DF91CF91089560938001E1E86B
:10D7B000F1E06158DC012D91CD01208331966E138B
:10D7C000F9CF08951F920F920FB60F9211240BB646
:10D7D0000F922F933F934F935F936F937F938F930A
:10D7E0009F93AF93BF93EF93FF93809147018093F3
:10D7F000B6358091BF3522E8829FC00111248F5336
:10D800009A4C0E94AB6B8091BF358F5F833018F4C8
:10D810008093BF3502C01092BF350E947169FF919D
:10D82000EF91BF91AF919F918F917F916F915F9198
:10D830004F913F912F910F900BBE0F900FBE0F9005
:10D840001F9018951F920F920FB60F9211240F90F0
:10D850000FBE0F901F9018951F920F920FB60F9248
:10D8600011240F900FBE0F901F9018951F920F92CA
:10D870000FB60F9211240F900FBE0F901F901895A6
:10D880001F920F920FB60F921124109247370F90EC
:10D890000FBE0F901F9018951F920F920FB60F9208
:10D8A00011241092BE350F900FBE0F901F90189547
:10D8B0001F920F920FB60F9211240F900FBE0F9070
:10D8C0001F9018951F920F920FB60F92112410926D
:10D8D000BB350F900FBE0F901F901895CF93DF931D
:10D8E000EC0189919991009729F060E070E00E9425
:10D8F0000F70F7CFDF91CF910895EF92FF920F93C2
:10D900001F93CF93DF938C017A01FC018081918179
:10D91000009741F08A34910511F1F80111821082CB
:10D9200083E04AC08DE294E10E94BA70EC01209736
:10D9300061F04E815F8168857985CE0102960E94F3
:10D94000516E0990D881C02DF2CF81E080932C14C4
:10D950008AE490E0F8019183808381E02DC06838EB
:10D96000E1F78DE294E10E94BA70EC01209781F317
:10D97000CE010296E816F906D9F4BE018DE294E1D3
:10D980000E94DA70E090E114F090E2148E859F8599
:10D990009093E2148093E114E889F989309719F0A3
:10D9A0008A899B891995F092E214E092E114D0CF14
:10D9B0000990D881C02DDACFDF91CF911F910F91BF
:10D9C000FF90EF90089510922C148DE294E10E9444
:10D9D000B67060E070E08BEA92E00C940F70EF920A
:10D9E000FF920F931F93CF93DF93EC01E090E1142C
:10D9F000F090E214FF86EE86398B288B1B8B0A8B06
:10DA000080912C14882379F08BEA92E09093E214B1
:10DA10008093E114CE0102960E94516EF092E214BE
:10DA2000E092E11404C04E835F8368877987BE016A
:10DA30008DE294E10E94DA70BE018DE294E1DF9103
:10DA4000CF911F910F91FF90EF900C94F570CF93B1
:10DA5000DF93EC0180912C14882329F0CE010296EB
:10DA60000E94856E04C01B861A861D861C86BE0118
:10DA70008DE294E1DF91CF910C94DA70CF92DF9236
:10DA8000EF92FF920F931F9380913314909134146F
:10DA9000892B49F410922F141092301410923114E3
:10DAA0001092321441C00E94C2648B019C01E0912B
:10DAB0003314F091341444815581668177818081DB
:10DAC0009181A281B381840F951FA61FB71F801B70
:10DAD000910BA20BB30B0084F185E02D3097C1F0C0
:10DAE000C480D580E680F780408151816281738156
:10DAF0004C0D5D1D6E1D7F1D401B510B620B730B8A
:10DB0000481759076A077B0730F7DB01CA01E3CFE3
:10DB1000800F911FA21FB31F80932F149093301476
:10DB2000A0933114B09332141F910F91FF90EF9096
:10DB3000DF90CF90089585EB92E00C943070EF92D7
:10DB4000FF920F931F93CF93DF938C01FC01808191
:10DB50009181009799F089359105D9F0F8011182EA
:10DB6000108283E068C0828593858417950709F049
:10DB700049C00084F185E02D3097A9F71092341444
:10DB80001092331489E590E0F8019183808381E05D
:10DB900052C0673891F16238A9F7C0913314D0911F
:10DBA0003414E12CF12C209769F3CE010E948B7084
:10DBB000892BF1F0AE0168E88A859B850E94E16FB0
:10DBC000892BA1F41B861A8688859985E114F104B6
:10DBD00021F0F7019187808704C0909334148093DB
:10DBE0003314198618860E943E6DD7CF0E949B6D14
:10DBF0007E010884D985C02DD6CFE0913314F091F1
:10DC00003414BACFF0933414E0933314A085B18563
:10DC1000109709F4B7CF1A968D919C911B97841792
:10DC2000950739F418968D919C9119979187808763
:10DC3000EDCFFD01EBCFDF91CF911F910F91FF90C1
:10DC4000EF900895CF93DF93EC010E949B6D2A859E
:10DC50003B859091331480913414232B91F0E92F5C
:10DC6000F82F309771F0EC17FD0739F48091E1142B
:10DC70009091E2149387828710C00084F185E02D93
:10DC8000F0CF2091E1143091E2143B872A879887E6
:10DC90008987D0933414C0933314DF91CF910C94BF
:10DCA0003E6DCF93DF93EC010E945D70CE01DF915A
:10DCB000CF910C94226ECF93DF93EC010E946D7094
:10DCC000CE01DF91CF910C94226ECF93DF93EC01C4
:10DCD0000E947F70CE01DF91CF910C94226E21E0E3
:10DCE00030E0FC0182859385892B11F020E030E043
:10DCF000C901089581E090E02091331430913414EB
:10DD0000232B11F480E090E00895CF93DF93EC0192
:10DD1000E0913314F09134148E179F0769F48885CD
:10DD2000998590933414809333140DC08085918528
:10DD30008C179D0721F0FC013097C1F706C088853C
:10DD40009985918780870E943E6D198618861B866B
:10DD50001A86DF91CF9108951F93CF93DF93DC0153
:10DD60001496ED91FC9115973097E1F0162FEC0188
:10DD70009093E2148093E11482E08887CD010696A7
:10DD80001995082E000C990B0297029710F0133882
:10DD900039F4BE01CE01DF91CF911F910C94DC6E5E
:10DDA00081E08887DF91CF911F910895FC01208544
:10DDB00020FD0C94AC6E0895CF92DF92EF92FF920B
:10DDC0000F931F93CF93DF93E090E114F090E21450
:10DDD000C090E314D090E414F601E817F90739F085
:10DDE000309709F44BC00190F081E02DF6CF0097F9
:10DDF00009F444C08B01EC018885882309F1188659
:10DE0000C114D10461F0CC15DD0529F0AE0167E83D
:10DE1000C6010E94D66EF601C080D180F1CFEC81A0
:10DE2000FD81309769F0C017D10751F0D093E2140B
:10DE3000C093E11440E050E063E8CE0106961995E6
:10DE4000E091E314F091E414CE17DF0741F48881E8
:10DE500099819093E4148093E3140CC0FC013097F3
:10DE600049F0808191818C179D07C1F78881998144
:10DE700091838083F092E214E092E114DF91CF91DC
:10DE80001F910F91FF90EF90DF90CF9008951F9317
:10DE9000CF93DF9310923D14C091E314D091E4141A
:10DEA00011E0209779F08985882341F01887198639
:10DEB00040E050E062E8CE010E94AC6E0990D8814B
:10DEC000C02DEFCFDF91CF911F9108958091E01485
:10DED00091E0980F9093E01408958AE88093E014FD
:10DEE0001092DE141092DF141092E4141092E314D6
:10DEF0001092E2141092E114089580913D14811162
:10DF00000E94476F5091DF14552309F452C0E091ED
:10DF1000DE142E2F30E085E0E89FF0011124E25C52
:10DF2000FB4E608160933C14A181B281B0933B149D
:10DF3000A0933A1483819481909339148093381478
:10DF40002F5F3F4F2F7133272093DE145150509392
:10DF5000DF14009731F58091E3149091E4149093CD
:10DF60003714809336148091361490913714892B8E
:10DF700001F180913D1481110E94476F40913A1444
:10DF800050913B1460913C14809136149091371459
:10DF90000E94D66EE0913614F09137148081918101
:10DFA000DECF613819F421E0FC012087AD010E9429
:10DFB000D66E80913D142091DF1490E0820F911D68
:10DFC00008959C019091DF149032B9F0E091DE1435
:10DFD000E90FEF71E093351485E0E89FF00111241B
:10DFE000E25CFB4E608352834183348323839F5FD3
:10DFF0009093DF1480E090E0089581E090E0089530
:10E00000CF93DF93C091E114D091E2140E94D66EB9
:10E01000D093E214C093E114DF91CF910895AB0146
:10E020003091E3142091E414E32FF22FE817F9075D
:10E03000B1F0309721F00190F081E02DF7CF0097FB
:10E0400071F0FC01308321839093E4148093E314F6
:10E0500021E020871782168261E80C9400700895F1
:10E06000009749F0FC0120852150223020F421E066
:10E07000218720933D1408950C9465798091E514CF
:10E080009091E6140097C1F01092E6141092E514F6
:10E09000DC0114966D917C9115971296ED91FC918F
:10E0A00013971995E091E514F091E614309721F05B
:10E0B000808191810C947F790895CF93DF93EC0157
:10E0C0004C835D836E837F830E94C26468837983FF
:10E0D0008A839B83DF91CF910895FC014081518118
:10E0E0006281738184819581A681B781840F951F98
:10E0F000A61FB71F80839183A283B3830895CF9314
:10E10000DF93EC010E94C264688379838A839B83D6
:10E11000DF91CF910895CF92DF92EF92FF92CF934C
:10E12000DF93EC010E94C264C880D980EA80FB8042
:10E13000DC01CB018C199D09AE09BF090196A11D17
:10E14000B11D21E030E0CC80DD80EE80FF80C8167C
:10E15000D906EA06FB0610F020E030E0C901DF91A5
:10E16000CF91FF90EF90DF90CF900895FC01118246
:10E1700010820895FC01808191810895DC01ED9168
:10E18000FC91309731F080819181009729F0FC015A
:10E19000FACF80E090E00895CF010895DC01ED9181
:10E1A000FC911197309721F0208131812D933C9380
:10E1B000CF010895DC01ED91FC913097A9F0A0E02A
:10E1C000B0E020813181E617F70741F4109709F498
:10E1D000DC012D933C9311821082089521153105A5
:10E1E00019F0DF01F901EDCF08950F931F93CF933D
:10E1F000DF938C01EB010E94DA7019821882C8014A
:10E200000E94BE70009711F4F80101C0FC01D18397
:10E21000C083DF91CF911F910F910895DC01ED91A3
:10E22000FC9180E090E0309729F001960190F08118
:10E23000E02DF9CF0895009721F0FC0180819181B4
:10E24000089580E090E00895CF93DF93EC014A8138
:10E250005B8160E070E08C819D810E9480922A81C8
:10E260003B8188819981289FA001299F500D389F6B
:10E27000500D112460E070E08E819F81DF91CF917D
:10E280000C948092FC018281938120E030E0281779
:10E290003907D1F0A481B581A20FB31F4C91411170
:10E2A00010C081E08C9380819181289FA001299FDB
:10E2B000500D389F500D112486819781840F951F32
:10E2C00008952F5F3F4FE3CF80E090E00895FC0179
:10E2D000868197814281538120E030E02417350701
:10E2E000D1F08617970781F4A481B581A20FB31FDF
:10E2F0008C91181614F481508C9384819581FC01C3
:10E30000E20FF31F80810895A081B1818A0F9B1FC6
:10E310002F5F3F4FE3CF8FEF0895FC0126813781B8
:10E3200062177307A0F0A081B18142815381A49F3D
:10E33000C001A59F900DB49F900D1124280F391F87
:10E3400081E090E06217730720F080E0089580E09C
:10E3500090E008952F923F924F925F926F927F923A
:10E360008F929F92AF92BF92CF92DF92EF92FF92E5
:10E370000F931F93CF93DF93CDB7DEB768970FB698
:10E38000F894DEBF0FBECDBFEDE4F7E324A535A5BD
:10E3900046A557A550A441A432A423A4948C858CEF
:10E3A000768C678C808D8983918D9A83828D8B8307
:10E3B000938D9C8384898D8395899E8386898F83A1
:10E3C000978998878089898791899A8782898B879D
:10E3D00093899C8784858D8795859E8786858F8781
:10E3E0009785988B8085898B91859A8BB284A3843D
:10E3F000F480E580D680C78080818F8B9181988F53
:10E40000128103812B8B3C8B4D8B5E8B0E94DC64D5
:10E410005E895F934D894F933C893F932B892F935E
:10E420002F923F924F925F926F927F928F929F9224
:10E430002C812F932B812F932A812F9329812F9326
:10E4400028852F932F812F932E812F932D812F930A
:10E450002C852F932B852F932A852F9329852F93F6
:10E4600028892F932F852F932E852F932D852F93DA
:10E47000AF92BF922A892F9329892F93CF92DF924F
:10E48000EF92FF920F931F93288D2F932F892F9335
:10E490009F938F937F936F93E3EAF7E381811F92BA
:10E4A0008F9380811F928F9386E393E19F938F9345
:10E4B0000E9446930FB6F894DEBF0FBECDBF68969C
:10E4C0000FB6F894DEBF0FBECDBFDF91CF911F9185
:10E4D0000F91FF90EF90DF90CF90BF90AF909F9003
:10E4E0008F907F906F905F904F903F902F90089506
:10E4F000EF92FF920F931F93CF93DF938C01EB0169
:10E500007A010E940E73F801F086E78265ED79E0EA
:10E51000CE01DF91CF911F910F91FF90EF900C945E
:10E5200032730C9416730C94CA73DC011796ED9138
:10E53000FC9118970190F081E02D309709F0199423
:10E540000895DC011796ED91FC9118970280F381F4
:10E55000E02D309709F019940895DC011996ED919A
:10E56000FC911A970280F381E02D309709F01994FD
:10E5700008950F931F93CF93DF931F921F92CDB7F0
:10E58000DEB78C0188E10E944975BC01CE0101967D
:10E590000E94F873D8011996ED91FC911A97019099
:10E5A000F081E02D309729F0BE016F5F7F4FC801E9
:10E5B00019950F900F90DF91CF911F910F910895B2
:10E5C000EF92FF920F931F93CF93DF938C01EB0198
:10E5D0007A0147ED59E00E947872F801F286E186EF
:10E5E0006BED79E0CE01DF91CF911F910F91FF90FC
:10E5F000EF900C9432730C949172CF93DF93EC01F3
:10E6000063EA77E388E10E943F75CE01DF91CF9105
:10E610000C94937287EE94E10C94B670FC017383B2
:10E620006283BC0187EE94E10C94F570BC0187EE27
:10E6300094E10C94DA70CF93DF93EC0187EE94E1D0
:10E640000E94BA70009749F0FC01228133812C1797
:10E650003D0729F00E941B71F5CF80E090E0DF912B
:10E66000CF9108950F931F93CF93DF938B010E9457
:10E670001B73EC01892B31F01D830C83C8010E94B0
:10E6800032838E83DF91CF911F910F910895CF92A6
:10E69000DF92EF92FF920F931F93CF93DF937C0152
:10E6A0008B016A0189EE94E10E94BA70EC01892B1A
:10E6B00051F0EC81FD81309711F0C8011995CE0120
:10E6C0000E941B71F3CFA601B801C701DF91CF9162
:10E6D0001F910F91FF90EF90DF90CF900C94A1725B
:10E6E0000F931F93CF93DF931F921F92CDB7DEB787
:10E6F0000E9404838C0189EE94E10E94BA70009715
:10E7000079F0DC011296ED91FC911397309729F086
:10E7100089839A8319959A8189810E941B71EFCF11
:10E720000115110549F0C8010F900F90DF91CF91AD
:10E730001F910F910C9495720F900F90DF91CF91D4
:10E740001F910F910895CF92DF92EF92FF920F9356
:10E750001F930E944F750E94D7740E9499810E9456
:10E760000283C12C88E0D82E87E0E82EF12C00E04F
:10E770001EE120E030E040E052E060E070E082E046
:10E7800090E00E94C9821F910F91FF90EF90DF905F
:10E79000CF900895CF93DF93EC010E9417830097E9
:10E7A00061F00E945F74E091F609F091F709BE01F3
:10E7B00087E493E7199581E090E0DF91CF91089588
:10E7C000E0911E0AF0911F0A1994E091E809F09176
:10E7D000E9091994E091240AF091250A1994E0912D
:10E7E000260AF091270A199480E090E00895089590
:10E7F000FB0120813181FC0131832083089542E0B7
:10E8000050E00E946A9221E030E0892B11F020E074
:10E8100030E0C9010895BC0183EA97E30C94F873D2
:10E82000E091A609F091A7091995E0911C0AF091D1
:10E830001D0A1995E091F409F091F5091995E091F7
:10E84000E609F091E70919942091A2153091A315DA
:10E850002817390798F04091A0155091A115480F3D
:10E86000591F5093A1154093A015281B390B3093C5
:10E87000A3152093A21581E090E0089580E090E038
:10E8800008959093A3158093A21508958091A015E3
:10E890009091A115835E9A4E089580919F1590E006
:10E8A00083519B4E089581E090E02091EB143091CC
:10E8B000EC142D51354111F480E090E008950E9450
:10E8C0005374892B61F06091EB147091EC144091BA
:10E8D000A2155091A3158DE195E10C9477922091AA
:10E8E000A0153091A11521153105B9F08091A2151F
:10E8F0009091A315C096EDE1F5E1AF014D5E544155
:10E900004817590734F4DF01A20FB31F4C9141930C
:10E91000F4CF1092A1151092A01508958091A21520
:10E920009091A315089580919F1590E3981B2091D5
:10E93000A2153091A315A901490F511DCA010895CF
:10E940000F931F93CF938C01C0919F158C2F90E054
:10E95000801791076CF00E949374800F911F81388B
:10E96000910530F4C01BC0939F1581E090E002C078
:10E9700080E090E0CF911F910F910895CF93DF93A6
:10E98000EDEAF7E31192119287E3ED3DF807D1F735
:10E99000C5EAD7E360E07AE0CE010E94F8732296E0
:10E9A00087E3CD3AD807B1F7DF91CF910895109260
:10E9B000A1151092A0151092A3151092A21580E334
:10E9C00080939F158DE195E19093EC148093EB1467
:10E9D0000C94BE74EF92FF920F931F93CF93DF932B
:10E9E0001F921F92CDB7DEB78C0169837A830E9494
:10E9F000D7746981E62E7A81F72E81E8E816F10452
:10EA000018F080E8E82EF12CA701B8018091EB14F2
:10EA10009091EC140E947792F092A315E092A215C7
:10EA2000C7010F900F90DF91CF911F910F91FF9031
:10EA3000EF900895FC0190E3ADEAB7E301900D92E9
:10EA40009A95E1F788E0FB01A5EAB7E301900D9202
:10EA50008A95E1F70895E82FF0E0EE0FFF1FE355E8
:10EA6000F84C7183608381E090E00895E82FF0E036
:10EA7000EE0FFF1FE355F84C80819181089590E0DF
:10EA8000880F991F8B58984C0E94F87381E090E092
:10EA9000089590E0880F991F8B58984C08958FEB3C
:10EAA00092E00E9424718FEC92E00E94247187EC26
:10EAB00092E00C9424710F931F93CF93DF93EC019A
:10EAC000BC018FEC92E00E948D71892BA9F0099016
:10EAD000D881C02DFE0161917191CF010E94EA742D
:10EAE000BE016E547F4FCE018E579F4FDF91CF9165
:10EAF0001F910F910C941A75BE0187EC92E00E9451
:10EB00008D71892BD1F00E94D774688179818A81B7
:10EB10009B810E94EA748CA990E00E94A0740CA9C9
:10EB200010E00E944D74BE016C5F7F4FA801DF9121
:10EB3000CF911F910F910C947792DF91CF911F91FC
:10EB40000F91089587E19CE10E946F6E892B21F05F
:10EB500087E19CE10C94656E0895E091031CF091AF
:10EB6000041C309709F0199480E00895EF92FF9209
:10EB70000F931F93CF93DF938C01EA01FC018081F7
:10EB80009181009741F08A33934081F1F80111821D
:10EB9000108283E0F8C080E024E0829FF00111241D
:10EBA000EB5FF34E118210828F5F8430A9F7809360
:10EBB000021C8091E1149091E2149093161C8093B2
:10EBC000151C0E94666F8093DD3740E450E060E0E2
:10EBD00070E087E19CE10E94516E0E94467A8AE3D0
:10EBE00093E0F8019183808381E0CDC06230D9F455
:10EBF0008091DE379091DF37892B89F38091EF3751
:10EC0000863029F48091073881FD0E94A27581E049
:10EC10000E948D7A8091DE379091DF37892BF9F24F
:10EC20000E941077DCCF633060F5611114C020972B
:10EC3000B1F2D093DC38C093DB3883E00E948D7A48
:10EC40008091DE379091DF37892B11F00E94AD75EE
:10EC50000E94A275C4CF613011F6209709F4BFCF8E
:10EC6000D093D838C093D73885E00E948D7A8091B0
:10EC7000DE379091DF37892B09F4B1CF0E94AD7553
:10EC8000AECF673809F040C01092011C85E0E82E35
:10EC90008CE1F82E8091011C8430C0F4F701828150
:10ECA00093818C179D0749F4808191810E94727A2B
:10ECB000F7011182108213821282F4E0EF0EF11C30
:10ECC0008091011C8F5F8093011CE4CFE6EFF8E395
:10ECD000838194818C179D0719F41482138210820A
:10ECE000B09629E3E637F20799F7E3E7F9E3818580
:10ECF00092858C179D0711F4158214823D9689E345
:10ED0000E53FF807A1F76BCF683809F068CFC75126
:10ED1000DC4109F064CF87E19CE10E946F6E892B92
:10ED200009F45DCF1092011CE091011CE43008F061
:10ED300056CF20E2E29FF0011124E352F74C818D7F
:10ED40008823D9F087E19CE10E94656E8091011CC7
:10ED5000E0E28E9FC00111248352974C9093DC38DF
:10ED60008093DB3882E00E948D7A8091DE3790912B
:10ED7000DF37892B11F00E94AD758091011C8F5FE8
:10ED80008093011CD1CFDF91CF911F910F91FF9004
:10ED9000EF900895CF93DF93A091DB38B091DC38EA
:10EDA000109719F0ED016C9605C0C091D738D0913D
:10EDB000D83829968091D63886FF23C01092001C3F
:10EDC00080E0E5E0FCE18430C1F04081518114969F
:10EDD0002D913C9115974217530761F4228133819D
:10EDE0002115310539F08093001C398328831B825B
:10EDF0001A8205C034968F5FE6CF8093001C0E9474
:10EE0000A27588819981009741F04A815B81609168
:10EE1000DD37DF91CF910C940070DF91CF91089591
:10EE20000F931F93CF93DF938091EF37863009F0D4
:10EE30007AC08091DE379091DF37803F910508F4EA
:10EE400072C08897EC01D695C7959E01220F331F9B
:10EE50008E012817390710F40F5F1F4FCE018896D7
:10EE60009093DF378093DE379093E8378093E937CC
:10EE700010920B3810920A380E94407A8095909533
:10EE800090930B3880930A381092F1371092F03734
:10EE90000E942F7A809590959093F1378093F03768
:10EEA0000E94AD75C80188969093DF378093DE3756
:10EEB0009093E8378093E9378091D9389091DA3888
:10EEC000BC016C0F7D1FA8010E947792BE018EEFDE
:10EED00097E30E94DC798091E2378093FE3780913E
:10EEE000E3378093FF378091E43780930038809137
:10EEF000E5378093013810920B3810920A380E943F
:10EF0000407A8095909590930B3880930A381092B0
:10EF1000F1371092F0370E942F7A80959095909358
:10EF2000F1378093F037DF91CF911F910F910C94BF
:10EF3000AD75E091B609F091B709199480E090E0C1
:10EF40000895AF92BF92CF92DF92EF92FF920F930C
:10EF50001F93CF93DF93CDB7DEB7E1970FB6F89449
:10EF6000DEBF0FBECDBF7C016B01CE0101965C01FF
:10EF700081E3F50111928A95E9F781E089838CE0BC
:10EF80000E9436758C831D821F828091231C91E024
:10EF9000980F9093231C898713E018878DEC9BEAC8
:10EFA0009B878A8789E10E94497560E07AE00E9428
:10EFB000FF73892B31F082E08E838FEF8C878D87F2
:10EFC00009C089E10E944975BC01CE010C960E94DE
:10EFD000F8731E838DEC9BEA9D8B8C8B63EA77E341
:10EFE000CE0146960E94F8730E9446749FA78EA792
:10EFF0000E948E7499AB88ABC5010E947A838C0104
:10F000001127C8010E94A074892B31F10E944D7410
:10F01000A801BC01C5010E949D830091AC0910911B
:10F02000AD090E9493745C010E944D74B501F80112
:10F030001995E114F10481F0009739F0019761F41A
:10F0400041E050E064E070E004C041E050E060E086
:10F0500070E0C601F7011995E1960FB6F894DEBF8E
:10F060000FBECDBFDF91CF911F910F91FF90EF9019
:10F07000DF90CF90BF90AF9008950F931F93CF93E1
:10F08000DF934115510579F0FA018B01EC01828182
:10F0900093810E945B75B801CE01DF91CF911F91E2
:10F0A0000F910C94A177DF91CF911F910F9108954B
:10F0B0000F931F93CF93DF93CDB7DEB7E1970FB6D2
:10F0C000F894DEBF0FBECDBF0E948E748C010E94EB
:10F0D0004674AE014F5F5F4FB8010E949084892B48
:10F0E00009F443C088A999A99801281B390BC901C3
:10F0F0000E942474892BC9F18E8181110CC0BE013C
:10F100006A5E7F4F88E10E943F75E091F809F091B7
:10F11000F90919952AC02A853B852D3C9BEA3907B8
:10F1200019F02F3F3F4F09F5823019F088E090E049
:10F1300002C082E090E0019710F3E1E0F0E0EC0F14
:10F14000FD1FE80FF91F23852F3FA9F3BE01645F60
:10F150007F4F89E10E943F7589E10E94497563EA0A
:10F1600077E30E94FF73892B51F6E1960FB6F8946E
:10F17000DEBF0FBECDBFDF91CF911F910F910895DC
:10F180000E9452668093231CE091B609F091B70962
:10F190001994892B29F0E091B609F091B70904C0C0
:10F1A000E091B809F091B9091994FC01680F791F31
:10F1B00080E048E1E617F70781F0219198E0322FCF
:10F1C0003827532F517030FD84278695513009F42C
:10F1D00080682695915099F7EDCF08951F920F9270
:10F1E0000FB60F9211240BB60F922F933F934F93AC
:10F1F0005F936F937F938F939F93AF93BF93EF939F
:10F20000FF93809194009091950090939037809314
:10F210008F3781E08093813780917100807D80936A
:10F2200071000E943E70809181378823D9F18091CE
:10F2300094009091950040918F37509190378417AA
:10F240009507A0F48091553790915637A091573784
:10F25000B0915837875F924CAF4FBF4F809355376F
:10F2600090935637A0935737B09358372091940016
:10F2700030919500241B350B80915537909156376E
:10F28000A0915737B0915837820F931FA11DB11D20
:10F290008093553790935637A0935737B09358378C
:10F2A00010928137FF91EF91BF91AF919F918F9114
:10F2B0007F916F915F914F913F912F910F900BBE76
:10F2C0000F900FBE0F901F9018959FB7F894E1E72D
:10F2D000F0E08081807D808388B38F6288BB10924C
:10F2E0009000E1E9F0E010821092920010929500F7
:10F2F000109294008081856080839FBF08959C0157
:10F300009FB7F894309399002093980088B38F6248
:10F3100088BBE1E7F0E08081826080839FBF089531
:10F32000FB0141505109460F571FE417F50778F4C8
:10F33000208130E0322F22276181260F311D820F7C
:10F34000931F8217930708F401963296EECFE417C5
:10F35000F50751F4208130E0322F2227820F931FCE
:10F360008217930708F401960895CF93DF93C09115
:10F37000E937D0E064972091E83730E0322F222738
:10F38000C20FD31F48E050E062EF77E39E01280FE1
:10F39000311DC9010E949079AE016AEF77E30E94A6
:10F3A0009079009721F098278927982702C08FEF3E
:10F3B0009FEFDF91CF910895FC012381260F2093C9
:10F3C000E537A72FBB2792819A0F9093E4373181BD
:10F3D0003093E33740814093E237E92FF0E0EA17BA
:10F3E000FB0748F481E0830F8093E337811103C06A
:10F3F0004F5F4093E23730E077272617370788F4CE
:10F400009F5F9093E43791110CC08091E3378F5F39
:10F410008093E337811105C08091E2378F5F80933D
:10F42000E23708952091DB383091DC38BC01C90106
:10F4300008960E94DC79E091DB38F091DC38A2EE8E
:10F44000B7E38C91808711968C91119781871296E2
:10F450008C911297828713968C918387089544E14B
:10F4600050E066EE77E380E090E00E9490790097AC
:10F4700021F098278927982708958FEF9FEF089507
:10F4800086E00C94B57981E10C94B57980E0E82FA1
:10F49000F0E0EE0FFF1FE35AF64C118210828F5FEF
:10F4A0008430A9F780E090E2899FF0011124E352B3
:10F4B000F74C118E8F5F8430B1F780E094E0909329
:10F4C000291C8093281C80E09DE0989FF001112466
:10F4D000ED58F64C158214828F5F8A30B1F7809315
:10F4E000271C08959C0190E09430A1F0E92FF0E0F2
:10F4F00081E0890FEE0FFF1FE35AF64C40815181E6
:10F500004217530729F49093271C11821082089503
:10F51000982FEACF9093271C0895AF92BF92CF9275
:10F52000DF92EF92FF920F931F93CF93DF93C091DF
:10F53000DB38D091DC38843009F4DBC12EE038E3CD
:10F540003093DA382093D9383093E1372093E0377D
:10F55000833059F4898D8F70833009F06AC08889AF
:10F560009989892B09F0D4C67EC0823009F07FC00A
:10F5700080912D1C8F5F80932D1C811113C0809171
:10F580002C1C8F5F80932C1C81110CC080912B1C34
:10F590008F5F80932B1C811105C080912A1C8F5F87
:10F5A00080932A1C1092DF371092DE371092723946
:10F5B00010927139898D982F9D7F953041F48A8DF5
:10F5C0008F5F8A8F843109F0A3C6198EA1C6882364
:10F5D00009F49EC628893989232B09F440C09A8DE5
:10F5E0002FEF290F2A8F911193C69B8D983031F000
:10F5F0002FEF280F223048F4953039F4198E80E827
:10F600008093D6380E94CA763DC5953038F423E001
:10F61000092E01C0220F0A94EAF701C020E32A8FC5
:10F620009F5F9B8F8F708330A1F048F4813009F485
:10F6300044C3823009F06CC61092073841C386304B
:10F6400009F4BCC4883009F4B9C4843009F060C638
:10F65000B5C484E08093D6380E94CA7645C58F70C1
:10F66000833009F055C688E08093D63800C58530D0
:10F6700019F5E091D738F091D83884819581892B9C
:10F6800009F446C61092DC381092DB3882E098E329
:10F690009093DA388093D9389093E1378093E037AC
:10F6A00010927239109271391092DF371092DE3752
:10F6B00088E08093D6381BC18091E637853409F005
:10F6C00027C60091E83710E0102F00278091E93716
:10F6D000080F111D8091DE379091DF378017910759
:10F6E00008F416C61093DF370093DE378091EC37AD
:10F6F0008F7309F00DC6F090ED37F11009C68091B7
:10F700006D3990916E39C0912A0AD0912B0A8C17CD
:10F710009D0759F440916F395091703920912C0A0E
:10F7200030912D0A42175307A1F02091F6373091FE
:10F73000F7372817390709F0EBC52091F8373091D2
:10F74000F93780916F39909170392817390709F08E
:10F75000DFC50E942F7A019609F0DAC58091EF3754
:10F76000863009F429C18131E9F1813009F0D0C531
:10F770008091FA37883009F0CBC51092FA37809122
:10F78000FC379091FD37873F6FEF960710F0099691
:10F7900001C008969093FD378093FC378091F23733
:10F7A0009091F337A091F437B091F5378093F63705
:10F7B0009093F737A093F837B093F93780916D396C
:10F7C00090916E39A0916F39B09170398093F23772
:10F7D0009093F337A093F437B093F53780E4809398
:10F7E000EE3773C50C5111091093DF370093DE37E4
:10F7F00082E098E39093DA388093D938809100388A
:10F8000090910138892B29F00E94437A019609F0E2
:10F810007FC52091FC373091FD372115310509F462
:10F8200077C583E799E39093D8388093D738A09031
:10F83000FA37B090FB3740912E0A50912F0A609111
:10F84000300A7091310AA091F237B091F3370091EC
:10F85000F4371091F537E0902C0AF0902D0AE091E2
:10F86000D738F091D83889E3E53FF80708F050C55C
:10F8700084819581009721F12817390709F5868140
:10F880009781009719F0A816B906D1F4808191816B
:10F890008C179D0729F4C280D380CE14DF04B1F009
:10F8A0008417950729F4C280D380C616D70671F055
:10F8B000A817B90729F4828193810817190731F035
:10F8C0003D96F093D838E093D738C9CF1092DC3802
:10F8D0001092DB3882E08093D63882E098E39093F0
:10F8E000E1378093E03710927239109271390E949B
:10F8F000CA768091713990917239009709F408C5E0
:10F900009C01245E3F4F3093DF372093DE373093E6
:10F91000E8372093E937E091D738F091D83820853F
:10F920002093EE3721E12093EF3708969827892717
:10F9300098279093FF378093FE37109201381092EA
:10F940000038848195819093FB378093FA378681C4
:10F9500097819093FD378093FC3780916D3990911A
:10F960006E39A0916F39B09170398093F2379093CE
:10F97000F337A093F437B093F53780819181A2815A
:10F98000B3818093F6379093F737A093F837B0930D
:10F99000F9378EE098E39093DA388093D9380E9453
:10F9A000437A80959095009711F48FEF9FEF909395
:10F9B00001388093003889C40E94407A019609F08A
:10F9C000A7C44091FC375091FD374115510509F40A
:10F9D0009FC48091FA379091FB37009709F498C43F
:10F9E0006091F2377091F337E091F437F091F53789
:10F9F000CDEDD8E3298D2223A9F0AC81BD814A1732
:10FA00005B0781F4AE81BF818A179B0759F4A881F7
:10FA1000B9816A177B0731F4AA81BB81EA17FB071A
:10FA200009F466C1A09629E3CD35D20719F7809174
:10FA300007388F738230D9F45093251C4093241CCF
:10FA400080E0843091F0E82FF0E0EE0FFF1FE35AE2
:10FA5000F64C208131818F5F4217530791F7109246
:10FA6000271C80E0C0E0D0E07CC08093271C809100
:10FA7000073882FD4DC484E18093073888E290E026
:10FA80009093DF378093DE3780E58093063830919E
:10FA90000138809105388093013820910038809199
:10FAA000043880930038209304389091FF37809178
:10FAB00003388093FF37909303388091FE3780930B
:10FAC000271C409102384093FE37809302383F5FF5
:10FAD0003093053831110DC02F5F20930438211168
:10FAE00008C09F5F90930338911103C08F5F80938C
:10FAF00002388091FA379091FB379093251C8093C0
:10FB0000241C2091FC373091FD373093FB37209334
:10FB1000FA379093FD378093FC378091F2379091BC
:10FB2000F337A091F437B091F5378093F63790937F
:10FB3000F737A093F837B093F93780916D399091EA
:10FB40006E39A0916F39B09170398093F2379093EC
:10FB5000F337A093F437B093F5379CC3973089F00F
:10FB60008F5F8430C1F060E2869F90011124F9011B
:10FB7000E352F74C918D9111F1CF8093271CEF0147
:10FB80000CC0209721F0428D9A8D941748F7E90117
:10FB9000C352D74CE5CF8093271C209709F4B8C3F4
:10FBA000D093DC38C093DB3883E08A8F888F1E8A3D
:10FBB00084E08F8B1B8E8091FC379091FD379D8365
:10FBC0008C838091FA379091FB379F838E8380914D
:10FBD000F2379091F337A091F437B091F5378883DD
:10FBE0009983AA83BB8381E0898F80912A1C8C87AB
:10FBF00080912B1C8D8780912C1C8E8780912D1CD1
:10FC00008F8781E090E0998B888B809101388B877A
:10FC1000809100388A878091FF3789878091FE37ED
:10FC2000888781E090E00E94127A80910638982FB0
:10FC3000907F913508F441C082958F7090E00597D0
:10FC4000880F991F880F991F2091261CEF2DF0E037
:10FC5000E817F90774F5EA51F84C20A5211103C003
:10FC60001092261C28C0213011F4F394EFCF2230DB
:10FC7000D9F431A53430C1F42093261CF092271C0E
:10FC800082A590E0982F882723A5822B9093251C8E
:10FC90008093241C893C910510F088EC90E09B8BAC
:10FCA0008A8B9D8B8C8B09C031A5332311F0F30E09
:10FCB000CDCF2093261CF092271C80E1809307383B
:10FCC0008091073882608093073882E080930E38F5
:10FCD00084E080930F381092103888EC80931138AC
:10FCE0008CE290E09093DF378093DE3780E680C22D
:10FCF000D093DC38C093DB381092D6388091073827
:10FD0000782F7470F72E82FF03C0198E80E219C21B
:10FD10009091063892959F70990F990F9093271C98
:10FD2000091B1109045111091093DF370093DE37C5
:10FD3000922F9F70923029F4982F9F73923139F44B
:10FD40001FC0913021F4982F9F739230C9F0012B7E
:10FD500019F4982F9370A1F02091FE3798852913FC
:10FD60003DC22091FF379985291338C22091003870
:10FD70009A85291333C2209101389B8529132EC2FD
:10FD800084FF49C0688979896115710509F443C008
:10FD9000CE010C960E94DC79309102388091E237D6
:10FDA000381339C0209103388091E337281333C0CA
:10FDB000909104388091E43798132DC080910538D4
:10FDC0004091E537841327C03C872D879E878F8716
:10FDD0008B8D811119C09E89888D2A8D821B292FB8
:10FDE000269526952695821B980F9E8B87FD8195DB
:10FDF0002F89322F36953695231B820F8F8B969540
:10FE000096959695890F888F81E08093D638888D56
:10FE10008A8F198A188A298DE22FEF708E2F90E031
:10FE2000FC013197E830F10508F072C28827E656E8
:10FE3000FF4F8F4F0C9436888091D63880FF14C0C6
:10FE400083E0898F80E48093D638198A188A80915C
:10FE5000DE379091DF37009709F405C122E4209343
:10FE6000D6380E94127AFFC0809107388F73823093
:10FE700009F04EC222CF8091D63880FF6AC08091AF
:10FE800007388F73823109F064C080910638982F4B
:10FE9000907F913508F441C082958F7090E005976E
:10FEA000880F991F880F991F2091261CEF2DF0E0D5
:10FEB000E817F90774F5EA51F84C20A5211103C0A1
:10FEC0001092261C28C0213011F4F394EFCF223079
:10FED000D9F431A53430C1F42093261CF092271CAC
:10FEE00082A590E0982F882723A5822B9093251C2C
:10FEF0008093241C893C910510F088EC90E09B8B4A
:10FF00008A8B9D8B8C8B09C031A5332311F0F30EA6
:10FF1000CDCF2093261CF092271C83E0898F8091FF
:10FF2000FE3788878091FF378987809100388A87DC
:10FF3000809101388B8781E090E00E94127A82E400
:10FF40008093D638198A188A1092DF371092DE37DC
:10FF50008AC080E28093D6380E94CA76E091DB386E
:10FF6000F091DC38118E83CD8091073880FF28C056
:10FF700024FD26C088899989892B09F0C9C18091FF
:10FF8000DE379091DF3701960E94127A8091D63841
:10FF9000982F90619093D6382091DE373091DF37DB
:10FFA000232B19F082618093D6380E94CA7681E0B3
:10FFB00090E0998B888B88E0898F1B8E81E10FC13F
:10FFC00085FF1DC080910C3890E0982F88273091D4
:10FFD0000D38832B4091D9385091DA38480F591F8A
:10FFE0005093DA384093D9384091DE375091DF375B
:10FFF000BA01681B790B7093DF376093DE3740914D
:020000021000EC
:10000000DE375091DF374115510551F024FD08C00E
:100010009091D63892609093D638CA010E94127A95
:100020008091083890E0982F882720910938820F16
:10003000911D9093251C8093241C2C893D892817A1
:10004000390710F0892B21F43093251C2093241CB0
:100050008091241C9091251C9B8B8A8B8091D63893
:10006000837009F455C110927239109271390E944F
:10007000CA768091D63885FF07C0109272391092E7
:100080007139198E84E1ABC084FF0AC010927239B5
:100090001092713981E090E0998B888B84E08CCF4D
:1000A000209171393091723921153105E1F080FFCD
:1000B00002C0198A188A88899989009781F48A89E7
:1000C0009B898217930720F490937239809371393A
:1000D0008091713990917239998B888B04C090937B
:1000E0007239809371391B8E8091E0379091E1379E
:1000F0009093DA388093D938809171399091723920
:10010000892B59F088899989009739F088969093BE
:10011000DF378093DE3788E10BC08091D63881FFCE
:10012000F7C088E290E09093DF378093DE3780E17C
:10013000809307385CC08091D63880FFE9C0198E63
:1001400080E18093D6380E94CA76E2C08091DE3783
:100150009091DF37009711F00E94127A9091073842
:100160008091D63890FF0BC080FF06C087E0898F52
:100170001A8E198A188A19C086E0898F16C080FFE6
:100180001EC085E0898F198A188AC2C08091DE3727
:100190009091DF37009711F00E94127A8091073812
:1001A00080FF0DC087E0898F1A8E81E090E00E9469
:1001B000127A80E18093D6380E94CA760FC080916F
:1001C000DE379091DF37892B49F4A2C08091D63871
:1001D00080FF9EC087E0898F1A8E9AC080E180934D
:1001E000073888E290E09093DF378093DE3780E530
:1001F00080930638888580930238898580930338F8
:100200008A85809304388B85809305388C8580930C
:10021000FE378D858093FF378E85809300388F85DC
:100220008093013886E08093EF378C819D81909395
:10023000FB378093FA378E819F819093FD378093AF
:10024000FC3780916D3990916E39A0916F39B091E2
:1002500070398093F2379093F337A093F437B093CB
:10026000F53788819981AA81BB818093F637909375
:10027000F737A093F837B093F937898D84FF05C01D
:10028000109209381092083805C01092083888EC8E
:100290008093093880E48093EE378091DE37909127
:1002A000DF379093E8378093E93710920D3810923A
:1002B0000C3810920B3810920A380E94407A8095C0
:1002C000909590930B3880930A3885E48093E637B5
:1002D0001092E7371092ED371092EC3780912E1C78
:1002E00090912F1C019690932F1C80932E1C90931D
:1002F000EA378093EB371092F1371092F0370E9473
:100300002F7A809590959093F1378093F03704C0C1
:100310001092DF371092DE371092D638DF91CF91EE
:100320001F910F91FF90EF90DF90CF90BF90AF9013
:10033000089582E39CE10C94B6709093311C8093F5
:10034000301C089582E39CE10C94BA70EF92FF9206
:100350000F931F93CF93DF938C01EB017A0182E31C
:100360009CE10E94BA700097D9F0DC0112962D91A1
:100370003C9113972C173D0781F41696ED91FC9153
:100380001797309769F09701AE01B801DF91CF91CF
:100390001F910F91FF90EF9019940E941B71E3CF72
:1003A000DF91CF911F910F91FF90EF9008950895E5
:1003B0000F931F93CF93DF93C3E7DCE1488159810B
:1003C0006A817B8100E010E022E032E883E59CE175
:1003D0000E94EF6C0E945266BC0180E090E0288190
:1003E00039814A815B810E94F587AB01BC0127E21C
:1003F00032E88FE39CE10E94EF6CDF91CF911F9177
:100400000F9108958091731C9091741CA091751C9C
:10041000B091761C40916F1C5091701C6091711CC2
:100420007091721C880F991FAA1FBB1F481759078C
:100430006A077B0710F4DB01CA018093731C909359
:10044000741CA093751CB093761C0C94D881CF9328
:10045000DF930E94D7740E944674EC0119821882BF
:100460000E94A28128813981009719F1FC01408501
:100470004423F9F0FC0142815381F901EE0FFF1F83
:10048000EE0FFF1FEC0FFD1F53834283FC014481DD
:1004900055812F5F3F4FF901EE0FFF1FEE0FFF1F3A
:1004A000EC0FFD1F51834083398328830E941B7109
:1004B000D9CFC901880F991F880F991F02960E94F2
:1004C000417488819981892B31F084E39CE1DF912B
:1004D000CF910C94FD72DF91CF910895AF92BF92AE
:1004E000CF92DF92EF92FF920F931F93CF93DF9300
:1004F0001F921F92CDB7DEB75B010E9446748C013C
:10050000FC01E080F180FA82E9820E948E749701FA
:10051000220F331F220F331F2E5F3F4F8217930787
:1005200098F0C12CD12CCE14DF0471F0F801448175
:10053000558162817381C5010E94A681FFEFCF1AA8
:10054000DF0A0C5F1F4FEFCF0F900F90DF91CF911D
:100550001F910F91FF90EF90DF90CF90BF90AF90E1
:1005600008950F93013099F48091671C9091681C55
:10057000A091691CB0916A1C8093731C9093741CA9
:10058000A093751CB093761C0F910C94D8810F9199
:1005900008954F925F926F927F928F929F92AF9247
:1005A000BF92CF92DF92EF92FF920F931F932A0197
:1005B0003B014801590142E35AE0BC0184E39CE15C
:1005C0000E94E072E4E3FCE143AA54AA65AA76AA79
:1005D00087AA90AEA1AEB2AEC3AED4AEE5AEF6AED3
:1005E00081EB92E81F910F91FF90EF90DF90CF90F9
:1005F000BF90AF909F908F907F906F905F904F9043
:100600000C949D810C940A73CF93DF93E091360A8A
:10061000F091370A1995EC01892B29F06A817B81C9
:1006200081E00E942B75CE01DF91CF9108950F9349
:100630001F93CF93DF93EC01E091380AF091390AD0
:1006400019958C016A817B8181E00E942B7581E084
:1006500090E0012B11F480E090E0DF91CF911F91A9
:100660000F910895E0913A0AF0913B0A1994CF93C3
:10067000DF93FC01DB0185E0EB0119928A95E9F734
:100680008581837011F082E08C938781837021F0E3
:1006900082E012968C9312978581837081F0878116
:1006A000837069F0238934898185928528173907F9
:1006B00031F481E0848312961C92129701C0148257
:1006C00085818370823029F0833011F488E001C085
:1006D00080E011968C93119787818370823029F086
:1006E000833011F488E001C080E013968C93DF9191
:1006F000CF910895CF93DF9300D01F921F92CDB773
:10070000DEB7BE016F5F7F4F0E943783898190E023
:1007100003962A81820F911D2B81820F911D2C81BE
:10072000820F911D2D81820F911D0F900F900F90C0
:100730000F900F90DF91CF9108953F924F925F926B
:100740006F927F928F929F92AF92BF92CF92DF92E1
:10075000EF92FF920F931F93CF93DF9300D01F92DE
:100760001F92CDB7DEB78C017B013A01BE016F5FEE
:100770007F4F0E94378369817A81472F50E0EB8158
:100780003C80232D30E0862F90E00396840F951F48
:100790008E0F911D820F931FAD818A0F911D6816D8
:1007A00079060CF4A4C0D80111968C91119780FBA6
:1007B000882480F8912C83E0880C991C8A95E1F7B5
:1007C00012968C91129780FBAA24A0F8B12C94E089
:1007D000AA0CBB1C9A95E1F78A288C918770882A0D
:1007E00013968C91139780FBCC24C0F8D12CF5E0A4
:1007F000CC0CDD1CFA95E1F7C82814968C9180FB8F
:10080000442440F8512CA6E0440C551CAA95E1F76D
:100810004C28D7014C92D80115968C918370B4E086
:100820008B9F60011124D80116969C919370B0E1C2
:100830009B9FC00111248C29D8011796FC9190E44C
:10084000F99FD00111248A2BD70111968C93D801DE
:1008500018968C91D70112968C93623071F4D8015E
:1008600019968C91D70113968C93D8011A968C9176
:10087000D70114968C9385E001C083E0780F872F11
:10088000972F941B4115510561F041505109D80132
:10089000A40FB51F1B968C91D701A90FB11D8C9386
:1008A000EECFE23071F4D701A70FB11DF8019389A3
:1008B0009C9391E0970FD701A90FB11D8E5F94898A
:1008C0009C93F32DF80F8F2F821B2115310561F0BA
:1008D00021503109D801A20FB31F55969C91D70121
:1008E000A80FB11D9C93EFCF8F2F90E002C080E046
:1008F00090E00F900F900F900F900F90DF91CF919D
:100900001F910F91FF90EF90DF90CF90BF90AF902D
:100910009F908F907F906F905F904F903F90089541
:10092000AF92BF92CF92DF92EF92FF920F931F93FD
:10093000CF93DF93633071050CF4B3C0EA016B0110
:100940007C01FC01908196FBAA24A0F88181282FCC
:10095000269526952370B82EB294B694B69453E09B
:10096000B522392F3770388393FB332730F9398319
:1009700094FB332730F93A8395FB992790F99B83B1
:10098000AC822D83829583708E83BF82828188871B
:10099000222379F13381848190E0982F8827830F77
:1009A000911D9A87898787010B5F1F4F223071F451
:1009B00060E07AE0CE010B960E94F873F701868121
:1009C0008B8785818C870E5F1F4F1EC02330E1F41B
:1009D000F7013D96DE011B969E012D5E3F4F9E2F37
:1009E0008F2F42914D93A217B307D9F7092F182FD4
:1009F0000BC087010D5F1F4F60E07AE0CE010B96C0
:100A00000E94F8731A861986BB20A1F1A1100DC0AF
:100A1000F8012081818190E0982F8827820F911D15
:100A20009C8B8B8B0E5F1F4F04C089859A859C8B96
:100A30008B8BF2E0BF120EC060E07AE0CE014596EB
:100A40000E94F873F80181818D8B80818E8B0E5FFF
:100A50001F4F18C0F3E0BF1215C0085F1F4FD80129
:100A6000FE017596CE014D962E912193E817F90758
:100A7000D9F708C060E07AE0CE0145960E94F8738D
:100A80001C8A1B8A98012E193F09C601821B930BF1
:100A900098AB8FA71EA70DA7C216D30614F0C901E5
:100AA00002C080E090E0DF91CF911F910F91FF9005
:100AB000EF90DF90CF90BF90AF90089520E030E0AE
:100AC0000296FC0132974081442331F0FC013197BA
:100AD0004081240F311DF4CFC9010895FC0120810C
:100AE00030E0322F22278181282B02C0220F331FB2
:100AF0006A95E2F7232F3327FA01E45CF54F8081F2
:100B000090E08223932328E030E0241B350B02C0C1
:100B1000969587952A95E2F708956F927F928F9226
:100B20009F92AF92BF92CF92DF92EF92FF920F937C
:100B30001F93CF93DF937C018B015A01E901283089
:100B4000310544F4A901B501C8010E946E85F70181
:100B5000808346C0690183E0D594C7948A95E1F704
:100B6000452B21F04701612C712C06C0FB01D701F8
:100B7000CB018C0D9D1D1FC048E050E0B501C801A0
:100B8000860D971D0E946E85F40181934F01FFEF42
:100B90006F1A7F0A6C147D0479F7AE0147705527F0
:100BA00041155105E9F0E701C60DD71DB501C80192
:100BB000860D971D12C0E817F90719F021912D93A2
:100BC000FACFAE01477055274115510549F0E701AD
:100BD000CC0DDD1D60E070E0CF010E946E85888342
:100BE000DF91CF911F910F91FF90EF90DF90CF9009
:100BF000BF90AF909F908F907F906F9008958F924D
:100C00009F92AF92BF92CF92DF92EF92FF920F939B
:100C10001F93CF93DF931F921F92CDB7DEB70E9431
:100C200046748C0182E090E00E942474892B19F4B0
:100C300080E090E05FC0F801218130E0322F222770
:100C40008081A901480F511DCA010E941B737C01BC
:100C5000892B71F30E9446744C01F7019681292F6C
:100C600026952695269530E0977041E050E011F4E6
:100C700040E050E0C901840F951F0E942474892B25
:100C8000B9F2F70104811581A12CB12CF801808102
:100C9000882379F1F801C180D12CA501477055272F
:100CA000B50193E0759567959A95E1F7680D791D03
:100CB000883168F09601CE0101960E948D85BE01B3
:100CC0006F5F7F4FF80180810E943F750DC01A82CF
:100CD00019829601CE0101960E948D8569817A81E3
:100CE000F80180810E942B75AC0CBD1C0E5F1F4F5C
:100CF000CDCFC7010F900F90DF91CF911F910F9132
:100D0000FF90EF90DF90CF90BF90AF909F908F902B
:100D10000895DC0150E0E0E1F0E0CF01861B970B85
:100D2000821B930B02C0440F551F8A95E2F78C91EA
:100D3000852B8C9311968C911197482B11964C937F
:100D400008956F927F928F929F92AF92BF92CF92AF
:100D5000DF92EF92FF920F931F93CF93DF93283090
:100D600031051CF4FA0140815AC05901E3E0B59401
:100D7000A794EA95E1F76115710541F03901EA019F
:100D80008B017C014A01C12CD12C05C0EA01FC0178
:100D90004A0D5B1D2AC0F40141914F0128E030E06B
:100DA000B801C7018C0D9D1D0E948986FFEFCF1AE7
:100DB000DF0ACA14DB0479F7930127703327211562
:100DC0003105E9F1CC0DDD1D488150E0021B130B0C
:100DD000085F1F4F02C0559547950A95E2F760E0FE
:100DE00070E0C7018C0D9D1D1AC0C417D50719F0FE
:100DF00069916193FACF2770332721153105F9F0F6
:100E0000488150E068E070E0621B730B02C05595AA
:100E100047956A95E2F760E070E08A0D9B1DDF91CF
:100E2000CF911F910F91FF90EF90DF90CF90BF90E7
:100E3000AF909F908F907F906F900C948986DF91F8
:100E4000CF911F910F91FF90EF90DF90CF90BF90C7
:100E5000AF909F908F907F906F9008956F927F9248
:100E60008F929F92AF92BF92CF92DF92EF92FF92BA
:100E70000F931F93CF93DF931F921F92CDB7DEB7CF
:100E80007C01FC018681082F069506950695202F8A
:100E900030E0877001E010E011F400E010E0020F94
:100EA000131FC80102960E94A074009709F448C05D
:100EB0000E944D74F7012281FC012083F7012381F8
:100EC000FC0121830E944D7402965C01A80160E040
:100ED00070E00E948092F701048115810F5F1F4F1F
:100EE000812C912CF80131978081882339F1F80108
:100EF000C080D12C3401F7E06F227724740193E095
:100F0000F594E7949A95E1F7EA0CFB1C883128F0F8
:100F10000E9449759601AC0108C00E9436759A83FB
:100F200089839601AE014F5F5F4FB301C7010E94F5
:100F3000A1868C0C9D1C0E5F1F4FD4CF81E090E0EA
:100F40000F900F90DF91CF911F910F91FF90EF9035
:100F5000DF90CF90BF90AF909F908F907F906F90D9
:100F60000895DB018F939F930E945C88BF91AF919E
:100F7000A29F800D911DA39F900DB29F900D1124F3
:100F80000895991B79E004C0991F961708F0961BE5
:100F9000881F7A95C9F780950895AA1BBB1B51E15C
:100FA00007C0AA1FBB1FA617B70710F0A61BB70BD9
:100FB000881F991F5A95A9F780959095BC01CD017E
:100FC000089597FB072E16F4009407D077FD09D0FB
:100FD0000E94CD8707FC05D03EF4909581959F4FE8
:100FE0000895709561957F4F0895A1E21A2EAA1B6E
:100FF000BB1BFD010DC0AA1FBB1FEE1FFF1FA217C9
:10100000B307E407F50720F0A21BB30BE40BF50BC5
:10101000661F771F881F991F1A9469F7609570954E
:10102000809590959B01AC01BD01CF010895052EDF
:1010300097FB1EF400940E942E8857FD07D00E9453
:10104000F58707FC03D04EF40C942E8850954095FC
:10105000309521953F4F4F4F5F4F08959095809564
:10106000709561957F4F8F4F9F4F0895EE0FFF1F33
:10107000881F8BBF0790F691E02D19940E94468837
:10108000332312F48A1B9B0B0C945788A29FB00148
:10109000B39FC001A39F700D811D1124911DB29FAC
:1010A000700D811D1124911D08950E944688B7FF7F
:1010B0000895821B930B08950E944688A59F900D6A
:1010C000B49F900DA49F800D911D11240895B7FF2A
:1010D0000C945C880E945C88821B930B0895DF93BC
:1010E000CF931F930F939A9DF02D219FF00D8B9D11
:1010F000F00D8A9DE02DF10D039FF00D029FE00D94
:10110000F11D4E9DE00DF11D5E9DF00D4F9DF00D0A
:101110007F936F93BF92AF925F934F93D5010E94DD
:1011200046888B01AC01D7010E944688EB01E80F8D
:10113000F91FD6010E94BF882F913F91D6010E94CE
:101140004688C60FD71FE81FF91FAF91BF910E94B5
:10115000BF882F913F910E944688C60FD71FE81F76
:10116000F91FD6010E944688E60FF71F9801BE01BD
:10117000CF0111240F911F91CF91DF9108950E940B
:101180004688460F571FC81FD91F08F43196089587
:10119000E894DF93CF93FC01DB010E9446887F93A4
:1011A0006F93E9019A01AC01BF93AF933F932F93E3
:1011B000DF010E94468826F46C1B7D0B820B930B8B
:1011C0009E01EB01FC010E94BF88AF91BF912F915E
:1011D0003F910E94BF88BE01CF01F9012F913F913D
:1011E000CF91DF910895689401C0E894F92FF12B15
:1011F00012F00C942789A0E0B0E0E1E0F9E80C944B
:101200009989092E059422F40E948389112392F46E
:10121000F0E80F26FFEFE094F09400951095B0945D
:10122000C094D094A194BF0ACF0ADF0AEF0AFF0A44
:101230000F0B1F0B0E94328907FC0E948389CDB7D8
:10124000DEB7ECE00C94B589689401C0E8948F9205
:101250009F92CF93DF930E943289DF91CF919F902D
:101260008F90089588249924F401E401B0E49F93B9
:10127000AA279A158B049C04ED05FE05CF05D0071F
:10128000A10798F4AD2FDC2FCF2FFE2FE92D982C3E
:10129000892E982F872F762F652F542F432F322F8B
:1012A0002227B85031F7BF9127C01B2EBF91BB2713
:1012B000220F331F441F551F661F771F881F991F5A
:1012C000881C991CEE1FFF1FCC1FDD1FAA1FBB1F10
:1012D0008A149B04EC05FD05CE05DF05A007B107C8
:1012E00048F08A189B08EC09FD09CE09DF09A00B1C
:1012F000B10B21601A94E1F62EF49401AF01BE0106
:10130000CD01000C0895609570958095909530956D
:101310004095509521953F4F4F4F5F4F6F4F7F4FF7
:101320008F4F9F4F08952F923F924F925F926F92EF
:101330007F928F929F92AF92BF92CF92DF92EF9265
:10134000FF920F931F93CF93DF93CDB7DEB7CA1BE6
:10135000DB0B0FB6F894DEBF0FBECDBF19942A8801
:10136000398848885F846E847D848C849B84AA84B9
:10137000B984C884DF80EE80FD800C811B81AA8146
:10138000B981CE0FD11D0FB6F894DEBF0FBECDBF11
:10139000ED0108950F93083090F0982F872F762F46
:1013A000652F542F432F322F22270850F4CF220FBE
:1013B000331F441F551F661F771F881F991F0A95EB
:1013C000B2F70F91089597FB10F8169400080F9349
:1013D000083098F00850232F342F452F562F672FB1
:1013E000782F892F902DF4CF059497958795779531
:1013F000679557954795379527950A95AAF70F91C1
:1014000008952A0D3B1D4C1D5D1D6E1D7F1D801F07
:10141000911F08950024A7FD00942A0F301D401D40
:10142000501D601D701D801D901D08952A193B09D7
:101430004C095D096E097F09800B910B08952A15EF
:101440003B054C055D056E057F05800791070895F6
:101450000024A7FD00942A173005400550056005BB
:1014600070058005900508955058BB27AA270E9453
:101470004C8A0C94B78C0E94A98C38F00E94B08CD6
:1014800020F039F49F3F19F426F40C946F8C0EF47D
:10149000E095E7FB0C94698CE92F0E94C88C58F307
:1014A000BA17620773078407950720F079F4A6F549
:1014B0000C94EA8C0EF4E0950B2EBA2FA02D0B01A4
:1014C000B90190010C01CA01A0011124FF27591B89
:1014D00099F0593F50F4503E68F11A16F040A22F8F
:1014E000232F342F4427585FF3CF46953795279500
:1014F000A795F0405395C9F77EF41F16BA0B620BFF
:10150000730B840BBAF09150A1F0FF0FBB1F661F45
:10151000771F881FC2F70EC0BA0F621F731F841F88
:1015200048F4879577956795B795F7959E3F08F0AE
:10153000B0CF9395880F08F09927EE0F9795879570
:1015400008950E94A98C60F080E891E009F49EEF74
:101550000E94B08C28F040E851E071F45EEF0CC0BE
:101560000C946F8C0C94EA8CE92FE0780E94C88C64
:1015700040F3092E052AB1F3261737074807590704
:1015800038F00E2E07F8E02569F0E025E0640AC087
:10159000EF6307F8009407FADB01B9019D01DC0154
:1015A000CA01AD01EF930E942F8B0E94B78C0E945D
:1015B000E48A5F91552339F02BED3FE049E450FD7B
:1015C00049EC0C94358A0895DF93DD27B92FBF7756
:1015D00040E85FE31616170648075B0718F4D92F93
:1015E0000E94F68C9F938F937F936F930E94818EBE
:1015F000E4E4F1E00E94828C0E94B78C2F913F912D
:101600004F915F910E94D78DDD2351F09058A2EA4F
:101610002AED3FE049EC5FE3D0785D270E944C8AD9
:10162000DF910C94B78C0E94458C08F481E00895FA
:101630000E942C8B0C94B78C0E94B08C58F00E94A6
:10164000A98C40F029F45F3F29F00C94698C51116A
:101650000C94EB8C0C946F8C0E94C88C68F39923CB
:10166000B1F3552391F3951B550BBB27AA2762179E
:101670007307840738F09F5F5F4F220F331F441FAB
:10168000AA1FA9F335D00E2E3AF0E0E832D09150DF
:101690005040E695001CCAF72BD0FE2F29D0660FCC
:1016A000771F881FBB1F261737074807AB07B0E80F
:1016B00009F0BB0B802DBF01FF2793585F4F3AF015
:1016C0009E3F510578F00C94698C0C94EB8C5F3F35
:1016D000E4F3983ED4F3869577956795B795F7959B
:1016E0009F5FC9F7880F911D9695879597F9089583
:1016F000E1E0660F771F881FBB1F6217730784071F
:10170000BA0720F0621B730B840BBA0BEE1F88F72D
:10171000E095089529F416F00C94698C0C94EA8CE9
:101720000C946F8C0E94D08CA8F39638A0F707F821
:101730000F92E8942BE33AEA48EB5FE70E94DA8DD8
:101740000F920F920F924DB75EB70F920E94908D3D
:10175000E1E7F1E00E94828C4F915F91EF91FF9160
:10176000E595EE1FFF1F49F0FE57E0684427EE0F96
:10177000441FFA95E1F74195550B0E94028D0F9099
:1017800007FE0C94F68C089597FB16F40E94728C59
:101790000C94088CE89409C097FB3EF490958095D2
:1017A000709561957F4F8F4F9F4F9923A9F0F92F27
:1017B00096E9BB279395F695879577956795B795A5
:1017C000F111F8CFFAF4BB0F11F460FF1BC06F5F8B
:1017D0007F4F8F4F9F4F16C0882311F096E911C09D
:1017E000772321F09EE8872F762F05C0662371F0BE
:1017F00096E8862F70E060E02AF09A95660F771FD2
:10180000881FDAF7880F9695879597F90895E894D9
:10181000F92F96EBFF2381F0121613061406440BE2
:101820009395F69587957795679557954040FF2353
:10183000B9F71BC099270895882351F49850D2F71F
:10184000872B762F652F542F432F322F20E0B1F3B3
:10185000121613061406440B88233AF09A95440F87
:10186000551F661F771F881FCAF755234AF4440F78
:10187000551F11F460FF04C06F5F7F4F8F4F9F4F64
:10188000880F9695879597F90895990F0008550F39
:10189000AA0BE0E8FEEF16161706E807F907C0F0F6
:1018A00012161306E407F50798F0621B730B840BFE
:1018B000950B39F40A2661F0232B242B252B21F4D8
:1018C00008950A2609F4A140A6958FEF811D811D78
:1018D000089597F99F6780E870E060E008959FEFB2
:1018E00080EC089590958095709560955095409501
:1018F000309521953F4F4F4F5F4F6F4F7F4F8F4F29
:101900009F4F0895DF93CF931F930F93FF92EF9212
:10191000DF927B018C01689406C0DA2EEF010E94F1
:10192000D78DFE01E894A59125913591459155916A
:10193000A6F3EF010E944C8AFE019701A801DA94F8
:1019400069F7DF90EF90FF900F911F91CF91DF919A
:10195000089500240A941616170618060906089515
:1019600000240A9412161306140605060895092E7B
:101970000394000C11F4882352F0BB0F40F4BF2BEA
:1019800011F460FF04C06F5F7F4F8F4F9F4F08952A
:1019900057FD9058440F551F59F05F3F71F0479520
:1019A000880F97FB991F61F09F3F79F08795089505
:1019B000121613061406551FF2CF4695F1DF08C024
:1019C000161617061806991FF1CF86957105610541
:1019D00008940895E894BB2766277727CB0197F9E9
:1019E00008950E94458C08F48FEF08959B01AC0187
:1019F00060E070E080E89FE30C94188B0C94698C95
:101A00000C94858E0E94D08CD8F39923C9F3940F3F
:101A1000511DA3F39150504094F059F0882332F0B7
:101A2000660F771F881F91505040C1F79E3F5105A8
:101A30002CF7880F911D9695879597F908955F3F2C
:101A4000ACF0983E9CF0BB27869577956795B79547
:101A500008F4B1609395C1F7BB0F58F711F460FF1C
:101A6000E8CF6F5F7F4F8F4F9F4FE3CF0C94EB8C8E
:101A70000E94488D29ED3BE54EED5EE30C94C48D4C
:101A800016F00C94858E0C946F8C68940C94698C71
:101A90000E94D08CA8F39923C1F3AEF3DF93CF93C8
:101AA0001F930F93FF92C92FDD2788232AF02197D8
:101AB000660F771F881FDAF720E030E040E85FEB21
:101AC0009FE3883920F0803E38F021968F770E947E
:101AD000358AE9E9F1E004C00E94358AE6ECF1E0DC
:101AE0000E94828C8B01BE01EC01FB2E6F577109A5
:101AF0007595771F880B990B0E94CC8B28E132E7F4
:101B000041E35FE30E94D78DAF2D9801AE01FF90B6
:101B10000F911F91CF91DF910E944C8A0C94B78C4A
:101B2000FA01DC01AA0FBB1F9B01AC01BF5728F4CF
:101B3000222733274427507820C0B75190F4AB2F89
:101B40000024469537952795011CA395D2F30020D4
:101B500071F0220F331F441FB395DAF30ED00C94AB
:101B6000348A61307105A0E88A07B94630F49B01D8
:101B7000AC016627772788279078309621F020835C
:101B800031834283538308950E94D78D0C94B78C80
:101B90000E94A98C38F00E94B08C20F0952311F09F
:101BA0000C94698C0C946F8C11240C94EB8C0E9417
:101BB000C88C70F3959FC1F3950F50E0551F629F3D
:101BC000F001729FBB27F00DB11D639FAA27F00D96
:101BD000B11DAA1F649F6627B00DA11D661F829FBD
:101BE0002227B00DA11D621F739FB00DA11D621FA2
:101BF000839FA00D611D221F749F3327A00D611DBF
:101C0000231F849F600D211D822F762F6A2F1124A0
